:020000040000FA
:10000000405A001081030000890300008B030000A8
:100010008D0300008F030000910300007E90FFEF2E
:10002000000000000000000000000000930300003A
:1000300095030000000000009703000099030000F2
:100040009B030000C10300009B0300009B03000012
:100050009B0300009B0300009B0300009B03000028
:100060009B0300009B0300009B0300009B03000018
:100070009B0300009B0300009B0300009B03000008
:100080009B0300009B0300009B0300009B030000F8
:100090009B0300009B0300009B0300009B030000E8
:1000A000CB1700009B0300009B0300009B03000094
:1000B0009B0300009B0300009B0300009B030000C8
:1000C0009B0300009B0300009B0300009B030000B8
:1000D0009B0300009B0300009B0300009B030000A8
:1000E0009B03000000F002F800F05EF80AA090E820
:1000F000000C82448344AAF10107DA4501D100F0E3
:1001000053F8AFF2090EBAE80F0013F0010F18BF51
:10011000FB1A43F0010318471C3400003C34000074
:100120000A444FF0000C10F8013B13F0070408BF1D
:1001300010F8014B1D1108BF10F8015B641E05D0BB
:1001400010F8016B641E01F8016BF9D113F0080F70
:100150001EBF10F8014BAD1C0C1B09D16D1E58BF02
:1001600001F801CBFAD505E014F8016B01F8016B39
:100170006D1EF9D59142D6D37047000000230024AC
:1001800000250026103A28BF78C1FBD8520728BFA7
:1001900030C148BF0B6070471FB59DE8030002F0F7
:1001A000CDFD1FBD10B510BD02F024FE1146FFF7B6
:1001B000F3FF00F0AFFB02F042FE03B4FFF7F2FFE3
:1001C00003BC02F073FE0000D0F800D0D0F804F0B9
:1001D000024600200B21C30700D0802303EB500010
:1001E00012F8013B491E184409B2C0B20029F2D1ED
:1001F000704770477047704770477047443322110B
:10020000FFB559A60446E1CE8DE8E100022902DAE5
:10021000002004B0F0BD6018002100F8011D6946FF
:10022000B3FBF2F502FB1535B3FBF2F34D5D00F8BD
:10023000015DA042F4D8ECE702460020342A01D048
:100240003F2A06D14A78342A03D18978322900D14D
:100250000120704702004FF0000009D0012A0ED0A3
:10026000022A04D1C978662907D0462905D07047EB
:10027000C9786B2901D04B29F9D101207047C97881
:100280006E29FAD04E29F8D07047F0B50646002006
:10029000044605460346F25CA2F13007092F01D857
:1002A000FDB209E0A2F14107052F02D8373AD5B2D5
:1002B00002E0613A052A05D95B1CDBB205EB0414A8
:1002C000042BE8D30988A14200D10120F0BD10B56C
:1002D00002F0D5FA2848294C006840B102F03DFCF4
:1002E000A0F5C820206002F038FC606010BD02F06C
:1002F00034FC6FF448210844206002F02EFC6FF4B7
:10030000C8210844F1E7F8B51C4D034600242E68C7
:100310007018696887188F4200D9881A00920246BF
:10032000304602F037FB2046F8BD0B460146134825
:1003300010B500680024184401F0B4FF204610BD39
:1003400070B500220D4C134608340AE0E65C855C6B
:100350005B1C7540DBB28554402B00D30023521C3C
:10036000D2B28A42F2D370BD3031323334353637AF
:100370003839414243444546CC0000101401001076
:100380000948804709480047FEE7FEE7FEE7FEE729
:10039000FEE7FEE7FEE7FEE7FEE7FEE70448054965
:1003A000054A064B7047000085190000E500000073
:1003B000400A0010405A0010404A0010404A001005
:1003C00010B54FF040210120086001F0D0FD10BDB4
:1003D0000648022141600021016741611D22C2607F
:1003E000C163012141600020704700000000094006
:1003F00010B591FBF2F491FBF2F302FB1411C0E98A
:10040000003110BDA71B000010B50178427801EB48
:10041000810102EB4101C902A1F5C0318AB2C17864
:100420000479303901EB810104EB41014901A1F567
:10043000C06101F4FC611143C27980796FF02F0330
:10044000303800EB800003EB40001044C0F3440060
:10045000084310BDF0B58DB004463022F949684616
:1004600002F01FFCE079A17A00EB4002C2EBC01061
:1004700001EBC001207A64225043627A102302EB20
:10048000820200EB420008444002742100EB41204C
:100490002179627901EB810103EB4101114480B2C2
:1004A00001F01F010143237800206D4655F82020FC
:1004B0001678B3420DD166785778BE4209D1A67836
:1004C0009278964205D14001203000F4F07001434B
:1004D00003E0401CC0B20C28E8D30DB00846F0BDC4
:1004E000D94910B5486980040CD4D84A906843F6BD
:1004F00098239468241A9C42FBD34869800401D451
:10050000012010BD052001F0CBFA002010BD70B510
:10051000CE4CA668042001F0C3FACD4D03E000BF25
:10052000FFF7DEFF48B1A068801BA842F8D308E0BF
:10053000FFF7D6FF08B1012070BDA068801BA8425C
:10054000F6D3002070BD10B5092001F0A9FAC14909
:100550000120487010BD2DE9F041002506462C46CB
:10056000BD4F0BE040222146BB48FFF7DEFE0020D6
:100570003958001D0D444028FAD34034B442F1D319
:100580002846BDE8F081B5A086B00FC88DE80F0001
:10059000B6A0B74900680490086800264FF6FF022D
:1005A0001040B44A40F4807010430860B249B34F21
:1005B0004FF4C8200E60B3493860B1480860B249B2
:1005C0004012B24D0860F8202870FF206870A870B3
:1005D000AF48B046D0F8109001F044FC9D4CDFF8D5
:1005E000B4A24FF0010B606801280FD14FF4C8206E
:1005F000FFF7B1FFE0B3D4F8042020204346514672
:1006000051F822703B54401C4028F9D36268002006
:100610005AF822102A180B5C401C82F8003460281B
:10062000F8D300F0D1FF012000F0F9FF4FF4E17A98
:100630005546514640F2491001F079FC294640F2F6
:100640009F1001F074FCA04601F040F998F80100F9
:1006500045460028F8D100218FA000F071FD04006C
:10066000F2D08E49087A66287DD046287BD0DCE01F
:10067000FFE784F800B003223B680221104601EB3B
:10068000932740F6FF7E13E0B0EB932F01D3714622
:1006900000E0411CC0F3032C4CEA0118A85405EB00
:1006A000020C09098CF80180801C8CF80210D21C05
:1006B0008742E9D8402240F204416748FFF735FEFF
:1006C00065498878032802D3584681F802B0C0B241
:1006D00004AA5746125C60685AF8203083F8432019
:1006E0005AF8203083F827204B786A4602EB131320
:1006F0005AF820C01B788CF844305AF820C08CF887
:1007000029304B7857F820C003F00F031DF8033051
:100710008CF8453057F820C08CF82E300B7857F8FD
:1007200020C002EB13131B788CF8463057F820C01A
:100730008CF83030097801F00F01515C57F8202017
:1007400082F8471057F8202082F8321057F820001E
:100750004030FFF73DFD616857F8211081F82D000A
:100760003D480C3000E01CE0FFF774FE616857F86C
:100770002120A2F8580057F82120A2F8520057F87B
:100780002110A1F8500034481C30FFF73DFE61688D
:1007900057F82120A2F8560057F82110A1F84E0072
:1007A00034E7487A722801D052283ED1887A6D28E1
:1007B00006D04D2804D0782801D0582835D10126FC
:1007C00036480078662801D046282ED140221101F3
:1007D0002148FFF7AAFD012E03D140211E48FFF753
:1007E000AFFD1D492D484F7A001D091DFFF74DFD36
:1007F000D8B16868A84628B14FF4C820FFF7ABFE0F
:10080000F8B112E038462549FFF716FD50B11248FD
:1008100022498079FFF71EFD20B14FF4C820FFF771
:100820009AFE28B1092001F03BF9FFF78CFE0BE797
:100830000A2001F035F900273D46072001F030F984
:100840003EE056E00033000000800920000009402F
:1008500080841E00C8000010BC0700103031323305
:100860003435363738394142434445464B4E4600CD
:100870000CED00E00000FA0510010010000100106E
:10088000005C0600F8000010FC000010BC01001025
:1008900030330000C00000104634320068080010F9
:1008A000A8050DD1204600F025FC0446A0F5706097
:1008B000FF381ED0032C1CD340F6F870844218D2A7
:1008C000402229464848FFF730FD4035012E03D12C
:1008D00040214548FFF734FD09EB0700402242491B
:1008E00000F0EEFC0720403701F0DAF8002DE7D0E9
:1008F000D6E70B2001F0D4F85446514640F29F1041
:1009000001F015FB214640F2491001F010FB88F878
:1009100001B099E601F036F801F040F9FFF758FD13
:1009200001F084F8002001F0BBF801F045FB2F4EE8
:1009300070692F4D2F4CDFF8C08040034FF0000747
:1009400002D5FFF7CDFD70B3042001F0A9F870695E
:10095000800414D4FFF7DBFD28B3FFF7D8FD10B3F4
:10096000FFF7D5FDF8B1042001F09AF8A0684146E0
:100970007269920403D4A268121A8A42F8D3A0685A
:1009800042F21071A268121A8A42FBD3706B10F007
:10099000004F14D501206860FFF799FC4FF4C82080
:1009A000FFF7D9FD58B100F0BFFC00284FF002005E
:1009B0000AD001F075F86868401C02D00AE06F6048
:1009C000F1E700F0ABFC05E001F06AF86868401C54
:1009D00000D16F60FFF77BFCA0684146A268121A45
:1009E0008A42FBD3FFF7CFFDBC070010008009202F
:1009F000C80000100000094080841E002DE9F84363
:100A000000250E460446FE4FA84634E0B4F5007FAC
:100A100019D2132C0DD0142C0ED0B4F5FF7F0ED0AC
:100A2000A4F58070FF380CD03E2C1CD8F548005D32
:100A300012E097F820000FE0388C000A0CE05520F7
:100A40000AE0AA2008E0B4F5006F08D2EE4820447E
:100A5000A0F5805090F8000E8DF8000005E0EB48FE
:100A6000006801280BD08DF80080E9499DF800004E
:100A7000641C48556D1CB542C8D3BDE8F8830122FB
:100A8000A4F500616846FFF750FCEEE770B5DC4D59
:100A90002C6B402C00D94024E86AE96902198A428B
:100AA00002D90C1A042169702146FFF7A7FF2246DC
:100AB000D749822000F05FFEE86A2044E862286B94
:100AC000011BD348296300F19F008268A2EB040256
:100AD000826005D06978022901D00021017370BDC0
:100AE00003216970F9E7CA4910B59F31C948086008
:100AF0000D22822000F03FFEC1490520487010BD44
:100B000070B50D46C4494A69520302D5496D49057D
:100B100021D4B0F5007F1ED3C04BB94CB0F5006FA7
:100B20001AD29968A269891ABD4A914204D3996878
:100B3000A161002161606161B54A00214032B24B80
:100B400007E044181C44565CA4F58054491C84F802
:100B5000006EA942F5D370BD616921B99968A161A0
:100B600099686161A060A949096829B10129F2D198
:100B7000AC4909780029EED199686269891AAA4AB4
:100B8000914217D29968A16199686161A168401A80
:100B90006168884203D9616A884200D26060062099
:100BA00000F07EFF2A466168BDE8704098484030FA
:100BB000FFF7A9BBBDE870400C2000F071BF10B575
:100BC0008F4CA178E06A4218E1698A4206D9081A76
:100BD000A07005206070022000F088FDA178E06A16
:100BE000FFF78EFFA178E06A0844E062206B421AAA
:100BF0008748226300F19F008368A3EB01018160B5
:100C000002D06178052904D100210173BDE81040AC
:100C100069E710BD2DE9F041794CA178E06A4218EE
:100C2000E1698A4206D9081AA07005206070022086
:100C300000F05CFD764B0021A07803F14005E26AEC
:100C400008E056186F5C9E5DBE4202D00021A16292
:100C500002E0491C8142F4D31118E162216B0A1AA7
:100C60006B49226301F19F018B68A3EB0000886050
:100C700002D06078052808D1A06A20B1002008734E
:100C8000BDE8F0412FE70120F9E7BDE8F0816048B9
:100C900010B58030D0F81110027D09BA21F0FF01A3
:100CA0001143574A4902D162C18A49BA49021163C4
:100CB000806888420DD0822000F018FD022000F0EC
:100CC00015FD534902209F310873FFF70CFF0020E8
:100CD00010BD012010BD70B54D48803002248168E0
:100CE00000F11F0529B1007B000607D4022000F0A7
:100CF000FDFC2C73FFF7F7FE002070BD012070BDD6
:100D000010B543483E4C80308068A178884200D2BC
:100D1000A0703F49A2784031822000F02CFD0320D2
:100D200060703B48A2789F308168891A81600021F9
:100D3000017310BD364810B58030816839B1007B31
:100D4000000601D5822000E0022000F0CFFC3049EF
:100D500000209F310873BDE81040C4E610B5FFF7CE
:100D6000BAFF00281FD02A487021403002220170AB
:100D7000002141708270C1700171417181710A223C
:100D8000C271017241728172C172302202730122FA
:100D900042738173C17301744174194912208870C0
:100DA000BDE81040ACE710BD1CB5FFF794FF00286C
:100DB00069D01E480A220621008883B26846FFF7E0
:100DC0001FFA134800224030802302704370827063
:100DD0000121C1702021017143718271C2714122D0
:100DE0000272542242724F2282724C22C2720173EA
:100DF000417381734622C17302745023437417E018
:100E0000DC000010C0320000BC010010CC0000105B
:100E1000BC070010555342530080092000000940D0
:100E2000A0860100C800001020A1070004040000F3
:100E3000722383746923C3746E230375742343750B
:100E40008175C2756C2202766122427673228276A7
:100E50006822C276017741778177C1779DF80110CA
:100E600080F820109DF8021080F821109DF80310E2
:100E700080F822109DF8041080F82310DC4924200B
:100E80008870FFF73DFF1CBD10B5FFF724FF002859
:100E90000CD0D84803210170002141708170C170CD
:100EA000D34904208870BDE8104029E710BD10B573
:100EB000FFF711FF002810D0CE4800210622017054
:100EC00042708170C170017141718171C171C849F5
:100ED00008208870BDE8104012E710BD10B5FFF77C
:100EE000FAFE002815D0C24AC248116A491E0B0EEC
:100EF00003700B0C43700B0A8370C17000210171E9
:100F0000417102238371C17108209070BDE81040C7
:100F1000F6E610BD10B5FFF7DEFE002819D0B54883
:100F20000021B34B0170417081700822C2701A6AAF
:100F3000140E0471140C4471140A8471C2710222DB
:100F4000027241728272C1720C209870BDE810402A
:100F5000D6E610BD2DE9F041A54DA64C0021A8789C
:100F60004034A44A02E0535C6354491C0346814266
:100F7000F9D31F2B72D120689F4988426ED19D4EB4
:100F800060685F364FF001087060A068B060607BF9
:100F900018B9A07B08B1102802D986F80C8059E056
:100FA000E07B1E28F9D00FDC12282ED005DC48B3D8
:100FB0000328F2D1BDE8F041D0E61528EDD01A287B
:100FC000EBD1BDE8F0415FE702272A2828D010DCEA
:100FD00023281DD025281ED02828DED1FFF757FE54
:100FE000002826D0207B000618D56F70BDE8F041A0
:100FF0004CE52F281ED05528CFD05A28CDD1BDE89A
:10100000F04154E7BDE8F04194E6BDE8F041CBE69D
:10101000BDE8F0417EE7BDE8F0415FE7022016E061
:10102000FFF735FE002804D0207B00060ED485F89B
:1010300001802AE6FFF72BFE0028FAD0207B00066D
:1010400004D485F80180C5F828801EE6822000F0CF
:101050004DFB3773BDE8F04145E5FFE7822000F026
:1010600045FB022000F042FB062068700DE6604858
:1010700010B54178022908D003290ED004290FD0D9
:10108000052901D10021417010BD5A484030C07B74
:101090002828F9D1BDE81040F8E4BDE8104022E569
:1010A000822000F023FBF8E710B55249022000F03F
:1010B00031FB4F498870487858B101280CD0022084
:1010C00000F014FB4B4902205F310873BDE810406B
:1010D00009E5BDE810403DE746484030C07B2A287E
:1010E00004D02F2805D1BDE8104093E5BDE810409D
:1010F00065E510BDFFB50246002002EB4205014642
:101100004FF400666C4603AA6B1844F82130B342D2
:1011100002DD002004B0F0BD384F07EB6307DB07AA
:101120003F78575401D03B095354535C8F0003F070
:101130000F035354BB40491C18440329E4DBE9E77F
:10114000F0B505460020044602462C4B4FF40077CC
:1011500000E0641C2E5D36B102EB040C9C449CF84C
:1011600000C4B445F5D0032C3DD302F5806018448B
:10117000047F457FC67F04EB0524857F2D0405EBA6
:1011800006652C4451EA040529D021B9184949685B
:1011900040318C4223D8174C00216C3455181D4423
:1011A00095F800546554491C0C29F7D3817EC27E02
:1011B00001EB0221027D407D120402EB00600C185D
:1011C0002046FFF797FF40F6F57501E0FFF792FF25
:1011D000C11EA942FAD3A0F57061FF3901D00020E9
:1011E000F0BD2046F0BD2032BA42B3D3F0BD0000BE
:1011F000DC000010FC07001055534243BC010010F6
:1012000030B4514C4F4A0323C4F8B031136843F44F
:10121000803313604D4A30BC104710B572B633248A
:101220004B4B10C307C34B484FF47A710068B0FBB7
:10123000F1F01860191D4648FFF7E2FF62B610BDD5
:10124000434A32231360C2E9010142484FF47A71E4
:101250000068B0FBF1F0D06002F114011046CFE756
:101260003B4A34231360C2E901013A484FF47A71D2
:101270000068B0FBF1F0D06002F114011046BFE746
:1012800010B572B60424344951F82420824212D990
:101290003149783951F82410814207D12146084656
:1012A000FFF7CEFF21460846FFF7DAFF2146084642
:1012B000FFF7C6FF02E0641C1D2CE5D962B610BD25
:1012C0002DE9F041254C236803B92060204D002012
:1012D0002835636803E00F5C1E18401CAF55904230
:1012E000F9D398184FF480766060B04213D120682B
:1012F000FFF7C6FF164D1435286800B1FEE7144904
:10130000324628312068FFF788FF286800B1FEE7E1
:101310000020606020600020BDE8F08110494FF49B
:1013200080400860FEF750BF00214FF480404FF42A
:10133000D02208C890421944FBD309B1002070475D
:101340000120704788C10F4000C00F40F11FFF1FF0
:101350007408001094010010A83300005C01001014
:1013600008ED00E0664800214FF001128180017015
:101370004170C0E90221704761491C31002000F032
:10138000C9B910B55E4C1434A288402A00D9402255
:101390008020216800F0EFF9216801442160A188D4
:1013A000081AA08010BD10B5554C002014342168D7
:1013B00000F0B0F9216801442160A188081AA080DA
:1013C00010BD00221146802000F0D5B94D49002003
:1013D00000F0A0B92DE9F041494C00271C34484DDC
:1013E0002178A4F10806082863D2DFE800F062043F
:1013F000647262628381FFF7BFFF2078C00900F04A
:1014000056F9E088B0802078C0F34111F1BB6178D3
:101410000C294AD2DFE801F00609490B49101A1DD0
:101420001F25314201F0A4FD4DE0002000E0012025
:1014300001F0DEFD50B306E010F01F0F35D1A078AB
:1014400040F080002870BDE8F041BAE701F054FD9B
:1014500039E000202AE010F01F0F26D12848401C58
:101460001AE010F01F0F20D101F00AFE70B1FFF753
:10147000A8FFBDE8F04100F071BA00F01F0001289C
:1014800013D1687810B12079A97800E00DE0884286
:101490000BD21B491031084430601CE000F01F00E3
:1014A000012802D101F094FEC4E7802000F01EF96B
:1014B000B780BDE8F081080608D4B0880028F8D0CD
:1014C000FFF771FFB0880028EFD0F2E7BDE8F041E8
:1014D0007CE7080602D5BDE8F04152E7287801060E
:1014E000E7D500F07F002870BDE8F04100F041B87A
:1014F000802000E00020BDE8F04100F001B90000CC
:10150000680100109C09001001460007C00E090682
:1015100000D5401C7047DD491022C1F80822C1F8EF
:10152000100200BFD1F80002C006FBD57047D74AB1
:101530001023C2F80832C2F8100200BFD2F800022D
:10154000C006FBD5C2F80832C2F81012D2F8000269
:10155000C006FBD57047CD493022C1F80822C1F83A
:10156000100200BFD1F800028006FBD5D1F81402AA
:10157000704730B5C649C74D41EA00442146284668
:10158000FFF7D5FF21462846BDE83040CFE7BF48EA
:101590000021C0F848124021C0F84C120122C0F8C6
:1015A0004822C0F84C1200BFD0F80012C905FBD584
:1015B0004FF0FF31C0F83812C0F83412C0F80812EA
:1015C0000C21C0F80412704730B5B34C1A202060CB
:1015D000221D116830EA0101FBD1B04901234B679C
:1015E0008B67AA4D0023C5F810318A23C1F8F83063
:1015F0002060116830EA0101FBD14FF0E0214FF08B
:101600008070C1F88002A64B202283F80024C1F824
:101610000001FFF7BCFFBDE830400020A9E710B58E
:10162000040001D0012000E000204FF4807141EA65
:1016300000419C48FFF77BFF9B494FF480200CB191
:10164000886310BDC86310BD704710B500B101209C
:101650004FF4807444EA00419448FFF768FF8B48D8
:101660000321C0F8441200BFD0F80012C905FBD511
:10167000C0F8084210BD10B502468078FFF744FF5D
:101680008249D1F84432012484402343C1F84432D2
:10169000C1F848029088C1F84C0200BFD1F800029E
:1016A000C005FBD54FF48070C1F8080210BD70472B
:1016B00000B5FFF729FF7E495DF804EB41EA0040E1
:1016C000891334E700B5FFF71FFF79495DF804EB94
:1016D00041EA004077492AE700B5FFF715FF744952
:1016E0005DF804EB41EA0040891320E700B5FFF7FD
:1016F0000BFF6F495DF804EB41EA00406E4916E7C5
:1017000000B5FFF701FF6A495DF804EB41EA0040CC
:1017100089130CE700F00F02012370B503EB82037D
:101720005A4AC2F8283200BFD2F820321C05FBD535
:10173000C3F309030024DD1C05E000BFD2F81862E2
:1017400041F8046B641CB4EB950FF7D30021C2F889
:10175000281241F24821C140C9070AD1FFF7D4FE3F
:101760004FF4A06141EA0040FFF7D5FE5348FFF770
:10177000D2FE184670BD70B513460546434C00F0C6
:101780000F00022202EB8000C4F82802C4F82432C1
:101790000020DA1C05E000BF51F8046BC4F81C629D
:1017A000401CB0EB920FF7D30020C4F82802284663
:1017B000FFF7AAFE4FF4A06141EA0040FFF7ABFE3D
:1017C0003F48FFF7A8FE184670BD2DE9F0412F4DA8
:1017D000D5F80032C5F80832180721D53148FFF78F
:1017E0009AFE3848FFF7B7FEC10605D5FFF7CFFED2
:1017F000BDE8F04100F0A3B8810705D5BDE8F04190
:1018000000F0010000F095B8010709D5400703D5A5
:10181000BDE8F04100F09AB8BDE8F04100F09DB895
:10182000294E58074FF001071CD4BDE8F081002471
:10183000D5F8302207FA04F10A4210D06008C5F842
:10184000381200BFD5F800128906FBD5D5F814125E
:10185000E2070CD056F8201009B103208847641C19
:10186000202CE5D3D5F830020028E0D1DDE73CB9E3
:10187000490705D5316819B1012088470124D7E708
:1018800056F820100029EAD00220E7E700C008201F
:10189000000180000005D000F4CF082000C0024005
:1018A00018E000E00005FE00008009200005D800D7
:1018B0000005400000012000000101000005F200C9
:1018C0000005FA000002FE00C434000070B5284C88
:1018D000607820B30026274D012810D002280DD1B2
:1018E000A8686168401A2449884215D32348406B90
:1018F000400011D50120FFF792FE667070BDA86808
:101900006168401A1E498842F8D30020FFF787FE1D
:10191000A86860600220607026700C2005E02078C6
:101920000028EBD1012020700D20BDE8704000F0B0
:10193000B7B8002802D10E4901204870704710B591
:10194000FFF710FD0A490020487010BD084801212A
:1019500041700849896841607047704770470228A4
:1019600003D0032803D1FFF782BBFFF79DBB70476D
:101970008C01001000000940A086010000800920B1
:1019800040420F0030B52648244A2021C0F8A0115B
:10199000D0F8A0114906FBD50121C0F80C1109238C
:1019A000C0F88430C0F88010AA23C0F88C305524C9
:1019B000C0F88C40D0F888506D05FBD52325C0F8C1
:1019C000A450C0F8A010C0F8AC30C0F8AC4000BFC4
:1019D000D0F8A8305B05FBD540F20113C0F8043104
:1019E00040F20123C0F80831C0F800110421C0F80A
:1019F000A8110C49C0F8C4100021C0F8C811D0F8D3
:101A0000B03143F00303C0F8B03145F23A0303604C
:101A1000054801600D20106030BD000088C10F40F6
:101A200000C00F40CE9FF8F708ED00E0002070479F
:101A30005849C20702D04FF000728A67800702D56A
:101A40004FF080608867002070475249C20702D07B
:101A50004FF00072CA67800702D54FF08060C867F8
:101A600000207047014600204A4ACB0703D0536F3D
:101A70009B0100D50120890704D5516F490101D58B
:101A800040F00200704710B50446FFF7EBFF034635
:101A9000FFF7DBFF24EA0300FFF7CAFF002010BDB9
:101AA00010B53D4B38B159680424042906D2DFE84B
:101AB00001F0061D375400205860986010BD0428BE
:101AC00007D005280AD0012402285ED001284CD076
:101AD00010BD0320FFF7B9FF01201EE0BDE8104054
:101AE0000120B2E7FFF7A4FF5C6010BD062808D014
:101AF0000328FAD00928ECD00D280AD00C28E8D009
:101B000010BD0320FFF7A1FF0220FFF791FF022085
:101B100021E00320FFF799FF0220BDE8104087E78E
:101B2000062808D00A280FD009281ED00C28D0D0AB
:101B30000D28EED010BD986810F01F0F00F10100C5
:101B40009860F7D102201DE00320FFF77EFF0120FF
:101B5000FFF76EFF0320586010BD07280AD00A283F
:101B6000B7D00B2811D00928F6D10320FFF76DFF5D
:101B70000120B7E7986810F01F0F00F1010098608E
:101B8000EAD10120BDE810407DE70320FFF75DFFAB
:101B90000220A7E700800920A4010010F0B5AB499E
:101BA000032008630020C1F80801A94804228265C7
:101BB000026C42F004020264A64A8A6600220A61AC
:101BC0001022C261026822F0100202600322C1F8F2
:101BD0007022C1F8742200224A644FF400328261FC
:101BE000026842F4003202600922C1F80021C1F803
:101BF00004211022C1F8D42052048263026A42F404
:101C0000001202620D22C1F8D020C1F8E0200022AB
:101C1000C1F8F4204FF00052C263026A42F0005251
:101C200002620022C1F8F0204FF08052C263026AC3
:101C300042F0805202621022CA6702048261026886
:101C400042F0004202601022C1F81421202787656B
:101C5000026C42F0200202641022C1F81C21802292
:101C6000C265026C22F0800202649026C1F8FC601A
:101C70000204C263026A22F0004202621022C1F82A
:101C8000DC20D204C263026A22F400020262012252
:101C90000A66CA654A660323C1F8D8300523C1F82D
:101CA000E4308A601123CB60CA630B640224C1F85C
:101CB00020411225C1F824510C604D600C604D602C
:101CC00010248C659405C461046844F480040460A5
:101CD0000124CC630B641023C1F82C31CB14C365F1
:101CE000036C43F4006303641023C1F830318B1498
:101CF000C365036C43F48053036440F282234B6258
:101D00009A240C62CB6110234B618761036843F016
:101D10002003036010238B6140248461036843F037
:101D20004003036001230B67CB6640F20243CB62A2
:101D30008B621023C1F8E83093068363056A45F08F
:101D4000806505621025C1F8EC50D506C563056AAB
:101D500025F0006505624E635503C561056825F4ED
:101D6000005505600025C1F8E4515506C567056EAC
:101D700045F0007505660025C1F8E851C367036E9C
:101D800043F0806303668A23C1F8F8300823C1F862
:101D9000C8309504C563066A46F48026066210269C
:101DA000C1F828610E15C665066C26F480660664C7
:101DB0000126C1F88060C1F88460C1F89060C1F864
:101DC000A060C1F8A460C1F8A860C1F8BC6000269A
:101DD000C1F81861C465046C44F0400404640B65E8
:101DE0001405C461046824F480140460CB64D40432
:101DF000C461046824F4002404608B64C561046831
:101E000024F4802404600024C1F80C418365036C31
:101E100043F008030364C1F8104110238365036C89
:101E200043F0100303640C480C4B0068984204D143
:101E300041F8B82F8A60CA60F0BD094A9042FBD1D0
:101E4000812041F8B80F8860C860F0BD00C0024032
:101E5000008009200200010064010010473F19279B
:101E6000473F19474D4900200867C86002224A6170
:101E700088613022CA634A498A684A49C1E9002018
:101E80004949086049490860784649490860002086
:101E900070472DE9F04341F288320024424F434E0F
:101EA000434B904208D8642800D228B942F21072FD
:101EB000914201D8052907D28620386078463460DF
:101EC00018608620BDE8F083DFF8D490D9F8085078
:101ED000344AD2F800C0A5EB0C05D2F804C00CEBD4
:101EE0004C08C8EBCC1CB5EBCC0F06D205203860F3
:101EF0007846346018600520E4E7284D4FF0020C66
:101F0000C5F804C048B1DFF8AC80B8FBF0F0401071
:101F1000A861C5F804C001206860D9F80800C2E9CA
:101F200000013C607846346018600020CAE770B554
:101F30001C4C00250E466560FFF7ABFF1A490006F2
:101F400001D5086870BD164B06EB46022068C2EB4F
:101F5000C6129E68361AB6EBC20FFAD30F48022299
:101F60004260C26B02F0FE02C2636560E9E70C48A2
:101F700080680C490A68801A4A6802EB4203C3EB86
:101F8000C212B0EBC20F08D3044802224260C26BF7
:101F900002F0FE02C26300204860704700800040EB
:101FA00000000940B0010010D0000010D400001063
:101FB000D800001080C3C90119480621016107211A
:101FC000016000214161416202214160C168C9068E
:101FD000FCD400E08168C1684907FBD40020704749
:101FE0000F498860C868C006FCD48868704700B58F
:101FF0000B46024604E000BF12F8010BFFF7F0FFAA
:102000005B1EF9D200BD00B50B46024604E000207D
:10201000FFF7E6FF02F8010B5B1EF8D200BD0000DF
:102020000000034070B500BF00BF00BF00BF00BF8D
:1020300000BF00BF00BF00BF00BF00BF00BF00BFA8
:1020400000BF00BF00BF00BF00BF00BF00BF00BF98
:1020500000BF00BF00BF00BF00BF00BF00BF00BF88
:1020600000BF00BF00BF4025CE4CE5610620FFF752
:10207000B7FFA56100BF00BF00BF00BF00BF00BF2A
:1020800000BF00BF00BF00BF00BF00BF00BF00BF58
:1020900000BF00BF00BF00BF00BF00BF00BF00BF48
:1020A00000BF00BF00BF00BF00BF00BF00BF00BF38
:1020B00000BF00BF70BD2DE9FC5FBB4DBB4EBC4FE8
:1020C0005FEA020A8B4604464FF000080DD001A9D2
:1020D000B84800F001F980B18220286021203060EA
:1020E000784638608220BDE8FC9FC5F800807846BD
:1020F000C6F8008038600020F5E703208DF8000066
:10210000200C8DF80100200A8DF802008DF80340A4
:1021100000BF00BF00BF00BF00BF00BF00BF00BFC7
:1021200000BF00BF00BF00BF00BF00BF00BF00BFB7
:1021300000BF00BF00BF00BF00BF00BF00BF00BFA7
:1021400000BF00BF00BF00BF00BF00BF00BF00BF97
:10215000944C4FF04009C4F81C9004216846FFF7E6
:1021600046FF51465846FFF74EFFC4F8189000BF8F
:1021700000BF00BF00BF00BF00BF00BF00BF00BF67
:1021800000BF00BF00BF00BF00BF00BF00BF00BF57
:1021900000BF00BF00BF00BF00BF00BF00BF00BF47
:1021A00000BF00BF00BF00BF00BF00BF00BF9CE773
:1021B0002DE9FC47044601A97E4800F08DF87A4DD0
:1021C0007A4EDFF8EC9148B18220286022207946CF
:1021D00030608220C9F80010BDE8FC879DF804003B
:1021E000800701D4FFF71EFF20208DF80000200992
:1021F0008DF8010020018DF8020000248DF80340C5
:1022000000BF00BF00BF00BF00BF00BF00BF00BFD6
:1022100000BF00BF00BF00BF00BF00BF00BF00BFC6
:1022200000BF00BF00BF00BF00BF00BF00BF00BFB6
:1022300000BF00BF00BF00BF00BF00BF00BF00BFA6
:102240004027DFF86081C8F81C7004216846FFF75A
:10225000CEFEC8F8187000BF00BF00BF00BF00BFAF
:1022600000BF00BF00BF00BF00BF00BF00BF00BF76
:1022700000BF00BF00BF00BF00BF00BF00BF00BF66
:1022800000BF00BF00BF00BF00BF00BF00BF00BF56
:1022900000BF00BF00BF2C60794634600020C9F841
:1022A000001099E770B5414D414E3F4C2AB1FFF700
:1022B00002FF000609D5206870BD86202060092035
:1022C000286078463060862070BD0020206028603D
:1022D00078463060002070BD2DE9F041364C0F4645
:1022E0000646A56806E0A068401BB04202D3012064
:1022F000BDE8F081384600F003F80028F3D1F7E795
:1023000070B5044600BF00BF00BF00BF00BF00BFE4
:1023100000BF00BF00BF00BF00BF00BF00BF00BFC5
:1023200000BF00BF00BF00BF00BF00BF00BF00BFB5
:1023300000BF00BF00BF00BF00BF00BF00BF00BFA5
:1023400000BF00BF4025174EF5610520FFF748FE8E
:102350000020FFF745FE2070B56100BF00BF00BF41
:1023600000BF00BF00BF00BF00BF00BF00BF00BF75
:1023700000BF00BF00BF00BF00BF00BF00BF00BF65
:1023800000BF00BF00BF00BF00BF00BF00BF00BF55
:1023900000BF00BF00BF00BF00BF207800F00100F9
:1023A00070BD000000800920D0000010D400001093
:1023B000D8000010A0860100000009402DE9F34F6D
:1023C00085B0044603A9B24800F0FDF8B14DB24E05
:1023D000B24F4FF0820B18B12120C5F800B060E079
:1023E000FFF720FE42208DF800004FF0000ACDF8E4
:1023F00001A0CDF805A0ADF809A000BF00BF00BF47
:1024000000BF00BF00BF00BF00BF00BF00BF00BFD4
:1024100000BF00BF00BF00BF00BF00BF00BF00BFC4
:1024200000BF00BF00BF00BF00BF00BF00BF00BFB4
:1024300000BF00BF00BF00BF00BFDFF864924FF0D5
:102440004008C9F81C800B216846FFF7D0FDC9F889
:10245000188000BF00BF00BF00BF00BF00BF00BFAB
:1024600000BF00BF00BF00BF00BF00BF00BF00BF74
:1024700000BF00BF00BF00BF00BF00BF00BF00BF64
:1024800000BF00BF00BF00BF00BF00BF00BF00BF54
:1024900000BF03A97E4800F096F848B12220C5F895
:1024A00000B0306078463860822007B0BDE8F08F19
:1024B0009DF80C00800701D4FFF7B4FD02208DF8D1
:1024C0000000200C8DF80100200A8DF8020006980B
:1024D0008DF803408DF8040000BF00BF00BF00BFAF
:1024E00000BF00BF00BF00BF00BF00BF00BF00BFF4
:1024F00000BF00BF00BF00BF00BF00BF00BF00BFE4
:1025000000BF00BF00BF00BF00BF00BF00BF00BFD3
:1025100000BF00BF00BF00BF4446C846C9F81C400A
:1025200005216846FFF763FDC8F8184000BF00BFEB
:1025300000BF00BF00BF00BF00BF00BF00BF00BFA3
:1025400000BF00BF00BF00BF00BF00BF00BF00BF93
:1025500000BF00BF00BF00BF00BF00BF00BF00BF83
:1025600000BF00BF00BF00BF00BF00BFC5F800A094
:102570007846C6F800A03860002096E72DE9F05FA5
:10258000444EDFF81491DFF814A1150083460F467E
:102590004FF000080ED000240AE0395D0BEB040078
:1025A000FFF70CFF000602D53068BDE8F09F641C01
:1025B000AC42F2D3C6F800807946C9F8008000200A
:1025C000CAF80010F1E72DE9F041364C0F460646F7
:1025D000A56806E0A068401BB04202D30120BDE818
:1025E000F081384600F003F80028F3D1F7E770B522
:1025F000044600BF00BF00BF00BF00BF00BF00BF58
:1026000000BF00BF00BF00BF00BF00BF00BF00BFD2
:1026100000BF00BF00BF00BF00BF00BF00BF00BFC2
:1026200000BF00BF00BF00BF00BF00BF00BF00BFB2
:1026300000BF40251A4EF5610520FFF7D1FC0020B0
:10264000FFF7CEFC2070B56100BF00BF00BF00BF28
:1026500000BF00BF00BF00BF00BF00BF00BF00BF82
:1026600000BF00BF00BF00BF00BF00BF00BF00BF72
:1026700000BF00BF00BF00BF00BF00BF00BF00BF62
:1026800000BF00BF00BF00BF207800F0010070BD98
:10269000A0860100D0000010D4000010D800001067
:1026A00000800920000009402DE9F047FE4E8046D9
:1026B0004FF0807730684024FC4DB84249D100BFCC
:1026C00000BF00BF00BF00BF00BF00BF00BF00BF12
:1026D00000BF00BF00BF00BF00BF00BF00BF00BF02
:1026E00000BF00BF00BF00BF00BF00BF00BF00BFF2
:1026F00000BF00BF00BF00BF00BF00BF00BFEC6154
:102700001520FFF76DFC0020FFF76AFC00F0FF09C1
:10271000AC6100BF00BF00BF00BF00BF00BF00BF73
:1027200000BF00BF00BF00BF00BF00BF00BF00BFB1
:1027300000BF00BF00BF00BF00BF00BF00BF00BFA1
:1027400000BF00BF00BF00BF00BF00BF00BF00BF91
:1027500000BF00BF00BF00BF00BF00BF00BF00BF81
:1027600000BF00BF00BF00BF00BF00BF00BF00BF71
:1027700000BF00BF00BF00BF00BF00BF00BF00BF61
:1027800000BF00BF00BF00BF00BF00BF00BF00BF51
:1027900000BFEC610620FFF723FCAC6100BF00BF67
:1027A00000BF00BF00BF00BF00BF00BF00BF00BF31
:1027B00000BF00BF00BF00BF00BF00BF00BF00BF21
:1027C00000BF00BF00BF00BF00BF00BF00BF00BF11
:1027D00000BF00BF00BF00BF00BF00BF00BF00BF01
:1027E00000BF00BF00BF00BF00BF00BF00BF00BFF1
:1027F00000BF00BF00BF00BF00BF00BF00BF00BFE1
:1028000000BF00BF00BF00BF00BF00BF00BF00BFD0
:1028100000BF00BF00BF00BF00BF00BFEC610120D0
:10282000FFF7DEFB4FEA8800FFF7DAFB3068B842BB
:1028300002D14846FFF7D4FBAC6100BF00BF00BF28
:1028400000BF00BF00BF00BF00BF00BF00BF00BF90
:1028500000BF00BF00BF00BF00BF00BF00BF00BF80
:1028600000BF00BF00BF00BF00BF00BF00BF00BF70
:1028700000BF00BF00BF00BF00BFBDE8F0872DE96B
:10288000F0474FF0000900BF00BF00BF00BF00BF0E
:1028900000BF00BF00BF00BF00BF00BF00BF00BF40
:1028A00000BF00BF00BF00BF00BF00BF00BF00BF30
:1028B00000BF00BF00BF00BF00BF00BF00BF00BF20
:1028C00000BF00BF00BF4025784EF5619F20FFF795
:1028D00087FB0020FFF784FB00F0FF080020FFF7D4
:1028E0007FFBC4B20020FFF77BFBC1B2B56100BF24
:1028F00000BF00BF00BF00BF00BF00BF00BF00BFE0
:1029000000BF00BF00BF00BF00BF00BF00BF00BFCF
:1029100000BF00BF00BF00BF00BF00BF00BF00BFBF
:1029200000BF00BF00BF00BF00BF00BF00BF604DC1
:10293000604E614FB8F1C20F01D1202C07D0822028
:1029400028602120306078463860822095E756481C
:10295000142912D0152913D0162915D0182916D0EC
:10296000C0F800900020FFF79FFEC5F80090784661
:10297000C6F80090386000207FE74FF4801101E036
:102980004FF400110160EDE74FF48001FAE74FF0DA
:102990008071F7E72DE9FF4F8DB00D46DDF86890A7
:1029A0000026434C07935FEA09013ED04FF480575D
:1029B00001463A466846FDF71BFDDDE900B10C9182
:1029C0003A46691C6846FDF713FDDDE90010CDE9C4
:1029D00004013A4668460F99FDF70AFDDDE90085D6
:1029E000A9EB0607C5F58050B84200D2074625B1CD
:1029F000D8457DD10C9885427AD14FF4805000F0B3
:102A0000B5F85FEA000A1CD0D8455BD10C98854226
:102A100058D12A464FEA08305146FFF74CFB0006D2
:102A200019D5504600F0D1F885E086202060214875
:102A300009210160784620490860862011B0BDE870
:102A4000F08F822020601B482221016079461A48BD
:102A500001608220F2E70598804509D1049901EBD5
:102A60000030C1F580525144FFF725FB0006D8D451
:102A70004046FFF79DFB0006D3D407983A468119DC
:102A800005EB0A0000F0C8F8EA194FEA0830514691
:102A9000FFF774FD0006C4D4059988453ED104981B
:102AA00000EB0130049909E0B80100100080092012
:102AB000D0000010D4000010D8000010C1F58052E2
:102AC000514427E0059988450AD1049800EB01306C
:102AD0000499C1F580525146FFF7EDFA0006A0D4E3
:102AE0004046FFF765FB00069BD40798811900E07C
:102AF00018E00F983A463044FFF740FD000690D4A6
:102B0000059988450AD1049800EB01300499C1F574
:102B100080525146FFF732FD000682D4504600F045
:102B200054F80AE007983A4681190F983044FFF7A5
:102B300025FD000601D5206880E73E44002508F108
:102B400001084E45FFF44CAF0549002020600860A5
:102B5000784604490860002070E703480068704721
:102B6000D4000010D8000010B801001070B506465F
:102B700000F0CAF8056806F10B0020F00704B44223
:102B80009CBF002070BD2B466A68BAB11068A04295
:102B900010D304F1080188423CBF5068586007D345
:102BA0005168101941601168091B01605860146078
:102BB000101D70BD13465268002AE7D121462846F1
:102BC00000F0A8F80028DED170BD70B50446051FDE
:102BD00000F09AF80068002C14BF446870BD002C07
:102BE00018BFAC423CBF20466468F8D301680A189D
:102BF000AA4218BF456003D12A6805461144016006
:102C000028684119A1421CBF6C6070BD6168696091
:102C100021680844286070BD032A40F2308010F01B
:102C2000030C00F0158011F8013BBCF1020F624467
:102C300098BF11F801CB00F8013B38BF11F8013BF8
:102C4000A2F1040298BF00F801CB38BF00F8013BA5
:102C500011F0030300F02580083AC0F0088051F815
:102C6000043B083A51F804CBA0E80810F5E7121D20
:102C70005CBF51F8043B40F8043BAFF30080D2073F
:102C800024BF11F8013B11F801CB48BF11F8012B0B
:102C900024BF00F8013B00F801CB48BF00F8012B2E
:102CA000704710B5203AC0F00B80B1E81850203AB8
:102CB000A0E81850B1E81850A0E81850BFF4F5AFDC
:102CC0005FEA027C24BFB1E81850A0E8185044BF66
:102CD00018C918C0BDE810405FEA827C24BF51F8D3
:102CE000043B40F8043B08BF7047D20728BF31F8C7
:102CF000023B48BF11F8012B28BF20F8023B48BF18
:102D000000F8012B7047000000487047E4090010EC
:102D10007047704738B504460A4600206946AFF34D
:102D20000080002808BF38BD02460099204600F008
:102D30003FF8012038BD012000F054B8F8B5AFF3DA
:102D40000080054600200C46102000BF0646A8194A
:102D5000A0420DD9324669460020AFF3008007003B
:102D600008BF00F03FF80098A04218BF0546C419FC
:102D7000FFF7CAFF05600746F01D20F0070046195F
:102D8000284600F00AF8B44208BFF8BDA21B31463D
:102D90003868BDE8F84000F00BB800210160C0E9D8
:102DA000011070471020704700487047DC09001080
:102DB000034640688C46002818BF88423CBF034643
:102DC0004068F8D318681844884207D00CF1030013
:102DD00020F00700001D411A521A0146081D0A6022
:102DE000FFF7F3BE10B500F039F8BDE8104000F071
:102DF0002FB870477546FFF7D7FFAE460500694606
:102E0000534620F00700854618B020B5FDF7C6FAF6
:102E1000BDE820404FF000064FF000074FF00008DB
:102E20004FF0000B21F00701AC46ACE8C009ACE85C
:102E3000C009ACE8C009ACE8C0098D46704710B5C0
:102E40000446AFF300802046BDE81040FDF7B5B959
:102E5000002801D000F02AB87047000010B5012802
:102E600005D0002103A000F027F8012010BD09A122
:102E7000F8E7000053494752544D454D3A204F75ED
:102E800074206F662068656170206D656D6F727962
:102E9000000000003A2048656170206D656D6F721A
:102EA0007920636F7272757074656400014918202F
:102EB000ABBEFEE72600020070B505460C460A20B0
:102EC00000E06D1C00F011F835B128780028F8D129
:102ED00002E0641C00F009F814B120780028F8D151
:102EE000BDE870400A20AFF3008008B569468DF850
:102EF00000000320ABBE08BD194810B5007810F0E3
:102F00001F0F1748C07829D115490839012806D064
:102F1000134A0228937806D003281FD112E01148E3
:102F20000860122012E01048002204E004780CB17E
:102F300044882044521C9342F8D1027872B1086050
:102F4000408803E009481844086000788A88824273
:102F500000D98880FEF715FA012010BD002010BDB1
:102F6000840100102034000032340000533400008B
:102F700070B51D481C4D0078A5F1080510F01F0420
:102F80000AD01948A5F11401184B4A780079012C90
:102F900006D0022C26D109E01348183828601DE01D
:102FA00002B3897888421DD2002015E000F08F041A
:102FB000200605D504F00F064FF48030B04001E044
:102FC0000120A0400AB922070CD18A68024209D028
:102FD000C9680142E8D0012018802B60FEF7D1F9C2
:102FE000012070BD002070BD840100109C090010FC
:102FF00070B502462148A0F11C04017811F01F03AE
:103000000146498804D0012B29D0022B27D111E099
:10301000012924D132B10120FEF716FBA08840F02F
:10302000020005E00020FEF70FFBA08820F0020060
:10303000A08021E0007900F08F00030605D500F0A4
:103040000F034FF480359D4001E0012585406378F2
:103050002BB1030703D0A3682B4200D009B1002095
:1030600070BD22B1FEF742FBE068284303E0FEF7A3
:1030700047FBE068A843E060012070BD84010010B8
:103080002DE9F84F504F00200090B8784FF000091C
:103090004FF0010A4FF4803BA7F11C0600286AD0CC
:1030A0004A4C64E06078022804D0042840D0052807
:1030B0005BD140E06179B878814237D17070207976
:1030C000B070414900200C3901F80090401C0428E0
:1030D000FAD301254FEA06080AFA05F0D8F80810D5
:1030E000084202D02846FEF7EDFAD8F808100BFA8D
:1030F00005F0084203D045F08000FEF7E3FA6D1CAE
:10310000102DE9D34FF00110C8E902090120FEF7A4
:103110009CFAE0794006B8F8040002D540F00100BE
:1031200001E020F00100A8F804001EE060881DE026
:10313000E078009019E00098B8B9A07800F08F0509
:10314000280604D505F00F010BFA01F001E00AFA98
:1031500005F0B16801432046B160FEF78CFA2846BD
:10316000FEF7A6FA2846FEF7B7FA2078044420783E
:10317000002897D11FE086F8019001245546D846D3
:10318000B16805FA04F0084202D02046FEF79AFA28
:10319000B16808FA04F0084203D044F08000FEF75A
:1031A00091FA641C102CEBD34FF00110C6E9020910
:1031B0000020FEF74AFAB8787178884202D10120DF
:1031C000BDE8F88F0020FBE78401001032340000D6
:1031D0002DE9FC5F384D00273E466878BB46B8466F
:1031E000002866D0BA46354C05F11C095DE06078D0
:1031F000022804D0042808D0052854D119E06079A9
:10320000697888424FD060884EE0A77899F804101A
:10321000E6784FF00008B94245D199F80200B04273
:1032200041D125484FF0010A103010F807B0C655BB
:1032300039E099F80410B94235D1A17801F08F0135
:103240000191090605D5019901F00F024FF4803173
:1032500001E0019A01219140009199F80200B042E9
:1032600013D1A8680843A860E96800988143204604
:10327000E960FEF700FA0198FEF71AFA0198FEF7E6
:103280002BFA009948EA01080DE05E450BD118EAD7
:10329000010F08D1A8688843A860E8688843E860FF
:1032A0000198FEF70FFA20780444207800289ED178
:1032B0005046BDE8FC9F0000680100103234000059
:1032C000EB3C904D53444F53352E30000202010029
:1032D0000110000004F802000100010000000000DD
:1032E00000000000000029EFBEADDE41544F4C202D
:1032F000465072696E7446415431322020200000DD
:10330000143500000435000020350000243500008D
:103310003035000018350000103500000C35000075
:103320001C350000283500002C3500000835000051
:10333000000000000010000000200000003000002D
:10334000004000000050000000600000007000001D
:10335000008000000090000000A0000000B000000D
:1033600000C0000000D0000000E0000000F00000FD
:103370000000010000800100000002000080020047
:10338000000003000080030000000400008004002F
:103390000000050000800500000006000080060017
:1033A0000000070000800700FF0F0000FF1F000063
:1033B000FF2F0000FF3F0000FF4F0000FF5F0000F5
:1033C000FF6F0000FF7F0000FF8F0000FF9F0000E5
:1033D000FFAF0000FFBF0000FFCF0000FFDF0000D5
:1033E000FFEF0000FFFF0000FF7F0100FFFF010073
:1033F000FF7F0200FFFF0200FF7F0300FFFF0300CB
:10340000FF7F0400FFFF0400FF7F0500FFFF0500B2
:10341000FF7F0600FFFF0600FF7F0700FFFF07009A
:10342000120110010000004051C2031300010420EA
:103430004801090220000101008032090400000255
:10344000080650620705820240000007050202409C
:10345000000000040309041C03410054004F004C09
:10346000002000200020002000200020002000205C
:10347000002000280346005000720069006E0074AE
:1034800000200046006C00610073006800200020EE
:1034900000200020002000200020001A03460069C0
:1034A0000072006D0077006100720065003000302E
:1034B00000300030000E034D0065006D006F00729B
:1034C00000790000D5130000000000005F19000023
:1034D00000000000000000000000000000000000EC
:1034E00000000000000000000000000000000000DC
:1034F00000000000000000000000000000000000CC
:103500000000000046656200446563004175670085
:103510004A756C004A616E004A756E005365700012
:103520004D617200417072004F6374004E6F7600FF
:103530004D6179005435000000000010BC0100000E
:1035400020010000FC350000BC0100108458000080
:103550007C010000A00D41544F4C20465072696E12
:1035600074280546D4284B3D39609F4574616C6FC3
:103570006E609920126612341232124E1230120FFF
:103580001BDE30071230122E12663272326D1E466A
:1035900034324E30011546524D202008BC41973739
:1035A000383738263D6E2B38024340061B10600426
:1035B000411AFF01014C100D455F5553494E475FBD
:1035C0004D4F5645B81328085838365F54554E4568
:1035D0005F4550494C4F47551F8A291F175348498B
:1035E00046543103392A0810080E270780C3C90141
:1035F000148793031B6CDCE90116000030C80A6FC6
:103600007C9017481B88B436277C40B68EFE275C1A
:10361000AB8B180AB2203D66C140A3C1AD3AACBF26
:10362000B4292636CA2A3973645FC26D88C57B1DEA
:1036300075C441901596F0FBF5F8E202C817BA5F21
:1036400072CFBDF09F5C1C3187667D0EE6C2297D7E
:10365000EB7E14F7C983515EE7CBD32F8A5F4ABB59
:10366000400055C4FB844942CB790A422F54FB44A5
:10367000EA92CAB77A1B9872520D5436D153B7C921
:1036800024ECF3D27B5C38CDC3537FC2AF89FC7F7F
:1036900008E6A628425EBF772C56076A31540F39D8
:1036A000DB07005AB494967A45B9F859FF032F29DD
:1036B000D52CCF6F432087C4F1FC4348E83E0E6110
:1036C00089147AFE2DD12D02DC490B9DEFC93BBB3D
:1036D000DBA2BA5EC67ECADC872F032B3A313C914F
:1036E0008CD7815C9580879392A02BD8190008FD18
:1036F0006375ABF50010306D2AA5856937C5693251
:10370000C6C52B8BC70AAD66FD0F594C660A93E3FD
:103710007F71EF4A80E28A0035DEDE84663359F23B
:1037200093EB5E774DA7BA9A360EF9C1F655AFFA0C
:1037300095356E1CEF943C503D2F0932CC22F1960A
:10374000E7C7271E31FB465CD7E027BE6F082F3640
:103750003826589C48DC9B2E33B29F13C59E7C159F
:10376000D3E78ACA7397FF85EF1CED411C9B05A91F
:10377000DC7331588576FABE0CCA29FBBC9575A25C
:103780002B04DE5637DCC973BA3FE6552C5238C1DC
:1037900077B7A23E0D4F0C782933423B91BB1D4BAE
:1037A000EC23E586CFCBE4F2F50E44E492EE9BD811
:1037B0000BFD5DF2198DBB50456F1B2C40AF884D42
:1037C0005EF69BC01AB67D7665905EE42D210E8074
:1037D00023BC0EE8962A3C25FE862F79AC7EEBBCF6
:1037E000CD5F14B8B625CCE77F7AD4EEEBC8717EF6
:1037F0000C779FC6B08106E1E9A9966E1930971142
:1038000041FBD293E4CFB457BA0EDE155217772C92
:103810005C167966F1E509B11738DE93C883103676
:103820009F2A907690CDFB50F934B58D6D7B436B1C
:103830003F020E36CEB8A0DC6FDDD8FAECDB8CA1EF
:103840009239199F5D6731DA0E6BD87CD68C30E8DF
:10385000C028E99C371F36A940406C385C15DEF65D
:103860002A5CF7253282BD4C0D9BC9E4217F6D6D2A
:10387000C6F7A99E50BB92CA5C66F2E8AAB6FEE102
:1038800042906BEBBCD4009785E41DB863E371C133
:10389000DA7317014BA4FD93C597B87F51FEDCE99D
:1038A0005A70AEEDB672EA3600FB34D9D704B9A42B
:1038B000B303EEE963720D9BDC7FCDFF89A2471C49
:1038C0007370F8B8FE33F3B4C43D5F118792A97AE0
:1038D00083F33D6E9F5F67A21C46EC7CEE3F113A7E
:1038E0005660D24F09D136AF84B9C75BA9B25A57D7
:1038F0002346E77476EDE5B9E89D0BFA7A0201AA52
:10390000D75D2BC0AD17E80FC948712113A00B2359
:10391000E9624EA89A78B80483C343E87C54CB6527
:103920000AE46AA6A72A62601B3FFBAC06CC0441EE
:1039300091C725EDA8D47108F162ED02D77BB79449
:10394000FB0ABA4BA88052061469F7D6FBD155235F
:1039500089D030E05EAB0D51647B5579B2BD39251D
:10396000DFB1AE722E168FDF47B2FF79554B650877
:1039700073F0A8923FD7504EC486B811C8BFEE7EF0
:10398000C0DADF1BE7584571803A05A85CC98ED3C1
:103990007BCE9D7F0BC96F805579125CC8EF13E811
:1039A000BEC09271C5B63BD28FCEA0A36EF839D3FC
:1039B00059460A7EFFBFCDCA246A5B5520EBE968F1
:1039C0005CE199CA8E1D37AB806593CEE8DDEE7E53
:1039D0008905BF74587541ADC12BC9F767CD19462C
:1039E00093552F8D7267A09871FA1E8C2A92512DD3
:1039F000BEE627935F99B840E6EA66E195AB636D52
:103A000085319AEF61A672C54529E865CFC1565147
:103A1000330F0DE76E2BF1FD9341709664B1FCBE40
:103A2000693C3745111157A6370C07853EAF3F4E0D
:103A300053D54917B51CD973B165E6307ACD4041ED
:103A400027C2EA0DBF1D4BA1E312B5977A7B0EDBAF
:103A50008F807A8E47EFF0C5C234117C701B911DA8
:103A6000BFF4A4DA242345FA512E9785DC6C5CD38D
:103A70004071659C220E09565C91B9257C206BE64D
:103A80009CE58B2C503F5974FFC53B60B73E459178
:103A9000D8BBB4C1EB86BE475001798A2A203EE4E8
:103AA00060AE614884455FED576438104F7C68A470
:103AB0006A8309FD2F943B47E06AB683F8D152D759
:103AC000B8007CC4E308355453B31709007A8784DF
:103AD000BD0F7D6822A282CB773671322DC631D3DD
:103AE0007BC00DC995461DF651271CCA4A569568DC
:103AF000FAA3614A46A02D2A0F9CD93F82A8259A95
:103B000084AAB581BC90085F52DD809FB689F60219
:103B1000DFC9D74E8027690A84E3583E892D181DD6
:103B20009D0C43D71525FCA70979A0B5A57284F68D
:103B3000F660458FA584D528088052BB473EB41D4A
:103B4000A19BF28FDD14A8ECF093859E63AEC0D1EB
:103B5000807E6DCCD61F4B302A213D184F9A8E5255
:103B6000E47ECCB21A3584E3C621FAE8ABA865003E
:103B7000A2A1CE4B64B7B482DC3B8396A3CEE1E72F
:103B8000DA9540410794E24D4C702BFEAD6D5B8C95
:103B9000221B667A48A9624E410155AC116F22A2E0
:103BA00021CA7B91073196A87582C9CFDBAFFCAAE9
:103BB000798B47813383005F237A06BB2AE4CCD616
:103BC0004B333EC7897DDA2843F5F123908E6C6430
:103BD000D3438D18657BA4A9405D5B77626A47AFCC
:103BE000124131DA379C5EDEE0BE78510D9B0D83C9
:103BF00008DE48EC8A5A60EFA47155DBB61BAAE8D0
:103C00001BD8E8952129D0E423C8AD5AEB3EB8E192
:103C1000BF08F75FF0D7A92C2C8E216BB827D0F600
:103C2000B14001B46C5913F18EF9CA9F2CE6F64DE0
:103C30001FD774CCD04F5926C148605F8A9FDC21C2
:103C4000FDBE9BAD194AC2C67BE3C2F77275E96837
:103C5000BB93DE746507C3B19D533A7731C4AE5749
:103C600048729381987C9054DD26DB71C30CB8A315
:103C7000A162DDB8EFA42C86F1CFFB68E6294837B6
:103C8000EF4F28F8CC232625814EE46E71D5F27AC9
:103C9000FD49707E7FF7501D37B6D927FA11C0262F
:103CA000B446AF5C228EF72204E90079C710C6E45F
:103CB000417FB705CDEE21E6D22CBCDF4E65AF17B4
:103CC00014A00CEFB33A9A54DC2514E411E97A13EA
:103CD000A0498125057B3FAEA44E700C01B9B0030D
:103CE000D836ECB141D8FF626B14473CB5F8ACDB79
:103CF0001F397968E0ECEBEDD7AC2E4990BCABB244
:103D000069D51058932866ED9EF314C0010D75FF18
:103D10001254DBB768E7750E82A6A111769D1C8F41
:103D20008C49BFA45B1E68FA2F58B29389DF52A654
:103D3000F0C869C4CF0FCA3D6FD34BD8033782F2A6
:103D4000ADAC3BDF75879600E994414D22B7342630
:103D5000CC572E118389DDDC84C8FF25FE9EE298B6
:103D6000EE18CAD775334AF22BD07D83E3CECC2927
:103D700083605F5897138E63938C1C6700E99A8663
:103D8000D320A64C530A36EA5C5D7C5484C2D5BD70
:103D9000E1204F09CBEE2B56427BEAFD678B40D4E6
:103DA000E41809599D1C1CBF3D10D0E51FF766C2E1
:103DB0005DF38642762185E5F38C878048C8C4236D
:103DC00098EB7B22CA771EC525EEFD47B03DBAA70A
:103DD000FB9E3AF3855971CDAA68C41DDE3414AD3B
:103DE0002D8506DCD74E1E1A932111CEDCCF991FEC
:103DF000D322C929F80A1C932EFBF085798DA47A69
:103E000047129C69C0009340522B2DCF6CE489C1AE
:103E1000F33876ACE7006BCD6E769EB231D35DE0C1
:103E2000046BF308684DDC8DC6CE413136F47D86D7
:103E3000A5958BC3E1F1CC4C7ED611B5615842906B
:103E40004C6E3706CC91C7432819AAF444682F401A
:103E50003FA722CD6FCFA9410403855C08D8EFE8C6
:103E6000FB2825C17ED7ECB8A3662C18591943034B
:103E70009AEAAC316F206BE54EB369667FA1C2E46C
:103E8000D61571DEAC89234EC689D195B3C7EFA391
:103E9000BC225F7DF2609814722B727772CBC704DC
:103EA000DCF67D4B6050D586227592C58ABEEECE7B
:103EB00097C0A1748D18AAF434A05925AB6A0EF5E9
:103EC000390764DAF71A1522D67D4C9B66D1C525D1
:103ED0009B1822208CB040354E2624F58D8FD5EAD4
:103EE00039080B70CA667104B4733F21DD7ECBC9FB
:103EF000ED6974282999BD8DF4258B14C351612077
:103F0000E46A22ECEBE9C101F7CF601B47325B8822
:103F100082D2BFBF161D8F225D7E0FCE7544F73D46
:103F200099DDC97D4B12FDBB0C7415D982FB18E1DC
:103F30008E842E64AA51702171BEC75B4C4FECC6B3
:103F4000EC18D3930502ECDBCA8B45916DBE48900B
:103F5000168B17929C512EDDF642C624E04935F8A7
:103F600019E97D6A5134F79AB8C56C068210A25CD3
:103F7000DC6CF973F15DA4F0B40279A24C40278E99
:103F800032B293058CC0F625E2C07CB5E5A5389B1E
:103F90009916B1BA5DAAF5AFB0CCF0070C1C05ECD0
:103FA00084E391218081862293C75440FC1E5AB835
:103FB000E028AF1B66C9CF65340BFF3EFAB8C2C11B
:103FC000B2A6CE726126B7A874E629F94541FE74FF
:103FD000E81DFE0E6A63D4C37C692C80E1A6262806
:103FE000DB70C355245BE6D2B277B2A04763B0540E
:103FF000268EC153F6458A4E995F8AC6688F5C90BB
:10400000C88100101947030021470300234703001C
:1040100025470300274703002947030066D3EBEF3A
:104020000000000000000000000000002B4703001B
:104030002D470300000000002F4703003147030015
:10404000334703004D49030033470300A3AA03008D
:10405000334703006D8C03002F8F0300A3910300EF
:10406000F1930300519B03003347030033470300E0
:10407000334703003347030033470300334703004C
:10408000334703003347030033470300334703003C
:10409000334703003347030033470300334703002C
:1040A00027CF0300334703003347030033470300A0
:1040B00029DD030033470300334703003347030080
:1040C00033470300334703003347030033470300FC
:1040D00033470300334703003347030033470300EC
:1040E0003347030000F002F800F086F80AA090E8D9
:1040F000000C82448344AAF10107DA4501D100F0A3
:104100007BF8AFF2090EBAE80F0013F0010F18BFE9
:10411000FB1A43F00103184760220500A0220500A6
:104120000A444FF0000C10F8013B13F0070408BFDD
:1041300010F8014B1D1108BF10F8015B641E05D07B
:1041400010F8016B641E01F8016BF9D113F0080F30
:104150001EBF10F8014BAD1C0C1B09D16D1E58BFC2
:1041600001F801CBFAD505E014F8016B01F8016BF9
:104170006D1EF9D59142D6D370470000002300246C
:1041800000250026103A28BF78C1FBD8520728BF67
:1041900030C148BF0B60704769293EF09D87642994
:1041A0003EF09A8775293EF097876F293FF02E8061
:1041B00078293FF055800368DB0928BF41F0800172
:1041C00063293FF0F28373293FF0F783E3293FF03F
:1041D0000284002070471FB59DE803003FF01CFBE0
:1041E0003FF076FC04000020002140F08FFD401CD1
:1041F00060601FBD10B510BD3FF044FC1146FFF7D5
:10420000EAFF00F013F93FF067FC03B4FFF7F2FF99
:1042100003BC3FF097FC000010B5782119483FF02F
:10422000B6FA19494FF0FF30088010BD16480188D2
:10423000491C09B201800A290CD001EB4102114945
:10424000436841F8223001EB820183684B60C0680B
:1042500088607047FEE70C4910B5B1F90000421CB8
:104260000ED0084A00EB4003401E52F8234002EBF8
:1042700083024C6053688B609268CA60088010BDEE
:10428000FEE70000800500100000001030B5024677
:104290004FF6FF7318464B4C08E000BF12F8015B65
:1042A00085EA1025655D85EA002080B2491E89B245
:1042B000F4D2584030BD10B541F221033CE000BFBC
:1042C00011F8014B80EA0420040402D583EA40007F
:1042D00000E0400080B2040402D583EA400000E020
:1042E000400080B2040402D583EA400000E04000B0
:1042F00080B2040402D583EA400000E0400080B2AE
:10430000040402D583EA400000E0400080B20404C7
:1043100002D583EA400000E0400080B2040402D5E8
:1043200083EA400000E0400080B2040402D583EA42
:10433000400000E0400080B2521E92B2C0D210BDD8
:1043400030B50346002002461F4C0AE013F8015B1B
:10435000521C85EA102592B234F8155085EA0020E7
:1043600080B28A42F2D330BD41400020CA0700D05B
:104370005E208A0701D580F0BC004A0701D580F095
:1043800061000A0701D580F0C200CA0601D580F09D
:104390009D008A0601D580F023004A0601D580F0F1
:1043A0004600090601D580F08C007047024610B522
:1043B000FF20002905D0054B545C4440491E185D80
:1043C000FAD110BDCA620400CA63040040000010A4
:1043D0000A4900EB4000084410F8030C70470749F5
:1043E00000EB4000084410F8020C7047034900EB52
:1043F0004000084410F8010C704700006C8704006E
:104400004F5639DC9B1B02000034704770477047E1
:104410004D6179203330203230313600704770479B
:1044200030393A35383A31380000000088B0C44C91
:104430000027039720883E4640F002002080C148B4
:104440002EF020FEC048007802281CD1FFF7EEFEB7
:1044500003A830F0ADFD000601D502F0EAFEFFF73B
:10446000FAFE0398B0F58C7F0DDAFFF7DFFE00212E
:10447000B6A037F08CFD000601D502F0DAFEFFF79A
:10448000EAFE02F0D6FEAF4D288830F4504010D03E
:104490000127FFF7CBFE32201AF0DFFF012012F0D8
:1044A0009FF810B1082037F083FFFFF7D4FE02F029
:1044B000C0FE2888810B06D0012710F0EAFA00061A
:1044C00001D502F0B6FEAC482E80007828B12FF05E
:1044D00089FD10B1A9A037F04AFF26F011FF0006B0
:1044E00001D502F0A6FE01F0B7FA06F09AFE00062A
:1044F00001D502F09EFEA74DAE6805A82EF0D0FCB7
:1045000001F062FA10B1012702F093FE01F0E6FA21
:10451000DFF88482C0B1FFF789FE01F037FCFFF7B6
:104520009AFED8F80000062802D000219BA004E0E3
:104530009F490220087000219EA037F028FD2088A6
:1045400040F0020020800CE001F0E5FC38B1FFF7FC
:104550006DFE01F01BFCFFF77EFE02F06AFE01F02B
:1045600080FF39F042F99848A968891B8142FBD342
:1045700006A82EF095FC954EDFF85492307800EBAB
:10458000400159F831008047000601D502F051FE84
:1045900001F0C8FF000601D502F04BFE9DF81A009D
:1045A0009DF81610884201D0012000E0002001F0A3
:1045B000FBFF00B1012702F055F800F0C7FD02A98A
:1045C00053201BF01FFF000601D502F032FE9DF8BC
:1045D000080000F001008DF808006FB9B0B10120AB
:1045E00011F0FEFF000601D502F023FE11F004FBDE
:1045F000000601D502F01DFE9DF8080030B1012033
:1046000011F0EEFF000601D502F013FE30F0B7FB0B
:104610004F46E94638F082FF307800EB400007EB68
:10462000C000C0688047000601D502F002FE307865
:1046300000EB400007EBC00040688047000601D552
:1046400002F0F7FD307800EB400007EBC000806817
:104650008047000601D502F0ECFD002037F032F96A
:10466000D8F800000C2805D005F0BAF9000601D5ED
:1046700002F0DFFD207840071ED5012037F022F937
:10468000D0B9684605F09FFD50B909F1020005F068
:10469000ABFD28B909F1040005F0B7FD000601D50E
:1046A00002F0C7FD4B499DF804000870684607F00A
:1046B00051F808B907F0B2FE207810F0B80F35D0E5
:1046C000012037F0FFF8000630D4A8684249AA68F4
:1046D000121A8A42FBD32078000701D511F036FB6D
:1046E0002088010614D5810612D4C00613D411F017
:1046F00087FB000601D502F09CFD002007F078FF43
:10470000000601D502F095FD208820F08100208070
:104710002078C00601D506F0BFFF2078800605D5B9
:10472000012009F075FC012011F05AFF30F08DFBDB
:10473000000601D502F07DFD37F040FF6AE700007A
:104740004A1E00204C1E0020A80300108E9888816D
:104750008A802081809280908588209780918E82A7
:104760000A8E81908092889285919C2082209692D8
:104770008E0A0A0A0A000000411F0020C0E2F2EE81
:10478000EEF2F0E5E7F7E8EA20E2FBEAEBFEF7E518
:10479000ED0A000000000940080000108E98888192
:1047A0008A80208F808C9F9288208F840A0A000044
:1047B000481E0020878D208D852082828584858DEE
:1047C0000A0A0A0A0A000000E0C81000E81E0020D9
:1047D00034030010C11E0020A086010000F00F016C
:1047E000000900EB800001EB4000C0B270470A21D5
:1047F000B0FBF1F201FB1202B0FBF1F002EB001092
:10480000C0B27047002210B511460A2309E000BF6C
:10481000B0FBF3F403FB1404B0FBF3F08C40224430
:10482000091D0028F4D1104610BD2DE9F047FA4DBE
:10483000FA4EFB4F9046C3B15C1E0BD4DFF8E493F5
:10484000642200233EF018FB19F8023008F8043007
:10485000641EF5D5084310D08920286004203060FC
:10486000784638608920BDE8F087882028600920D4
:104870003060784638608820F5E700202860306096
:10488000784638600020EEE710B500220BE0835C2C
:1048900003F00F04092C03D803F0F003902B01D987
:1048A000002010BD521C8A42F1D3012010BD2DE919
:1048B000FF4FD94CD94DDA4E83B08246082A31D801
:1048C0007AB30020CDE9000001214FF0860B4FF0B4
:1048D000200E00BF0AEB020313F8019C09F00F033E
:1048E000092B14DCA1FB03784FEAD37C00FB038384
:1048F00001FB0C33DDE9008C18EB07074CEB030CD4
:10490000CDE9007C4FEA1919B9F1090F12DDC4F89D
:1049100000B07846C5F800E03060862007B0BDE8FA
:10492000F08FFFE7882020600920286078463060FB
:104930008820F3E74FF00A0CA1FB0C3800FB0C8039
:10494000002701FB0700A3FB091800FB09874FEABA
:10495000E97C03FB0C77DDE9008C18EB01014CEBE3
:10496000070CCDE9001C4FF00A0CA3FB0C18002724
:1049700000FB0C8003FB0700521EABD10698DDE95B
:104980000023C10001208840401EC117801A9941B0
:1049900007D2892020600420286078463060892072
:1049A000BCE76946069A04983EF0CDFD00202060E1
:1049B0002860784630600020B0E730B500B90120AB
:1049C000401E80B240F2B553B0FBF3F2B0FBF3F4FB
:1049D00003FB14009206401C120E80B24FF4B77312
:1049E00098420BD9521CD2B2A0F5B77003E0521C0A
:1049F000D2B2A0F26D1080B29842F8D2202801D233
:104A0000012319E01F3880B2930701D01C2300E076
:104A10001D23984201D802230EE0C01A814D0023C5
:104A200080B2643503E0001B5B1C80B2DBB2EC5C3F
:104A30008442F8D3DB1CDBB20A704B708870764975
:104A400000200860754908607846754908600020B4
:104A500030BD10B5027840F26D135A430A80714C94
:104A600043786E3434F813301A440A8083781A4439
:104A700093B20B800278940705D14078022802D8BF
:104A800003EB920003E0012000EB92001844088041
:104A90006149002008606149086078466049086003
:104AA000002010BD10B581784FF0FF32C9B14378B6
:104AB0000D2B18D2DFE803F017070D070A070A07C6
:104AC000070A070A07001F290BD80FE01E2908D87C
:104AD0000CE00078800702D01C2902D806E01D29CE
:104AE00004D9104610BD6FF0010010BD002010BDAC
:104AF00018B502880024B2F5FA6F0ED9C2788DF885
:104B0000022082788DF801200078A0F5FA608DF8F7
:104B100000006846FFF79DFF00E00C803E480460FF
:104B20003E48046078463E490860002018BD18B52C
:104B30000C466946FFF741FF9DF80200E0709DF8C2
:104B40000100A0709DF80000334900F5FA60208054
:104B5000002008603149086078463149086000202B
:104B600018BDC0F30722C0B2C0EB001002EB8000FA
:104B700008802949002008602849086078462849AB
:104B80000860002070473C22B0FBF2F30B70B0FBD2
:104B9000F2F302FB130048701F49002008601F4910
:104BA000086078461E490860002070472DE9F04FE4
:104BB00088460021184D194E194F82464FF086093C
:104BC000B3EB420F16D301201FE000BFA2EB000B96
:104BD0001AF80B4004F00F04092C0BDCA3EB400E79
:104BE0000EEB080C30348CF801401AF80B40240905
:104BF000092C06DDC5F800907846316038608620C3
:104C00008DE6303408F80E40401C9042DED9012079
:104C100000EB420030220CE00400001008000010FD
:104C20000C000010B25F0400A3EB000C401C08F85D
:104C30000C209842F8D9296078463160386000200D
:104C40006DE62DE9F84F82468B4601204FF086092C
:104C5000B54DB64EB64F00212BE000BFA2EB000EC3
:104C60001AF80E40303C092C14DC04F0FF0C00EB69
:104C7000D074A3EB640808EB0B04A4F10108CDF891
:104C8000008004F801CC0EEB0A0414F8014C303C0F
:104C9000092C07DDC5F80090784631603860862021
:104CA000BDE8F88F4CEA0414DDF800C0801C8CF8D5
:104CB00000409042D2DD521C9A4203DC9C1A0BF851
:104CC0000410F8E729607846316038600020E7E793
:104CD0007CB50D4601A9FFF770FE934C000601D587
:104CE00020687CBD9DF8040000909DF805309DF87B
:104CF000062090A128463EF05BF98C4900202060F8
:104D0000086078468A49086000207CBD3C2310B5C5
:104D1000B0FBF3F2B0FBF3F403FB1403D2B20A20AE
:104D2000B2FBF0F430340C70B2FBF0F400FB142250
:104D300030324A703A228A70B3FBF0F23032CA70D5
:104D4000B3FBF0F200FB12303030087176490020DE
:104D5000086076490860784675490860002010BDF3
:104D60003C2310B5B0FBF3F2B0FBF3F403FB1400EB
:104D7000744BD2B29A5C0A70185C48706A49002081
:104D800008606A490860784669490860002010BDDB
:104D90000278407802F00F03120902EB820203EB63
:104DA000420200F00F03000900EB8000D2B203EBD7
:104DB0004000C0B2C2EB021200EB820008805A49E8
:104DC0000020086059490860784659490860002069
:104DD000704718B50C466946FFF7EFFD52490006CB
:104DE00001D5086818BD9DF802205648825C2270E3
:104DF0009DF80120825C62709DF80020805CA070AC
:104E00000020086049490860784649490860002048
:104E100018BD70B5044611B93EF076FB014600227C
:104E200020230DE0A05CF02801DB103802E0C02850
:104E300002DB4038A05402E0802800DBA354521C5F
:104E40008A42EFDB002070BD70B5044611B93EF018
:104E50005BFB01460020202311E0225CF02A01DBED
:104E600023540BE0E02A01DB103206E0B02A01DB1C
:104E7000403A02E0802A01DB40322254401C884242
:104E8000EBDB002070BD10B5044600200146012276
:104E900002FA01F3234205D0C1F1070302FA03F33A
:104EA0000343D8B2491CC9B20829F1D310BD202848
:104EB0000BD0092809D00A2807D00B2805D00C28C8
:104EC00003D00D2801D0002070470120704770B535
:104ED0000546044600E0641C2078FFF7E8FF002840
:104EE000F9D120463EF010FB421C214628463EF0F8
:104EF0006FFB284670BD10B504463EF005FB011956
:104F000000E0491EA14205D011F8010CFFF7CFFFC8
:104F10000028F6D100200870204610BD10B5FFF71C
:104F2000D6FFBDE81040E6E70400001008000010BE
:104F30000C000010253032752D253032752D2530AE
:104F400032750000B25F0400F8B56A4E0D460746A0
:104F500002226946304630F0EFF8674C000615D45F
:104F6000BDF800002A4640F08040394630F0EFF8A6
:104F700000060BD4BDF8000002222844ADF8000062
:104F80006946304630F0E3F8000601D52068F8BDE8
:104F90005A4900202060086078465949086000207E
:104FA000F8BD08B50020ADF800000222694651485E
:104FB00030F0CDF808BD014602224E4830F0BCB8B2
:104FC0002DE9F04188B00025022201A9494830F0BE
:104FD000B3F8494C00064ED4012036F0CDFE000651
:104FE00049D448490888420606D520F04000088088
:104FF0001AF0B1FA00063ED4002705A8059705F07F
:10500000EBFD000637D406A8069705F0F6FD00066E
:1050100031D43D490220087004A962201BF0F2F946
:10502000000628D400264FF0200829E046F08040F2
:10503000012203A930F080F89DF81000400714D435
:105040009DF80C0043280DD0F3280BD0F42809D08C
:10505000F5280AD16D1CEDB28DF80C80022D04D11B
:10506000002502E00DB18DF80C80012103A836F077
:1050700060FC000603D5206808B0BDE8F081761C0E
:10508000BDF804008642D1D31C48276007607846EB
:105090001B4908600020EFE710B5FFF782FF164CB0
:1050A000000604D4052036F067FE000601D520680E
:1050B00010BD124900202060086078461049086041
:1050C000002010BD10B50C4C18B1FFF76AFF0006A8
:1050D00004D4012036F050FE000601D5206810BD32
:1050E00006490020206008607846054908600020D5
:1050F00010BD0000480F0020040000100800001040
:105100000C0000104A1E0020481E0020F8B516466C
:105110000D46044689480122694630F00DF8000624
:1051200002D587480068F8BD9DF80000204000D0F7
:1051300001202870022C06D08048401C02223146F3
:105140002FF0FAFFF8BD7D48C01CF7E710B5AAB0F4
:1051500027A80BF026FB7A4C00064BD426AA28A9D8
:105160000120FFF7D3FF000644D49DF8A00028B12A
:10517000BDF89800BDF89C10884209D971490020FB
:105180002060086078467049086000202AB010BD91
:10519000022036F083FC00062CD46C4837F0E7F888
:1051A000000627D46948143037F0E1F8000621D40E
:1051B00026AA28A90220FFF7A9FF00061AD49DF805
:1051C000A000C8B129A9BDF89800FFF7F6FB0006BA
:1051D00010D49DF8A4005D4900909DF8A5309DF87D
:1051E000A620263101A83DF0E3FE01A837F0BFF864
:1051F000000601D52068C9E75548018841F0020141
:105200000180544902200870012011F0E9F9BDE73E
:10521000FEB501A80BF0C5FA494C000632D46A4627
:1052200002A90220FFF772FF00062BD49DF80800A8
:10523000444D454E28B1BDF80000BDF80410884229
:1052400006D9002020602860784630600020FEBD2E
:10525000022036F023FC000614D43C4837F087F8CF
:1052600000060FD43948143037F081F8000609D40D
:105270003748018841F002010180012011F0B0F9A6
:10528000000601D52068FEBD91202060BE20286068
:10529000784630609120FEBD4FF0A04301460422C5
:1052A00018462FF049BF4FF0A0430146042218468C
:1052B0002FF04DBFF7B50446204882B00E46054694
:1052C000012269462FF038FF1D4F00060ED49DF8CD
:1052D00000000EB1204300E0A0438DF80000012241
:1052E000694628462FF033FF000602D5386805B01E
:1052F000F0BD022C06D01148401C022204A92FF058
:1053000026FFF4E70D48C01CF7E738B5002001225E
:10531000014600901046FFF7CDFF094C000606D469
:10532000012200210220FFF7C5FF000601D52068F9
:1053300038BD6846FFF7B7FF38BD000004000050D5
:1053400004000010080000100C0000103A60040077
:105350004A1E0020481E00202DE9F04F99B001247C
:1053600000250C94841A089571EB030404DA1646A0
:105370001C4607460D4603E00C46064617461D46EA
:1053800000218B46059116E002220023304621467B
:105390003DF0E9FD06460C46022200233846294628
:1053A0003DF0E1FD0D46012205991BEB020B41F199
:1053B000000107460591F00701D1F807E4D001206C
:1053C0000021CDE9220124AA0846279482E843005F
:1053D000711E64F10000CDE91610CDE91475CDE918
:1053E000127500BFDDE9260180468946C00729D134
:1053F000DDE92201C20702D1249AD2070AD03A1865
:1054000045EB0100CDE92220DDE92410711860414F
:10541000CDE92410DDE92201022200233DF0A3FDA5
:10542000CDE92201DDE92401022200233DF09BFDAC
:10543000CDE9240102220023404649463DF093FD78
:10544000CDE92601DDE91201C20704D0DDE92632EB
:10545000181A8A410BDA14A922A800F066FA16A9D4
:1054600024A800F062FA12A926A800F05EFADDE98D
:10547000260110900D91C007B4D00DF15008DDF851
:105480005C2098E80B009E46DDE922C3E1469A467F
:10549000BCEB000C8B4106DBDDE9248CB8EB0E0382
:1054A0007CEB020C0DDA17EB090345EB0A0CCDE996
:1054B000223CDDE9243CF31844EB0C0CCDE9243C00
:1054C000E2E7B9EB00006AEB0103CDE9220325987E
:1054D000B8EB0E0160EB0200CDE92410DDE91210FB
:1054E000109B0D9A5B1A62EB0002CDE92632002375
:1054F000591A73EB0002FFF675AF14E0DB1B60EB8B
:1055000005004FF0000CB3EB0C0C70F1000C17DB36
:10551000CDE92230901B61EB0401021E71F1000203
:105520000EDBCDE92401DDE92230D91B70EB05014A
:1055300006DBDDE92421B6EB020C74EB010CDDDBAC
:10554000002108461AE000BFDDE922720C9B089D8D
:10555000A3FB07C805FB078503FB0252CDE922C266
:10556000DDE92672A3FB07C8089D491C05FB0785DA
:1055700003FB0252CDE926C240F10000059AB1EBCF
:105580000B0370EB0202DFDBDDE9261081F0010185
:10559000014304D04FF0FF3019B0BDE8F08FDDE9D2
:1055A0002410711A64EB00042898C0E9001400204C
:1055B000F2E72DE9FF5F9CB00020CDE90200CDE9C4
:1055C000040092462E9907AA0A20CDE900029946C6
:1055D00014AB0122491C1BF033FB00287DD114AB16
:1055E00008AA195C0C0902F8104001F00F0402EB44
:1055F0004001401C4C700828F3DB9DF82F70DFF849
:10560000408311460E2000BF58F82740461C255CF9
:10561000A45D801E4E5D11F804C001F805C00E5552
:10562000F2D5002002EB400412F810106478904686
:1056300044EA01111954401C0828F3DB19460020E4
:10564000079B0DE01C1A0C440A5C14F8015D2E0146
:1056500046EA15150D54150145EA12122270401C38
:10566000B0EB530FEED3082312A914A8079AFFF743
:105670001EF90028B2D114A90FF000FC0028ADD10A
:105680000C2114A8FFF700F900287DD0DDE91501F1
:10569000CDE90801082208A90020131A0B440C5C6C
:1056A00013F8015D0D54401C1C70B0EB520FF4D385
:1056B00000252C462F462E462846C3464FF00A0E9C
:1056C0001BF800107246303901EBC101B1FBF2F357
:1056D000B1FBFEFC0EFB1C1100E0AEE04FF0640CD1
:1056E000A5FB0C2801EB810103EB410104FB0C84B9
:1056F000002305FB034455185C4107910A23A7FBCF
:10570000031C06FB03C3002207FB02321BF8003018
:1057100000F10100303B5F1842EBE3760828CFDB55
:10572000DDE91201401B61EB0401864A0023CDE94B
:1057300012013DF0A1FBCDE9122350EA01027CD019
:105740001AAA0692CDE90054DDE91C23FFF704FEF6
:10575000002872D1DDE91A50A7FB051206FB0522CD
:1057600007FB00248346DDE91C23084621463DF063
:1057700083FB14469846DDE91223A2FB050603FBD2
:10578000056302FB0B3100E06CE0DDE91C233DF01A
:1057900073FB15469B4654EA080203D0DDE92A0153
:1057A000012618E0012000211AE000BFDDE92A727D
:1057B000A0FB073C01FB07C100FB02111846BAEB36
:1057C000000379EB010205D252464B463DF054FBF3
:1057D00010461946761CF317371B73EB0803E5DBFD
:1057E000CDE91A0180460C4655EA0B0003D0DDE9ED
:1057F0002C01012617E00120002119E0DDE92C72BF
:10580000A0FB073C01FB07C100FB02111846BAEBE5
:10581000000379EB010205D252464B463DF02CFBCA
:1058200010461946761CF317771B73EB0B03E5DB69
:10583000A0FB085301FB083100E012E000FB04115B
:1058400052464B4628463DF017FB10461946DDE907
:105850001C233DF011FBDDE9120150405940084383
:1058600003D0002020B0BDE8F09F0120FAE7F0B59A
:10587000411E85B01E2932D2012404FA00F111F034
:10588000500F2CD0304FBE68401E2D4D8440083D37
:1058900069680C4229D1C1B204912C49002301EB63
:1058A000C001D1E90021CDE902212849284A403927
:1058B00001EBC001D1E90001CDE9000143F6E100AF
:1058C0001946FFF776FE0028286801D0204300E043
:1058D000A0432860B8681F49801B884202D300207B
:1058E00005B0F0BD68682043686028682040F7E78D
:1058F000411E1E290ED2012101FA00F212F0500FB2
:1059000008D0401E81400E48083842688A434260F1
:10591000012070470020704700B501231846FFF7AB
:10592000E7FF5B1C1E2BF9DD00BD30B5D0E900237D
:10593000D1E90045C0E90045C1E9002330BD0000C0
:105940001800001000E1F50500000940C0600400E7
:10595000BBF81A03404B4C0038B50446684604F0C7
:1059600086FB9DF80000204038BD38B504466846E7
:1059700004F07DFB000602D5FD48006838BD9DF8A7
:10598000000020438DF80000684604F067FB38BD36
:1059900038B50446684604F06AFB000602D5F448B0
:1059A000006838BD9DF80000A0438DF800006846EF
:1059B00004F054FB38BD01B5FEF738FC684604F02E
:1059C0006DFBFEF748FC08BD7CB5684604F070FB33
:1059D000E74C000638D49DF800000025082809D0BF
:1059E00009280DD0E348256005607846E249086043
:1059F00000207CBD684604F06CFB000624D40BE05C
:105A000001A805F0A6F800061ED49DF804000128A0
:105A10001CD013208DF80000684604F03FFB000600
:105A200012D48DF8045001A805F089F800060BD4B3
:105A30008DF8045001A804F078FB000604D443203C
:105A400019F00BFD000603D520687CBD0220E1E7BC
:105A5000012010F0C5FD7CBD2DE9F041002402209D
:105A600036F0C0FCC54DAE68C54F4FF4FA7811E072
:105A7000A868801BB8420DD301202CF001FDC8217D
:105A800040462FF05CF901202CF007FDAE68641C45
:105A9000042C04DC00202CF0E5FC0028E8D1012CCB
:105AA00006D0022C07D0032C09D0042C11D10EE013
:105AB00001F03EF90DE0022029F025F809E0B14C93
:105AC0000120207002F066FE0020207001E02EF020
:105AD00041FDBDE8F041012036F084BC0EB56846BA
:105AE0000FF047F950B1932803D1A2480068062867
:105AF00001D00E2000E01120FFF75DFF9C480068F8
:105B00000EBD2DE9F34F002789B088460F703E4641
:105B100008A938460DF0F8FA954C000639D49DF8DE
:105B20002000DFF85092DFF850A2400607D407A803
:105B300004F0ADFA00062CD49DF81C0068B3694649
:105B400009980EF013F9000623D40125EB4605A9A8
:105B5000284604F0B6FD00061BD405EB8501594428
:105B6000052205A8491F3DF07FFC00B101276D1CEF
:105B7000EDB2042DEBD9C7B18349099808804520BF
:105B800019F06BFC000604D4012010F029FD00067A
:105B90000BD520680BB0BDE8F08F26607946C9F8B8
:105BA00000600020CAF80010F4E788F80070F4E7FD
:105BB0002DE9F34F85B00320002408700E462746D8
:105BC000214601200FF025F90106694802D5006839
:105BD00007B0E0E70168DFF89C91DFF89CA10025A1
:105BE000052913D08046EB46694601200FF0EBF8FB
:105BF0000006D8F80000EBD405280DD005220BF1E3
:105C0000040005993DF030FC18B103E035700560E3
:105C10000DE0671C641CE7E737B1BC4201D10220EC
:105C200000E00120307000E03570C8F8005079467F
:105C3000C9F800500020CAF80010C9E730B5044682
:105C400085B00020208002200FF0F9F8484D05288B
:105C50000BD0694602200FF0B6F800061ED4BDF83E
:105C600000002188884200D9208001200FF0E7F849
:105C7000052802D06946012006E000200FF0DFF879
:105C800005280BD0694600200FF09DF8000605D4CA
:105C9000BDF800002188884200D92080286805B01E
:105CA00030BD2DE9F04387B00646694600200FF06D
:105CB000E5F82F4D000649D403A90B200DF024FA76
:105CC000000643D40C2203A968463DF0CDFB022711
:105CD000DFF8A080DFF8A090002408B137703EE024
:105CE00003A910200DF010FA00062FD469460420F5
:105CF0000FF0C4F8000629D4BDF80000BDF80C1060
:105D00008842EBD1694606200DF0FEF900061DD44D
:105D1000BDF80000BDF80C10401E8142DED169467E
:105D20000E200DF0F1F9000610D403A8FFF786FF4E
:105D300000060BD4BDF80000BDF80C108842CDD38E
:105D4000694600200DF0E0F9000603D5286807B089
:105D5000BDE8F0839DF800004007BFD534702C608B
:105D60007946C8F800400020C9F80010EFE70000AD
:105D700004000010080000100C0000100000094092
:105D8000C0C62D004E1E0020841E0020FEB502A8B5
:105D900004F08EF9FE4C000637D49DF8080000256B
:105DA000FC4EFD4F1D2812D004F083F808B104F01A
:105DB00002F801A804F0C3F9000626D49DF80400F7
:105DC00028B1012809D002280BD003280ED0256065
:105DD0007846356038600020FEBD012008F018F9D3
:105DE00001E008F063FF00060FD410E08DF80050CA
:105DF000684604F0A4FE000607D4432019F02DFBEA
:105E0000000602D40CF04CFFEDE72068FEBD012037
:105E100010F0E6FBFEBD2DE9F0418AB0002606A891
:105E20000EF0A7FFDFF87083D94CDA4D932806D126
:105E3000286808286DD005286BD0062833D00021AB
:105E400008460EF0E6FF000663D405A900200FF017
:105E5000B9FA00065DD4D14F387858B1002101203D
:105E60000EF0D7FF000654D405A901200FF0AAFABE
:105E700000064ED409A805F09CF9000649D49DF807
:105E8000240038B3002101200EF0C3FF000640D4E7
:105E9000694601200EF097FF05280DD001203978C2
:105EA00081430ED10AE00020206079462860C8F8BE
:105EB00000100AB0BDE8F0810020F0E7397888438F
:105EC00008D0932020600820794628609320C8F8E5
:105ED0000010EEE702200EF0B2FF000619D469466A
:105EE00002200EF070FF000613D4002102200EF0F5
:105EF00090FF00060DD405A902200FF063FA206878
:105F0000932806D12868082803D1761CB6B2032E40
:105F1000F1D32068CDE72DE9F04F97B00BA804F03E
:105F2000B6F89B4C00067DD413A805F042F9000694
:105F3000F9D4DFF868821026DFF85C9298F8000048
:105F4000944D4FF0000A4FF0160B9227C0B10CA8E9
:105F50000DF030F840F3C010401C8DF81C0011D03B
:105F60009DF84100010637D59DF84C1099B38DF886
:105F7000206008A804F092F8032027602860C8E198
:105F80008DF81CA09DF84C0098F80010084217D01E
:105F90002868032811D004280FD08DF820B000BF46
:105FA0009DF82000FFF707FD286809283AD9462008
:105FB00019F053FA30202760E0E78DF82060EFE712
:105FC000FFF7E4FEABE100BF8DF8200008A804F065
:105FD00065F817B0DFE5FFE7C00603D50CF060FEFB
:105FE0000006A0D49DF84100000708D50DF02DF95A
:105FF000000698D46A4836F0DFF8000693D4FFF71D
:106000000AFFDFF8A081932815D09DF84100000712
:1060100075D50DF01AF9000685D4614836F0CCF834
:10602000000600E07AE183D407A90FA8FFF7C0FDBE
:10603000002863D113E0FFF7A9FE0006D1D40E209B
:106040008DF8200008A804F029F80006C9D4002122
:1060500055A035F09CFF594902200870CEE19DF80B
:106060001C00022804D0012871D0002870D0EFE174
:106070009DF8410040076CD568460CF02EFF0028C3
:1060800068D102E0FFF797FCE0E109A904200EF0D7
:10609000F5FE0006F8D4BDF82400BDF80010401C41
:1060A000814273D19DF84100800609D5FFF76EFE4D
:1060B0000DF0CBF80006E7D4394836F07DF80FE054
:1060C00015A804F03CF80006DED49DF85400012821
:1060D00016D0FFF75BFE0006D6D40BA803F0D7FF5F
:1060E0000006D1D4BDF8000014A9FFF70AFD20680E
:1060F0008228C9D092284AD093287AD133E184E10A
:1061000011A804F060F80006BED411AEB01C04F073
:106110006BF80006B8D4301D04F077F80006B3D44D
:1061200027499DF84800087008A803F0C1FF000641
:10613000AAD49DF8200004280DD0052854D01D288D
:1061400047D0FFF723FE08A803F0B2FFC8E7ABE093
:10615000B5E0A0E003E103F0ACFE30B103F02BFEAC
:1061600011A805F0F7FA00068ED4012600270AA927
:10617000304604F06FF9000686D40A98761CF6B211
:106180000744102EF3D927B31D201BE032E06CE04A
:1061900004000010080000100C000010084400006B
:1061A000082300104A1E00208E9888818A80208F44
:1061B000808C9F9288208F840A0A0000481E00204D
:1061C000C11E00208DF8200008A803F067FF00061C
:1061D00087D4B8F8001011A841F00401A8F8001005
:1061E00005F0B8FA00068FD406F018F900068BD433
:1061F000A9E73DE0FFF7CAFD000685D49DF8410000
:106200009DF82C1000F04000491E084306D1BDF84F
:106210002410BDF80000891C884214D00CF040FD09
:1062200000067BD414208DF8200008A803F036FF68
:10623000000673D44E2019F010F900066ED4012028
:1062400010F0CEF9C5E6401E80B214A9FFF759FC44
:106250002068822862D0922802D0932803D182E05D
:10626000286808287DD11320AEE62868082878D150
:106270009DF8500008B11520A6E608A803F018FF05
:1062800000064BD49DF820001D2869D047E001206E
:106290009AE6022098E68DF8206008A803F0FEFE3A
:1062A00000063BD4332007E08DF8206008A803F0F7
:1062B000F5FE000632D4412019F0CFF89EE0FFF73A
:1062C00065FD00062AD49DF841004FF0310610F01C
:1062D000600F29D09DF84C0008B38DF820B008A8B5
:1062E00003F0DCFE000619D4422019F0B6F808A924
:1062F00053201AF087F8000610D49DF8200010F003
:1063000002008DF8200002D0012010F069F927600A
:106310002E6079469220C9F800105AE680E09DF878
:106320002C000028B5D0B2E768460CF0D6FDB0B915
:1063300014A8FFF7B6FC822872D0922811D09328B7
:1063400011D09DF8500080B1022836D088202060FE
:106350000220794628608820C9F8001039E600E05C
:1063600076E00F208EE60E208CE60FF073FE012003
:1063700010F036F95E2019F070F80DF0BCFA000646
:1063800064D4FE4D0121FD4810F0B3F900060AD592
:10639000FDF74CFF0CF084FC000657D4FDF75BFFC3
:1063A0002078000652D40DF0E6FA00064ED495F897
:1063B00040000028E6D1182019E09DF84C0080B17B
:1063C0008DF820B008A803F069FE00063ED44220F4
:1063D00019F043F8B8F8001041F00201A8F80010D5
:1063E00092E79DF82C0008B1012000E002208DF812
:1063F000200008A803F052FE000627D4B8F80010C9
:1064000041F00201A8F8001019E7FFF7BFFC9DF862
:106410004C0000289DF82C000DD010B10C2001E09C
:1064200014E00D208DF8200008A803F037FE0006C8
:106430000CD4402040E708B1012000E002208DF894
:10644000200008A803F02AFE000601D52068C0E558
:10645000C4F800A07946C5F800A00020C9F80010D3
:10646000B7E510B5C648C74C86B0007820B1042007
:10647000FFF7FDF940B123E00620FFF7F8F9F8B97E
:106480000420FFF7F4F9D8B90120FFF7F0F9B8B903
:10649000372018F0E2FF02A9532019F0B3FF0006DD
:1064A00034D49DF8080010F002008DF8080007D0E1
:1064B000B548018841F002010180012010F090F8F8
:1064C000012004A9CDE90001024603AB0421092003
:1064D0001AF0B6FB000619D49DF80C00062818D156
:1064E00037F04FF9A8B932F088F900060ED46720CA
:1064F00018F0B3FF000609D4682018F0AEFF0006BC
:1065000004D4012010F06CF8000602D5206806B013
:1065100010BD9E4900202060086078469C490860B4
:106520000020F4E738B5684603F0C2FD954C00063C
:1065300029D4984D2878752827D00220FFF70CFA27
:1065400070B17B202870684603F0B9FD00061AD4AC
:106550001C208DF80000684603F0A0FD000612D450
:106560000120FFF7F9F980B151202870684603F047
:10657000A6FD000607D417208DF80000684603F03A
:106580008DFD000601D5206838BD9DF800000F285C
:1065900001D17E2028707D49002020600860784667
:1065A0007B490860002038BD2DE9FC41804603206E
:1065B0002CF03AFC754E764F724C002530B9B8F18C
:1065C000000F03D00420FFF7C7F9E8B36946532052
:1065D00019F018FF9DF8000010F002008DF800007F
:1065E00002D001200FF0FCFF3D2018F036FF9DF88F
:1065F000000010B101200FF0F3FF6649752008700C
:10660000684603F055FD00061BD4684603F068FD9C
:10661000000616D401A803F03AFD000611D49DF837
:10662000040008B1192000E01A208DF80000684627
:1066300003F034FD000604D40420FFF796F90006A9
:1066400003D52068BDE8FC8106E082202060784602
:10665000356038608220F5E725607846356038601F
:106660000020EFE72DE9F0438BB000273E4607A856
:1066700003F01EFD434C00067ED49DF81C00DFF89D
:106680000C81DFF80C910025022803D0192801D0D5
:106690001A2872D103A9352019F0B4FE00066BD474
:1066A0009DF80E0000F00F01000900EB800001EBE7
:1066B000400000F5FA60ADF814009DF80D0000F000
:1066C0000F01000900EB800001EB40008DF816007F
:1066D0009DF80C0000F00F01000900EB800001EBB9
:1066E00040008DF8170009A905A8FEF701FA03A9D3
:1066F000362019F087FE00063ED49DF80E0000F00B
:106700000F01000900EB800001EB400000F5FA608A
:10671000ADF814009DF80D0000F00F01000900EB2A
:10672000800001EB40008DF816009DF80C0000F091
:106730000F01000900EB800001EB40008DF817000D
:1067400008A905A8FEF7D4F968460AF02AF8000659
:1067500078D404A82CF0A4FB000673D4BDF8240060
:1067600010B3BDF8001081421ED39DF81000172809
:106770001AD2012703AB0FE064E067E020060010A7
:1067800008440000040000104A1E00200800001009
:106790000C000010C01E002035223946022003954F
:1067A0001AF094FA00064DD4BDF8200088B1BDF867
:1067B000001081420DD39DF8100050B1012603ABAB
:1067C00036223146022003951AF080FA000639D4A9
:1067D000E7BB56EA070045D006A9342019F012FE9F
:1067E00000062FD49DF81800012826D0022804D0D6
:1067F000032837D14D497D20087006A9532019F090
:1068000001FE00061ED49DF8180010F002008DF85D
:10681000180004D001200FF0E3FE000612D40EB1E0
:10682000482000E0472018F018FE9DF8180020B11D
:1068300001200FF0D5FE000604D404A82CF030FB94
:10684000000604D520680BB0BDE8F0830AE09DF88F
:1068500010000EB1401E00E0401C8DF8100004A88E
:106860002CF083FB25607946C8F800500020C9F859
:106870000010E8E738B50546684603F019FC2C4CD3
:10688000000604D4284603F002FC000601D5206867
:1068900038BD9DF8001006290FD008DC01290CD066
:1068A00003290AD0042908D0052908D105E00729C1
:1068B00003D0132901D0152901D1012028701D49C9
:1068C00000202060086078461B490860002038BD21
:1068D00038B50546684603F0FCFB154C000618D495
:1068E0009DF80010072916D006DC0DD2DFE801F074
:1068F0000C130C13131313000E290CD013290AD0F8
:10690000152908D01B2906D0284603F0C0FB000635
:1069100003D5206838BD012028700649002020607A
:106920000860784604490860002038BDC01E002079
:1069300004000010080000100C00001010B58AB010
:1069400005A835F05FFCCF4C000637D4684635F01B
:1069500059FC000632D40220ADF80A00ADF802005E
:10696000ADF804000A20ADF806000021684635F0B5
:1069700095F9000622D40021C3A035F008FB0006DB
:106980001CD40021C3A035F002FB000616D401215F
:10699000084635F019F9000610D40021BEA035F0E4
:1069A000F6FA00060AD4002105A835F077F90006AA
:1069B00004D4012035F072F8000602D520680AB030
:1069C00010BD35F0B0FCFAE72DE9F04F8346A5B0D5
:1069D0000D46084635F08EF8AA4C00067DD4584680
:1069E00035F029F900067DD42B465A46B1A16846F8
:1069F0003CF0DEFA0021684635F0C9FA000671D491
:106A0000B2482A22C589684629463CF096FE0A20EB
:106A10000DF805000DF101014FF0000905F8019096
:106A20004946684635F0B3FA00065BD435F0A5FD5B
:106A3000DFF89CA20646DFF89C829AF80000022844
:106A400005D000EB400108EBC10040688047A24F31
:106A5000BD680021A14835F09AFA000642D4002111
:106A60009E4835F094FA00063CD4002189A035F008
:106A70008EFA35F082FD861BB868411B4FF47A70A0
:106A8000B1FBF0F59AF80000022805D000EB4001B8
:106A900008EBC1004068804706EB4600C0EBC6101B
:106AA00005EBC000401EB0FBF5F7ABF1010035F07F
:106AB00067FD4FF47A714E436843B6FBF0F2FF1D59
:106AC000FB0887A168463CF073FA684635F04FFC36
:106AD000000607D400218AA000E003E035F057FA51
:106AE000000603D5206825B0BDE8F08F8549C4F8BD
:106AF00000907846C1F80090834908600020F2E7D2
:106B000070B58AB0064605A835F07CFB5D4D0006E1
:106B10003CD4684635F076FB000637D40121ADF849
:106B20000210ADF80060BDF81400ADF80410ADF827
:106B30000A10ADF80610401E35F029FDBDF82210F0
:106B400000FB01F4BDF80000401E35F020FD94FB71
:106B5000F0F0ADF80E000121684635F09FF8000610
:106B600014D40424032E02D10D2C00D10E2421466E
:106B70003046FFF729FF000608D4E41C0F2CF1D3A0
:106B8000002105A835F08AF8000602D528680AB069
:106B900070BD5C4900202860086078465A4908604A
:106BA0000020F4E710B5002035F045F8354C00061C
:106BB00035D400213EA035F0EAF900062FD401219A
:106BC000084635F001F8000629D400214FA035F021
:106BD000DEF9000623D40221012034F0F5FF00067F
:106BE0001DD4002149A035F0D2F9000617D40121A7
:106BF000022034F0E9FF000611D4002143A035F053
:106C0000C6F900060BD40221084634F0DDFF000669
:106C100005D400213DA035F0BAF9000601D5206861
:106C200010BD384900202060086078463649086069
:106C3000002010BD10B5012034F030FF114C0006CB
:106C400019D40121084634F0BFFF000613D40520F3
:106C500034F050FF00060ED4204B1822A5336421D7
:106C6000002035F058F9000605D400212AA035F09F
:106C70008EF9000601D5206810BDBDE81040012046
:106C800035F086B804000010465072696E742D32DB
:106C9000320000000A00000084A5ACAEADE1E2E0E5
:106CA000A0E6A8AEADADA0EF20AFA5E7A0E2EC0A4C
:106CB000200A0000200A98908894922025752C20A4
:106CC0009F908A8E91929C2025750A0008230010BF
:106CD000E81E00203403001000000940A0610400F9
:106CE000D1EAEEF0EEF1F2FC3A20257520D1D2D0B7
:106CF0002FD12028257520CCCC2FD1290A000000C7
:106D00000A200A00080000100C0000103132352063
:106D1000544543540A0000002034203630323234C7
:106D200032203030313733370A200A200A00000081
:106D300070B5B8B0022034F0B1FEB04D00067CD47E
:106D40000221084634F040FF0006F8D4ACA2AFA1FF
:106D500002A83CF02DF9002102A835F018F9012114
:106D6000084634F031FF0006E9D4A9A035F0FFFA57
:106D7000012034F093FEA2A2A4A102A83CF018F9CD
:106D8000002102A835F003F902A801F0C0F802A81A
:106D900000F070FD002102A800F029FD02A801F01A
:106DA000CBF8002102A800F09AFF02A801F0B3F985
:106DB000202229A99B482EF0BFF902AA98A19AA0E7
:106DC00000F09DFC02A835F0D2FA9AA131A8299AC8
:106DD0003CF0EEF802AA31A998A000F090FC02A8BD
:106DE00035F0C5FA93A131A82A9A3CF0E1F802AA3D
:106DF00031A997A000F083FC02A835F0B8FA8DA164
:106E000031A82B9A3CF0D4F802AA31A995A000F041
:106E100076FC02A835F0ABFA86A131A82D9A3CF099
:106E2000C7F802AA31A993A000F069FC02A835F0C6
:106E30009EFA80A131A82E9A00E0D3E03CF0B8F889
:106E400002AA31A990A000F05AFC02A835F08FFAEE
:106E500078A131A82F9A3CF0ABF802AA31A98FA0F3
:106E600000F04DFC02A835F082FA684634F008FACA
:106E70008EA131A8009A3CF09BF802AA31A98DA0FE
:106E800000F03DFC02A835F072FA02A800F03DFDCA
:106E90008DA035F06CFA35A831F0D3FE3598012875
:106EA00030D0042830D0052830D08AA102AA8BA087
:106EB00000F025FC02A835F05AFA8C4C202202A8DA
:106EC000E1893CF03AFC0E2289A102A83CF0C6FB05
:106ED00036A90120CDE90001014627AB0222092095
:106EE00019F0AEFE00067FD49DF89C3001A80A225E
:106EF000411E0A2B50D2DFE803F04F0B0F4F161A3A
:106F00001E262A4B7EA1D1E77FA1CFE77FA1CDE747
:106F1000E189084480A102E0E189084480A1096870
:106F2000016002711DE0E18908447FA1F7E7E08973
:106F300008447FA102E0E08908447FA10A6802605A
:106F4000898881800DE0E08908447DA1F6E7E18928
:106F50000DF1020008447CA10B68036089888180E0
:106F6000827102A835F003FA02AA79A17AA000F092
:106F7000C6FB02A835F0FBF97C4800788DF89C0030
:106F800070B101280FD0022802AA30D024A10CE051
:106F9000E089084476A1D1E7E189084476A1BEE7FB
:106FA00002AA77A101E002AA77A179A000F0A7FBCD
:106FB00002A835F0DCF931F020FC012034F0E8FEC5
:106FC000552018F04AFA28A803F0CAF800060BD496
:106FD00028A802F08DFC000606D428A803F0B6F815
:106FE000000600E000E004D5286838B070BD6DA14F
:106FF000DBE701200FF0F4FAF7E7000004000010CF
:10700000465072696E742D323200000025730A00FA
:10701000C8CDD4CED0CCC0D6C8DF20CE20CFC40AB5
:107020000000000008000020CDC0D0C0C1CED2CAF0
:10703000C00000002531306C7500000020C02DCE4E
:10704000D2D0C5C7D72E2CC2D1C5C3CE00000000F8
:1070500020C4C2C8C3C0D2C5CBDC2CC2D1C5C3CEEC
:107060000000000020C3CECBCEC2CAC02CC2D1C506
:10707000C3CE000020C02DCED2D0C5C7D72E2CD174
:10708000C1D0CED10000000020C4C2C8C3C0D2C548
:10709000CBDC2CD1C1D0CED10000000020C3CECBA0
:1070A000CEC2CAC02CD1C1D0CED10000253264439B
:1070B00000000000D2C5CCCFC5D0C0D2D3D0C020F4
:1070C000C3CECBCEC2CAC800D1C2DFC7DC20D1201C
:1070D000CFCA0A00556E6B6E6F776E0020CAC0CDA6
:1070E000C0CB20CEC1CCC5CDC0000000082300100D
:1070F00020D1CACED0CED1D2DC20C1DBCBC00000A3
:1071000052532D3233320000555342004554484506
:10711000524E455400000000313230300A00000069
:10712000323430300A000000393630300A000000B6
:1071300031343430300A000033383430300A000043
:1071400035373630300A00003131353230300A0000
:10715000343830300000000020D1CACED0CED1D299
:10716000DC20C2D0C5CCC5CDCDCE0000E81E0020AD
:1071700031393230300A0000343830300A00000033
:10718000C0D2CECB00000000D8D2D0C8D5000000BD
:1071900020CFD0CED2CECACECB20CEC1CCC5CDC092
:1071A00000000000C0D2CECB20CDCEC2DBC9000093
:1071B0002DE9F843F44DF54FDFF8D483002440B9AE
:1071C000694601202BF02AF9000617D40098C00761
:1071D0001DD0F04E3088800506D5012200211046D2
:1071E00009F02CFF000609D43078000609D50122E9
:1071F0001146002009F022FF000602D52868BDE8EC
:10720000F883308810F4207F08D1800406D42C60E5
:1072100079463C600020C8F80010F0E74FF4FA749B
:10722000FA2120462DF08BFD214600202DF087FD10
:10723000F6E72DE9F04F95B04FF00009D24FDFF897
:1072400058B3CDF84890DFF844A33B68CBF8003042
:10725000DAF80000CF49DFF83883CBF804007F2646
:10726000CE4C0988D8F800204D46892B10D010DC70
:10727000812BFBD006DC062B77D2DFE803F0F7F793
:1072800076F7F7F7822B71D0862BEFD0872B6CD156
:10729000ECE0932B14D00ADCA3F18A010929EBD28C
:1072A000DFE801F0E463636363FBE4E43E00962BF4
:1072B00070D0A12BECD0A22BFAD0A32BE7D12EE1DA
:1072C0000A2819D008DC052816D00628E0D008289E
:1072D00012D0092806D10FE00B280DD0802819D034
:1072E000812817D00090AE4901A83BF061FE002133
:1072F00001A834F04CFE03E009B9AAA00DE0042572
:10730000B0492670022008704B2018F0A6F8FF2D17
:107310003CD1EAE00029F2D1ABA00EF0DEFCEEE7B2
:10732000FCF784FF13A803F044FFFCF794FF9DF8DB
:107330004C0000287DD0DAF8000008282BD00ADCA9
:1073400019D2DFE800F018282828282828283860D3
:10735000CAF800003FE02A2819D008DC09281AD012
:10736000202814D0282806D111E0A8E040E03028D9
:1073700038D0312836D000219DA034F008FE267088
:107380009049022008704B2018F067F8A6E00EF034
:1073900066FC2AE0C1E00EF062FC8A49CBF800905E
:1073A0000220CBF8049008704C4612A9532019F023
:1073B00029F800066FD4129810F00200129007D03E
:1073C0009248018841F00201018001200FF008F984
:1073D0003C60CAF8004079460020C8F8001015B09B
:1073E000BDE8F08F082034F0E3FF7E202070C7E76F
:1073F000252864D2DFE800F0631E1E2B2B256313C3
:10740000296340323A6340636336633A3A636363A5
:107410001E2B3434633A63633A5C5C632B0031B9EE
:1074200068490220087000215EA034F0B0FD0425F8
:1074300053E070E019B9002175A034F0A8FD0225D1
:107440004BE000217BA034F0A2FD012545E019B9F5
:10745000002181A034F09BFD03253EE00A253CE09D
:1074600009253AE0844800780228F5D0CBF800904E
:107470004846CBF804906AE714A9622018F0C2FFCE
:10748000000608D49DF850000007EFD5684602F0CA
:1074900086FF000602D53868A1E71AE09DF80000D3
:1074A0000028E3D05948018841F080010180DDE7E0
:1074B00019B9002171A034F06AFD08250DE0009093
:1074C000374901A83BF074FD002101A834F05FFDAD
:1074D00003E003281FD007281DD026706D00FF2D64
:1074E00003D012A9284600F01FF80020FFF760FE25
:1074F00036F014F8694C6A4E207800EB400006EB39
:10750000C00040688047207800EB400006EBC000D8
:1075100080688047E3E7484619E70428FBD07946AE
:107520001846C8F800105AE770B5040008680D4600
:1075300005D0611E88420FD14FF4FA6110E059491D
:10754000584A363A31F9101032F910002DF0A9FBE3
:10755000002818D11B240CE0C00703D04FF4FA71A7
:10756000002002E0C8214FF416702DF09AFB00288D
:1075700009D101202AF0AFFF2868401C2860A042F2
:1075800001D10020286070BD040000100800001028
:107590000C0000104C1E0020501E0020C01E0020B9
:1075A000B05505008EE8A8A1AAA020AFA0ACEFE2DC
:1075B000A8208F84200A0A0A0A0A0A0A0A0A0A0A62
:1075C0000A0A0000481E002091A1AEA920AEA1AC7D
:1075D000A5ADA020E120AFA0ACEFE2ECEE208F84BF
:1075E000200A0A0A0A0A0A0A0A0A0A0A0A0A0000F9
:1075F0008EE8A8A1AAA0209D8A8B870A0A0A0A0AF7
:107600000A0A0A0A0A0A0A0A000000004A1E0020A2
:1076100091A1AEA920AEA1ACA5ADA020E1209D9185
:107620008F87930A0A0A0A0A0A0A0A0A0A0A0A0A2F
:10763000000000008220E7A0E1A0E520ADA5A2A502
:10764000E0ADAEA520A2E0A5ACEF0A0A0A0A0A0A3C
:107650000A0A0A0A0A0A0A0091A1AEA920AEA1AC40
:10766000A5ADA020E1208E87930A0A0A0A0A0A0A19
:107670000A0A0A0A0A0A0000A803001091A1AEA98A
:1076800020AEA1ACA5ADA020E1208F8F87930A0A80
:107690000A0A0A0A0A0A0A0A0A0A0A00E81E002056
:1076A00034030010946204002DE9F041804634F068
:1076B0005EFE002821D0FA4CFA4D4FF496764FF436
:1076C000FA7701202AF007FF314638462DF037FBC4
:1076D00001202AF000FFA068A168091AA942FBD383
:1076E00034F021FE0028ECD10021EFA034F04FFC53
:1076F0004046BDE8F04134F03ABEBDE8F0812DE9E6
:10770000F05F14468B4682463BF0FEFE81465846AB
:107710003BF0FAFEE54D064609EB0600E9890A272B
:107720004FF00008884217D2202220463CF005F88E
:107730004A46514620463BF006FFE8893246801B08
:10774000204459463BF0FFFEE8892754E989641C30
:1077500001F80480BDE8F09F012000EB41012022E8
:1077600020463BF0EAFF4A46514620463BF0EBFEFE
:10777000E889324659462754E889C6EB4000204440
:10778000401C3BF0E0FEE88904EB40004770E989CB
:1077900004EB410181F80280DCE710B5044686B0B5
:1077A000012034F07BF905A904A80CF040FEC0A02C
:1077B000FFF77AFF049864214843059990FBF1F2A2
:1077C000C0A168463BF0F4FB22466946BFA0FFF724
:1077D00096FF2046FFF768FFC04900200860C049B7
:1077E00008607846BF49086006B0002010BD30B57B
:1077F00085B00546002004900C4604A82DF0D8FB67
:10780000FCF714FD0499642091FBF0F200FB1212C6
:107810000A2392FBF3F391FBF0F2B3A168463BF02D
:10782000C7FB2A466946B3A0FFF769FF2846FFF762
:107830003BFFFCF710FDAA48006814B111280ED0D8
:1078400010E011282A4608D0B1A19FA0FFF757FFEA
:107850002846FFF729FF05B030BDAFA1F5E7206846
:10786000401C2060AEA1684622683BF0A1FB2A467E
:107870006946EAE770B5044688B0012034F00EF995
:107880008A4E01252846FEF733F8002838D02A46CC
:10789000A6A120463BF08CFB2046FFF705FFF189AF
:1078A000202220463BF049FF07A91420CDE9000122
:1078B00002AB012229460A2019F0C2F92846FDF739
:1078C000D6FF50B1079A611C530002A8FDF76EF96C
:1078D000F189201F084499A109E007985822410026
:1078E000601C3BF02AFFF189A01F084495A13BF0E2
:1078F0005FFBF289601C002111542046FFF7D4FE83
:107900006D1C1E2DBEDB08B070BD10B504468CB0DA
:10791000012034F0C3F88DA0FFF7C6FE8E490A8817
:10792000A2F5194099382FD08CA168463BF040FB56
:10793000224669468BA000BFFFF7E1FE2046FFF715
:10794000B3FE09A90AA80DF018FDBDF8242083A1F3
:1079500068463BF02DFB2246694683A0FFF7CFFE29
:107960002046FFF7A1FE40F204407CA10288684651
:107970003BF01EFB224669467CA0FFF7C0FE204676
:10798000FFF792FE0CB010BD79A27CA168463BF0D7
:107990000FFB2246694673A0FFF7B1FE2046FFF7B2
:1079A00083FE774A75A168463BF002FB2246694692
:1079B00074A0FFF7A4FE2046FFF776FE734A6FA17E
:1079C00068463BF0F5FA2246694671A0B4E710B567
:1079D0000420FDF7CAFF0106404801D5006810BD2C
:1079E000002101603E48016078463E490860002061
:1079F00010BD6948002100F8081FFF2101760177BA
:107A000080F820107047F0B5074687B00C46002676
:107A100003202BF009FAD0B101263046FFF7D7FF3B
:107A200000283BD18DF800008DF801008DF8020090
:107A300040F2DA70ADF8140001208DF816008DF8D0
:107A4000170005A82BF0B2FA68462BF08EFA6846AC
:107A50002BF026FA12499DF8025088684F4A8B682D
:107A60001B1A9342FBD368462BF01AFA0EB1FFF7AC
:107A7000C0FF9DF8020064B1A84202D12068401CFA
:107A8000206027A101A822683BF092FA3A4601A99A
:107A900088E0A8423A4602D01DA183E088E07FE05A
:107AA0000000094020A107000A0000000823001080
:107AB000CFC0CCDFD2DC20C1D3D4C5D0C020CACB4C
:107AC0000A0000002575252500000000C8D1CFCE92
:107AD000CBDCC7CEC2C0CDCE000000000400001039
:107AE000080000100C00001025752E25303175C2DD
:107AF00000000000C1C0D2C0D0C5DF20D7C0D1CEA9
:107B0000C228322E32202D20332E332900000000CF
:107B1000CDCED0CC00000000CDC5CDCED0CC000065
:107B20002530346420CED8C8C1CECA00CACEC42005
:107B3000C7C0D9C8D2DB2025750A0000CDCED0CC75
:107B40000A000000CDC5CDCED0CC0A00494420D1DA
:107B5000C5D0C8C83A0A0000044400002530347576
:107B6000000000002031000020320000203300001F
:107B7000CED2CBC0C4CED7CDC0DF0000257300006D
:107B80001044000020C4E0F2E03A0000204400006D
:107B900020C2F0E5ECFF3A0000400240E0C81000CF
:107BA000AFF28C01FBA0FFF7AAFD3846FFF77CFD82
:107BB00007B0F0BD30B50C00F9A187B00546D1E99A
:107BC0000001CDE900010ED02BF032FA10B120688F
:107BD000401C2060AFF2B80102A822683BF0E8F92F
:107BE0002A4602A908E02BF023FA2A4610B1AFF288
:107BF000D80101E0AFF2E8016846FFF780FD2846B2
:107C0000FFF752FD07B030BD30B5E7A30C4605467F
:107C10000FCB89B08DE80F0008A908460DF0ADFB29
:107C2000E5480068D0B109282A4620D0E3A168467B
:107C3000FFF765FD6CB12068401C2060AFF2201199
:107C400004A822683BF0B4F92A4604A96846FFF765
:107C500056FD2846FFF728FD09B030BD2A46AFF291
:107C600050116846FFF74BFD002CE7D1F1E7AFF26A
:107C700058116846FFF743FD002CEAD02168491CE3
:107C80002160DBE77FB50C46054619F077F880B137
:107C9000C9482A460068012809D0AFF28411C8A05B
:107CA000FFF72DFDBCB12068401C206008E0C3A197
:107CB000F5E72A46AFF2A811C1A0FFF720FD54B1A5
:107CC000AFF2A411684622683BF072F92A46694671
:107CD000BBA0FFF714FD2846FFF7E6FC7FBD7FB58C
:107CE0000C4605462EF048FD30B12A46B3A10FE000
:107CF0002068401C206018E00CF08FFA70B1AE488C
:107D0000016803290AD0042908D02A46AFF2F811E5
:107D1000ADA0FFF7F4FC002CEAD111E02A46AFF247
:107D20001021A9A0FFF7EBFC54B1AFF20C2168467B
:107D300022683BF03DF92A466946A3A0FFF7DFFC25
:107D40002846FFF7B1FC7FBD30B50546A0A085B041
:107D500000680C46049003F086F9000607D42A4612
:107D6000AFF2542104A8FFF7CAFC6CB917E092489F
:107D70002A460068192816D090A104A8FFF7BFFC76
:107D80006CB12068401C2060AFF26C21684622680C
:107D90003BF00EF92A46694604A8FFF7B0FC2846D6
:107DA000FFF782FC57E5AFF29021E6E72DE9F043BB
:107DB000814688A00C468BB007C801AB002683E83B
:107DC0000700012033F06AFE08A80CF0D2FF7A4DBC
:107DD000932803D12868062800D0012600210846F0
:107DE0000DF017F8002712E02868082815D117B9F8
:107DF0007BA0FFF759FCBDF8002080A14846521C2B
:107E00003BF0D6F84846FFF74FFC01267F1C694639
:107E100000200DF0D7FA0028E6D1DFF8E881D8F885
:107E20000000932800D10126002101200CF0F1FF71
:107E3000002712E02868082815D117B972A0FFF7AB
:107E400033FCBDF800206DA14846521C3BF0B0F851
:107E50004846FFF729FC01267F1C694601200DF0EA
:107E6000B1FA0028E6D1D8F80000932800D1012605
:107E7000002102200CF0CDFF002712E0286808281E
:107E800015D117B967A0FFF70FFCBDF800205BA163
:107E90004846521C3BF08CF84846FFF705FC01268B
:107EA0007F1C694602200DF08DFA0028E6D1D8F833
:107EB000000093280BD096B14A46AFF2A43101A836
:107EC000FFF71DFCECB12068401C20600EE0286824
:107ED000802801D08128EFD14A4638A1EFE74A46F1
:107EE000AFF2D43101A8FFF70AFC54B1AFF2D031A0
:107EF00004A822683BF05CF84A4604A901A8FFF7F1
:107F0000FEFB4846FFF7D0FB0BB0BDE8F0833EB563
:107F100004462BF098F800F00F03C0F3031247A1BA
:107F200068463BF045F82246694646A0FFF7E7FB66
:107F30002046FFF7B9FB3EBD70B58AB0064605A8DE
:107F40000CF017FF20B13F220C2105A83BF0F5FBF8
:107F500000258DF820502022052105A83BF0EDFBDF
:107F6000324605A93CA0FFF7CAFB3046FFF79CFB51
:107F700000200CF064FF234C20B9694600200CF06F
:107F800022FF28B13F22142105A83BF0D6FB74E064
:107F90006AE00000D5CEC420D7C0D1CEC200000018
:107FA000CFCE20CFC4000000CFCE20CFC0CCDFD2B8
:107FB000C820CFC40000000008000010CDC5D200CA
:107FC000DDD1CFCFC7D30000CFCFC7D30000000093
:107FD000CEC7D300CFE0ECFFF2FC20CFC4000000FE
:107FE000CFCEC2D0C5C6C4C5CDCDDBC520D4C8D187
:107FF000CAC0CBC8C7C0D6C8C83A0A002325303487
:10800000750A000004000010CFCEC2D0C5C6C4C59A
:10801000CDCDDBC520C0CAD2C8C2C8C7C0D6C8C86B
:108020003A0A0000CFCEC2D0C5C6C4C5CDCDDBC58F
:1080300020D1CCC5CDDB3A0A0000000025752E25E5
:1080400075000000DDCBC5CAD2D0CECDCDDBC920B6
:10805000C1CBCECA00000000D1C5D0C8C9CDDBC994
:1080600020CDCECCC5D000000A23052205A90DF1F4
:108070000B00FCF79BFD00063AD48DF81E503246EB
:1080800005A9F9A0FFF73BFB3046FFF70DFB9DF874
:1080900014003F2816D0BDF8000005A9FCF718FE13
:1080A000000625D4324605A9F5A0FFF728FB304687
:1080B000FFF7FAFAF748007828B301200CF0BFFE6A
:1080C00050B904E0F4A105A83BF0FAF9EAE76946E3
:1080D00001200CF078FE20B1EFA105A83BF0F0F9EB
:1080E00009E0BDF8000005A9FCF7F2FD000602D585
:1080F00020680AB070BD324605A9EAA0FFF7FFFA72
:108100003046FFF7D1FAEC48256005607846EB4928
:1081100008600020EDE710B58CB004461822E8A1F5
:1081200005A83BF09BFA0BA803F043F89DF82C0040
:1081300008B1E9A101E0AFF27C11224605A8FFF7E2
:10814000DEFA2046FFF7B0FA9DF82C00002879D01F
:10815000694600200CF0D5FD002873D1BDF8002041
:10816000DEA101A8521E3AF023FF224601A9DDA09C
:10817000FFF7C5FA2046FFF797FABDF80000D7A130
:10818000C0F1190201A83AF013FF224601A9DAA0B2
:10819000FFF7B5FA2046FFF787FA694602200CF090
:1081A000B0FD00284ED1BDF80020AFF2506101A80B
:1081B0003AF0FEFE224601A9D2A0FFF7A0FA20461F
:1081C000FFF772FA04A902200CF06CFD002839D1E7
:1081D000BDF81000BDF80010421AAFF2806101A88E
:1081E0003AF0E6FE224601A9C3A0FFF788FA20462E
:1081F000FFF75AFAA7480078002823D069460120E3
:108200000CF07FFD00281DD1BDF80020B3A101A80E
:108210003AF0CEFE224601A9BCA0FFF770FA204634
:10822000FFF742FABDF80000ACA1C0F1400201A87E
:108230003AF0BEFE224601A9AFA0FFF760FA204641
:10824000FFF732FA0CB010BDF0B5074695B00C46FA
:10825000002503200BF07FF8B14E000602D53068F0
:1082600015B0F0BD0BF090F8000605D411A905205B
:108270000AF04AFF00060AD514B12068401C2060AD
:1082800001253F220A2168463BF057FA14E00A23F1
:108290000522694611A8FCF789FC13A900200AF001
:1082A00033FF000608D49DF84C00000604D514B135
:1082B0002068401C2060012500208DF80A006A46D5
:1082C00098A105A83AF074FE44B1AFF2AC710DA8C4
:1082D00022683AF06DFE3A460DA906E015B1AFF2FC
:1082E000C87101E0AFF2D8713A4605A8FFF707FA66
:1082F000FBF79CFF3846FFF7D7F9FBF7ACFFAEE77B
:1083000070B5064688B003200BF025F8844C0006B3
:1083100002D5206808B070BD0BF036F828B1FBF725
:1083200085FF3246AFF26C3109E005A905200AF05D
:10833000EBFE30B1FBF77AFF3246AFF624015CA0CA
:108340004BE00A230522694605A8FCF72FFC00250F
:108350008DF80A503246694655A0FFF7D0F93046ED
:10836000FFF7A2F904A900200AF0CEFE9DF8100044
:10837000000701D558A101E0AFF2C03132466CA030
:10838000FFF7BDF93046FFF78FF99DF81000400761
:1083900001D551A101E0AFF2DC31324668A0FFF710
:1083A000AEF93046FFF780F99DF81000000601D5C0
:1083B00049A101E0AFF2FC31324665A0FFF79FF919
:1083C0003046FFF771F968460BF0FAFD68B1FBF72C
:1083D0002DFF3246AFF6C00163A0FFF790F930469B
:1083E000FFF762F9FBF737FF93E7324669465EA075
:1083F000FFF785F93046FFF757F92F4825600560EC
:1084000078462E490860002084E770B5584C054630
:10841000B222E1893BF091F9E1890A2068540321F5
:1084200054A034F07EF800240021284633F0AFFD3C
:10843000641C0A2CF8D333F076FFBDE870400820A6
:1084400033F08ABB10B50446012030F0BBF92BF0A5
:10845000ACF8A0F55960B0F5C04F224602D0AFF697
:1084600048118BE088E00000D0C5C3C8D1D2D0C08D
:10847000D6C8CECDCDDBC920CDCECCC5D000000036
:10848000C4C0D2C020D0C5C3C8D1D2D0C0D6C8C8FD
:1084900000000000084400003F3F2D3F3F2D3F3FBC
:1084A00000000000C4C0D2C020C7C0CCC5CDDB20B6
:1084B000DDCACBC700000000080000100C0000104F
:1084C000CFC0CCDFD2DC20CFC420C0CAD2C8C2C843
:1084D000C7C8D02E00000000C4C00000253032758F
:1084E0000000000020CFC5D0C5D0C5C3C8D1D2D0B0
:1084F000C0D6C8C9000000002020D1C2CEC1CEC461
:10850000CDCE000020D1CCC5CD00000020C0CAD205
:10851000C8C2C8C7C0D6C8C920DDCACBC7000000C2
:1085200004000010DDCACBC72028257329000000F5
:1085300020C0CAD2C8C2C8C7C8D0CEC2C0CDC00031
:1085400020C0D0D5C8C220CED2CAD0DBD200000015
:1085500020CDC5C8D1CFD0C0C2C8CCC0DF20CED8B6
:10856000C8C1CAC00000000020C2C5D0D1C8DF0009
:10857000082300101B330000AFF66C21FEA0FFF7AC
:10858000BEF82046BDE81040FFF78EB870B505462E
:108590000C46FAA0FFF788F8FAA0FFF785F804F078
:1085A0000F0003282ED0FBA0FFF77EF8E00708D0CD
:1085B0002A46AFF69C21FDA0FFF7A1F82846FFF759
:1085C00073F8A00708D52A46AFF6B421F9A0FFF743
:1085D00096F82846FFF768F8600708D52A46AFF6F0
:1085E000C821F6A0FFF78BF82846FFF75DF82007B3
:1085F00008D52A46AFF6E021F2A0FFF780F828461A
:10860000FFF752F8C4F303100C2818D0EFA0FFF7BF
:108610004BF8600608D42A46AFF60431E7A0FFF70E
:108620006EF82846FFF740F8200608D42A46AFF631
:108630001831E4A0FFF763F82846FFF735F8C4F3D4
:1086400003200A2818D0E6A0FFF72EF8600508D509
:108650002A46AFF63C31D9A0FFF751F82846FFF77C
:1086600023F8200508D42A46AFF65431D5A0FFF7E9
:1086700046F82846FFF718F8C4F30330052818D049
:10868000DDA0FFF711F8600408D42A46AFF6783170
:10869000CAA0FFF734F82846FFF706F8200408D5EB
:1086A0002A46AFF68C31C7A0FFF729F82846FEF717
:1086B000FBFFC4F3034003281AD0D5A0FEF7F4FF54
:1086C000600308D52A46AFF6B031BCA0FFF717F813
:1086D0002846FEF7E9FF20030AD52A46AFF6C8313F
:1086E000B8A0FFF70CF82846BDE87040FEF7DCBFE5
:1086F00070BD70B505460C46A0A0FEF7D5FFCAA018
:10870000FEF7D2FF04F00700042823D0A1A0FEF753
:10871000CBFFE00708D02A46AFF60441C8A0FEF719
:10872000EEFF2846FEF7C0FFA00708D52A46AFF6A1
:108730001841C5A0FEF7E3FF2846FEF7B5FF600726
:1087400008D42A46AFF63041C1A0FEF7D8FF28462C
:10875000FEF7AAFFC4F3C20003281AD0BEA0FEF79A
:10876000A3FF200708D42A46AFF65441B4A0FEF771
:10877000C6FF2846FEF798FFE0060AD42A46AFF661
:108780006841B1A0FEF7BBFF2846BDE87040FEF788
:108790008BBF70BD2DE9F043C3B0002439943A94E7
:1087A0003B943C943D943E943F94409432A8419431
:1087B00033F028FDAB4D00062CD40221ADF8D210C9
:1087C00001213020ADF8CA10ADF8D600ADF8CC10BC
:1087D000ADF8C8100821A0462046ADF8D440ADF849
:1087E000CE1033F0D4FE4FF41074B4FBF0F0BDF8AB
:1087F000D610884208D2BDF8C800401E33F0C7FE2C
:10880000B4FBF0F0ADF8D600012132A833F046FAFF
:10881000000603D5286843B0BDE8F083022033F09A
:10882000E1FD91A0FEF740FF012033F037F995A05C
:10883000FEF73AFFDFF8689299F8000018B199A0A6
:10884000FEF732FF15E0082033F0B2FD00240021CE
:1088500097A033F09CFB30B9012033F071FD10B9C3
:1088600033F061FD08B1FEF7E4FC641CA4B20A2CED
:10887000EDD3012033F012F98EA0FEF715FF08208A
:1088800033F096FD934F0026002029F0EBFD48B110
:10889000022033F003F983A0FEF706FF012033F036
:1088A000FDF808E033F0E9FD38880643B6B27007FA
:1088B000EAD5B007E8D533F0E0FD38880028FAD1D2
:1088C000854CA068854DA168091AA942FBD384A0F4
:1088D000FEF7EAFE012033F0E1F829A80CF049FA8E
:1088E00020B13F220C2129A83AF027FF8DF8B08053
:1088F0002022052129A83AF020FF03AA29A97DA05A
:10890000FEF7FDFE03A8FEF7CFFE2FA82AF0F9FA26
:1089100018B930A82AF0C4FA20B177A103A83AF018
:10892000CFFD12E0BDF8BC209DF8C100A2F5FA62AF
:108930009DF8C0100092CDE901109DF8BE309DF861
:10894000BF2072A103A83AF033FB032033F0A6F84E
:1089500003A8FEF7A9FE012033F0A0F803A8FEF754
:1089600089FF71A273A103A83AF022FB002103A89A
:1089700033F00DFB03A8DFE0555342003F3F3F209B
:1089800000000000205749464920D7C0D1D2DC0A58
:108990000000000020C2D1C520D1C8C3CDC0CBDBB0
:1089A00020CDC020C2D5CEC40A0000002020CFC8F0
:1089B000CD2037002020CFC8CD2038002020CFC8C0
:1089C000CD2036002020CFC8CD20350020CFC8CD07
:1089D000203720C820CFC8CD203820C220300A0040
:1089E00020CFC8CD203720C220302C20CFC8CD20AA
:1089F0003820C220310A000020CFC8CD203720C245
:108A000020312C20CFC8CD203820C220300A0000D1
:108A100020CFC8CD203720C220312C20CFC8CD2078
:108A20003820C220310A00002047534D2F424C55B8
:108A300045544F4F544820D7C0D1D2DC0A00000023
:108A40002020CFC8CD2033002020CFC8CD20320039
:108A50002020CFC8CD20310020CFC8CD203120C26A
:108A600020300A00040000103D20D2C5D5CDCECB69
:108A7000CEC3C8D7C5D1CAC8C920CFD0CEC3CECDEA
:108A8000203D0A00D2C5D1D220CDCEC6C020C0C262
:108A9000D2CECED2D0C5C7D7C8CAC00A0000000007
:108AA000411F0020CFD0CECFD3D9C5CD0A000000C2
:108AB0000A0A0A00D2C5D1D220C4C0D2D7C8CACEB1
:108AC000C220CAD0DBD8CAC820C820C1D3CCC0C3FA
:108AD000C80A0000561F00200000094020A107001E
:108AE0003D3D3D2020CFD0CEC3CECD203120203DF6
:108AF0003D3D0A00CFC4000058582D58582D5858F5
:108B000058582058583A58580A00000025303275F5
:108B10002D253032752D2530327520253032753AAD
:108B2000253032750A000000465072696E742D328D
:108B30003200000025730A00FFF7E9F9FEA0FEF7F6
:108B4000B3FD33F09AFC387899F8001000F010006B
:108B5000084303AA0CD0FB49FBA0FEF7D0FD03A8F5
:108B6000FEF7A2FDB00703AA05D5F649083903E0D0
:108B7000F4490839F0E7F349F8A0FEF7C0FD03A86F
:108B8000FEF792FD700703AA02D5EE49083900E00E
:108B9000EC49F4A0FEF7B3FD03A8FEF785FDF3A0B2
:108BA000FEF782FD0021084630F0D5FD01210020AE
:108BB00030F0D1FD40B90221002030F0CCFD18B1D9
:108BC000E04903AA083901E0DE4903AAEBA0FEF759
:108BD00096FD03A8FEF768FDEBA0FEF765FD0820F3
:108BE00033F0E6FB002029F03DFC08B1012700E04E
:108BF00000270121002030F0AEFD30B1022100201D
:108C000030F0A9FD08B1012600E000263743E9D085
:108C1000032032F043FF0EB1DEA000E0E0A0FEF73B
:108C200043FD012032F03AFF0321002030F093FD94
:108C3000002029F017FC0028FAD1DCA0FEF734FD53
:108C40000021022030F087FD0121022030F083FD59
:108C500040B90221084630F07EFD18B1B94903AA97
:108C6000083901E0B74903AAC4A0FEF748FD03A8EC
:108C7000FEF71AFDC4A0FEF717FD082033F098FB9D
:108C8000002029F0EFFB08B1012700E000270121B7
:108C9000022030F060FD30B10221084630F05BFD6B
:108CA00008B1012600E000263743E9D0032032F066
:108CB000F5FE0EB1B7A000E0B9A0FEF7F5FC01206B
:108CC00032F0ECFE0321022030F045FDA068A168DF
:108CD000091AA942FBD3002029F0C4FB0028FAD1CD
:108CE00003A8FFF7AFFB002103A8FEF78CFE0021CD
:108CF00003A8FEF77CFD002103A8FEF75BFF00211F
:108D000003A8FEF781FF002103A8FFF71DF800214B
:108D100003A8FEF7B7FF002103A8FEF7E0FF00213C
:108D200003A8FFF743F803A8FFF7F5F9002103A80C
:108D3000FFF78AFA464638A91320CDF8E08017F0ED
:108D40002CFC08B1642038909CA129A8389A3AF0EC
:108D50002FF903AA29A99AA0FEF7D1FC03A8FEF7D0
:108D6000A3FC33F0E0FA03A8FFF74FFBAFF2C830E3
:108D7000FEF79AFC012032F091FE94A0FEF794FCDD
:108D8000082033F015FBA768002029F06BFB00B129
:108D9000A768A068C01BA842F6D36A4903AA08398D
:108DA0008CA0FEF7ACFC03A8FEF77EFC8CA0FEF7BF
:108DB0007BFC082033F0FCFAA768002029F052FB66
:108DC00000B9A768A068C01BA842F6D3032032F000
:108DD00065FE5C482430FEF767FC012032F05EFE41
:108DE000002029F03FFB0028FAD180A0FEF75CFCB0
:108DF000082033F0DDFA804F07E000BF29F06BFB5D
:108E0000A068A168091AB942FBD3002029F02AFB07
:108E100000284FF00300F1D029F03FFB022029F099
:108E20002FFB03AA75A146A0FEF769FC03A8FEF775
:108E30003BFC74A0FEF738FC082033F0B9FA4FF47D
:108E4000FA77C82138462BF07AFFA068A168091A82
:108E5000A942FBD3002029F005FB0028F1D003AA8A
:108E600066A137A0FEF74BFC03A8FEF71DFC00200F
:108E700029F0F8FA0028FAD1012032F00FFE64A0A0
:108E8000FEF712FC032032F009FE33F0F6FA664DCD
:108E90002878400702D42B48243001E029482C30A0
:108EA000FEF702FC012032F0F9FD60A0FEF7FCFBAA
:108EB000082033F07DFA604F32F0F5FCA068A1681D
:108EC000091AB942FBD3002029F0CCFA0028F3D0CC
:108ED000022032F0E3FD59A0FEF7E6FB012032F05C
:108EE000DDFD59A0FEF7E0FB082033F061FA33F016
:108EF000C4FA032032F0D2FD2878400702D5114889
:108F0000243001E00F482C30FEF7CEFB03A8FEF71B
:108F1000FCFC33F008FAADF8C46031A9392017F031
:108F20003CFBADF8B8602EA93A2017F036FB054996
:108F3000BDF8B82044318DE0C4C0D2D7C8CAC80A31
:108F400000000000187B000020CDCEC620C0C2D299
:108F5000CECED2D0C5C7D7C8CAC0000020CAD0DB89
:108F6000D8CAC80020C1D3CCC0C3C80052533233C2
:108F7000322D310A200A200A0000000020D0C0C78C
:108F8000CCDBCAC0CDC8C50020C7C0CCDBCAC0CDB1
:108F9000C8C5000020CDCED0CC0A0A0A00000000CF
:108FA00020CDC5CDCED0CC0A0A0A000052533233B0
:108FB000322D320A200A200A000000002575000028
:108FC000DFD0CACED1D2DC20D7CB0000CACDCECFE5
:108FD000CAC00A00D0C0C7CCDBCAC0CDC8C500001B
:108FE000C7C0CCDBCAC0CDC8C50A0A00C8CDC4C83A
:108FF000CAC0D2CED0DB0000400D0300CFD0CEC916
:10900000C4C5CD00C4C8CDC0CCC8CA0A0000000089
:10901000C4C5CDC5C6CDDBC920DFD9C8CA0A20C7A3
:10902000C0CAD0DBD20A0000541F0020D2C5D1D262
:1090300020C7C0CCCAC00A0000350C00CFD0CEC9B2
:10904000C4C5CD0A0000000020CED2CAD0DBD20AAF
:109050000000000029A839F0ABFF03AA29A975A0D8
:10906000FEF74DFB03A8FEF71FFBBDF8C42075A15A
:1090700029A839F09DFF03AA29A975A0FEF73FFB97
:1090800003A8FEF711FB542016F0E7F937A801F00A
:1090900067F837A800F02CFC37A801F057F8012634
:1090A0006E4D7DE0288840F00200288001200DF000
:1090B00097FA012032F0F2FCBDF8B830324668A1D0
:1090C00003A839F075FF03A8FEF7EEFA2FA829F0E0
:1090D00018FF18B930A829F0E3FE28B1AFF2E85123
:1090E00003A83AF0EDF913E0BDF8BC209DF8C100EB
:1090F000A2F5FA629DF8C0100092CDE901109DF82A
:10910000BE309DF8BF20AFF2FC5103A839F050FFEC
:10911000032032F0C3FC03A8FEF7C6FA012032F0A8
:10912000BDFC33F000F903A8FFF76FF9AFF28870C8
:10913000FEF7BAFA39A903A8FEF765FC3AA903A815
:10914000FEF755FB3BA903A8FEF734FD3CA903A895
:10915000FEF75AFD3EA903A8FEF7F6FD3FA903A8B6
:10916000FEF790FD40A903A8FEF7B9FD3DA903A8AD
:10917000FEF71CFE41A903A8FFF766F8A76803E005
:10918000002029F06FF980B9A06843F60952C11B8D
:10919000BDF8C4005043B1EB801FF1D3761CB6B2CA
:1091A000BDF8B80086427FF67DAF552016F055F920
:1091B00037A800F0D5FF37A800F09AFB37A800F0D9
:1091C000C5FF288840F00200288001200DF008FA31
:1091D00028A0FEF769FA032032F060FC2EA0FEF70B
:1091E00063FA288840F00200288001200DF0F8F989
:1091F000FEE710B586B0044605A9012017F002F974
:109200009DF8142027A1684639F0D2FE224669460F
:1092100026A0FEF774FA2046FEF746FA29490020F8
:1092200008602949086078462849086006B000208F
:1092300010BD0000D7C8D1CBCE20D6C8CACBCEC275
:10924000000000002530347520D1C5CA00000000A0
:10925000C7C0C4C5D0C6CAC0000000004A1E002056
:10926000D6C8CACB202530347520C8C72025303455
:10927000750A00003DD2C5D5CDCECBCEC3C8D7C56B
:10928000D1CAC8C920D2C5D1D220C7C0C2C5D0D882
:10929000C5CD3D0A0A0A0A0028CFCEC4CFC8D1DC0A
:1092A000290A0A002530326400000000CDCECCC56A
:1092B000D020CACACC20C220CCC0C3C0C7C8CDC52C
:1092C0000000000004000010080000100C00001056
:1092D00030B40F4C0D4A0323C4F8B031136843F483
:1092E000803313600B4A30BC10470B4910B5362051
:1092F000086014310848FFF7EBFF07481430016895
:1093000009B1002010BD406810BD000088C10F40A9
:1093100000C00F40F11FFF1FF8050010F0B50368F3
:1093200002790D68002462F30704EB18002242EB77
:109330000401FE4DFE4EDFF8FCC30C0A04D1FE4FC3
:10934000E824FF1A8C4108D289202860012030606F
:109350007846CCF800008920F0BD036001712A60D6
:1093600078463260CCF800000020F0BDF0B5002354
:109370000C681A460979057961F30702016865F3FB
:10938000070361185A41E94CE94DEA4E130A04D12A
:10939000E94FE8237F1A934107D2892020600120FA
:1093A0002860784630608920F0BD0160027100209D
:1093B00020602860784630600020F0BDF0B50022C3
:1093C0000C6813460979057961F30703016865F3B1
:1093D0000702D64DD64EDFF85CC30F1B72EB0307B6
:1093E00008D289202860022030607846CCF800003E
:1093F0008920F0BD091B62EB0302016002710020AD
:10940000286030607846CCF800000020F0BDF0B550
:10941000036809680022CB18C44CC54DC54E52EBF9
:10942000020106D1DFF810C3E827BCEB030C8F4123
:1094300007D289202060012028607846306089208A
:10944000F0BD0360226078462A6030600020F0BDE5
:10945000F0B5036809680022CB18B44CB44DB54E82
:1094600052EB020106D1DFF8D4C20227BCEB030C99
:109470008F4107D289202060012028607846306023
:109480008920F0BD0360226078462A6030600020A9
:10949000F0BD30B502680968A44BA54CA54D8A42C1
:1094A00007D2892018600220206078462860892031
:1094B00030BD511A01600020186020607846286095
:1094C000002030BDF0B5036809680022CB18974C26
:1094D000974D984E52EB020106D1DFF860C2022789
:1094E000BCEB030C8F4107D289202060012028604B
:1094F000784630608920F0BD0360226078462A609B
:1095000030600020F0BD30B502680968874B884C98
:10951000884D8A4207D28920186002202060784650
:109520002860892030BD511A016000201860206039
:1095300078462860002030BD10B5028809887C4B31
:1095400011447A4A7B4CB1F5803F07D389201060E3
:109550000120186078462060892010BD018000201D
:109560001060186078462060002010BD0021016066
:1095700001716E4801606E48016078466D4908606F
:10958000002070470021016081808171674801607F
:1095900067480160784667490860002070471CB53D
:1095A0000023CDE90033036800938388ADF80430CD
:1095B00080798DF8060000201060DDE9003409682C
:1095C000CB1A70EB040301D2411E05E0DDE9004334
:1095D000611A834101D20121116054490860544944
:1095E000086078465349086000201CBD2DE9FC4105
:1095F0000022CDE90022026800928288ADF80420A2
:1096000082798DF80620DDE900430A6800211419EB
:1096100041EB0302CDE90042150E444A444B454C50
:1096200008D1DDE90067DFF818C1464DBCEB06063E
:10963000BD4108D289201060012018607846206062
:109640008920BDE8FC81009D0560BDF8045085803F
:109650009DF80650857111607846196020600020E1
:10966000EFE72DE9FC410022CDE9002202680092DB
:109670008288ADF8042082798DF80620DDE9007338
:109680000A680021294C2A4D2A4EBF1A8B4107D265
:109690008920206001202860784630608920D0E74A
:1096A000DDE90073BA1A63EB0103CDE90023026020
:1096B000BDF8042082809DF80620827121607846E2
:1096C000296030600020BCE72DE9FF410022CDE990
:1096D0000222CDE900220A6802928A88ADF80C20A5
:1096E00089798DF80E10016800918188ADF8041019
:1096F00081798DF80610DDE90031DDE902421B19A0
:109700005141CDE900310C0E0849094A094B06D1F7
:10971000DDE900560A4F0B4C7D1BB44118D289205D
:10972000086001201060784618600DE00400001009
:10973000080000100C000010FF0FA5D4FFE30B542D
:10974000FFFF63A7B3B6E00D892004B0BDE8F08148
:10975000009C0460BDF8044084809DF8064084713C
:10976000002008601060784618600020EDE72DE9C1
:10977000FC410022CDE900220B68097961F3070260
:10978000016800918188ADF8041081798DF8061088
:10979000DDE900145B186241CDE90032140E8849FE
:1097A000884A894B06D1DDE90056884F884C7D1BDD
:1097B000B44107D289200860012010607846186003
:1097C00089203EE7009C0460BDF8044084809DF839
:1097D0000640847100200860106078461860002000
:1097E0002FE72DE9F0410546006809680024A1FB38
:1097F000002304FB003001FB04014FF4FA70101841
:1098000041F100014FF47A72234639F035FB6C4A7E
:109810006C4B6D4E31B9DFF8BCC10227BCEB000CBC
:109820008F4107D28920106003201860784630608D
:1098300089208BE72860146078461C603060002027
:1098400084E72DE9F0410546006809880024A1FB62
:10985000002304FB003001FB040141F288301018A2
:1098600041F1000142F21072234639F005FB544ADF
:10987000544B554E31B9DFF85CC10227BCEB000CEC
:109880008F4107D28920106003201860784630602D
:1098900089205BE72860146078461C6030600020F7
:1098A00054E7018842F20F72491C89B2018091424B
:1098B00001D9012101804249002008604149086026
:1098C00078464149086000207047018842F20F72D3
:1098D000491E89B20180914200D902803849002096
:1098E00008603849086078463749086000207047AA
:1098F0000168394A491C0160914201D90121016086
:109900002F49002008602F49086078462E490860DA
:10991000002070470168304A491E0160914200D919
:1099200002602749002008602649086078462649D9
:109930000860002070472DE9F0410446D1E900019C
:10994000D4E90023A0FB025601FB026100FB0311D6
:10995000681949418018594142F21075401941F186
:109960000001521943F1000392185B4139F084FA67
:10997000134B144D144E0A0A04D1184FE8223F1A13
:109980008A4107D289201860032028607846306019
:109990008920DBE6C4E900010020186028607846D1
:1099A00030600020D2E66422B0FBF2F102FB11012C
:1099B000B0FBF2F03229114600D3401C48437047F7
:1099C00004000010080000100C000010FFFF63A747
:1099D000B3B6E00DFFE30B54FFE0F505FF0FA5D490
:1099E0002DE9FF4718F048F96E4C000615D402F037
:1099F00007F9DFF8B481DFF8B4916D4F002668B144
:109A0000012820D087281DD0684601F0A2F8000662
:109A100003D49DF800000E287ED0AEE0684601F029
:109A200098F8000679D403A801F0BAF8000674D4B7
:109A30009DF800000E2805D1BDF80C00402801D18A
:109A40007120387089E0684601F083F8000664D41C
:109A50009DF800001D2827D2DFE800F0260F222203
:109A6000222214141414141414140F1212121212A9
:109A70000F24242424261212120025F087FC03E070
:109A8000202000E06020387002F068F9000674D4ED
:109A90009DF80000474D0E2811D0172812D014E071
:109AA0005020F0E73020EEE7882009212060C8F838
:109AB00000107946C9F8001004B0BDE8F0870CF03A
:109AC0005BFE05E02878022844D001200CF088FDD8
:109AD000000652D49DF80000172806D128780128E6
:109AE00035D125F0C3FC000647D49DF800000E28B0
:109AF00025D12878022826D10AF0DEFCD8B901A8A1
:109B000006F04FFE000638D40DF1060006F02DFEDB
:109B1000000632D4284801E027E02EE000788DF8D6
:109B2000080017208DF8090001A802F01FF80006B0
:109B300023D4322038709DF800000E2803D0C0B224
:109B4000172804D009E02878032803D005E02878F6
:109B5000022802D102F0F7FA2E7026607946C8F882
:109B600000600020C9F80010A6E7FAF75FFB25F0B7
:109B70000DFCFAF770FB02F0F1F820689CE708B5DD
:109B8000684600F095FA58B99DF80000082807D0FB
:109B9000092805D00A2803D008480088002800D0EA
:109BA000012008BD04000010080000100C00001087
:109BB000C01E002040010010C11E00200003001044
:109BC0002DE9F843CD4ECE4FCE4C05464FF08808D8
:109BD000B0F1004F06D0B5F1104F03D00220C4F809
:109BE00000800AE0684601F04BF9000628D49DF891
:109BF000000040B10A20C4F8008030607846386028
:109C00008820BDE8F8830122694628462BF094FAA3
:109C1000000615D49DF80000FF2809D0FF208DF81C
:109C200000000122694628462BF091FA000607D46D
:109C3000280F8DF80000684601F018F9000601D5DC
:109C40002068DEE7B04901200870002048602060ED
:109C50003060784638600020D3E7AB4900200870B8
:109C6000A8490860A54908607846A5490860002011
:109C70007047A54901200870A249002008609F494B
:109C8000086078469E49086000207047F8B568462D
:109C900001F0F6F89B4D000618D49DF80000974E91
:109CA000974FA8B19849002400070C70FF218DF848
:109CB0000010012269462BF04AFA000606D48DF8FE
:109CC0000040684601F0D2F8000609D52868F8BDC2
:109CD000882028600A203060784638608820F8BDE7
:109CE0002C607846346038600020F8BD2DE9F74FCD
:109CF00092B0144610A801F0C3F8824D000649D472
:109D00009DF84000DFF8F481DFF8F4918827B0B1C6
:109D1000060730462BF027FA7B4A401E4FF0000A18
:109D200051680B195B1D98420ED22F60C8F800A035
:109D300079468820C9F8001015B0BDE8F08F0A21D7
:109D40002F60C8F80010F3E746EA01078DF80040DD
:109D50001298ADF8010093466E462246F01C139906
:109D600039F0F1FB3019FF21C4700171221D711C03
:109D7000781C2BF0ECF900060CD40920B0EB177F0F
:109D800001D1621D00E00122694638462BF0DFF95F
:109D9000000601D52868CFE7DBF804102144091D2F
:109DA000CBF80410C5F800A07946C8F800A0002040
:109DB000C9F80010C0E72DE9F04F524D4F4F99B050
:109DC000D5F8009016A8D7F800A001F059F80006C1
:109DD00064D49DF85800DFF82881040700264FF06E
:109DE000010B012201A920462BF0A6F9000655D44B
:109DF0009DF80400F0B3FF284AD00444241D04F069
:109E000070402BF0B0F924F07041401E884211D30D
:109E10009DF8040040280DD8761CE2E7641E01225C
:109E200001A920462BF088F9000637D49DF80400DC
:109E3000402808D9882028607946C7F800B0C8F8BB
:109E4000001019B079E7241AA41E022215A9204691
:109E50002BF072F9000621D4A41C9DF8042002A95D
:109E600020462BF069F9000618D4BDF8540040F0E4
:109E7000005000E00CE09DF8042002A92BF067F9E7
:109E800000060BD49DF8040021180C1AE41E761E5F
:109E9000002EC3D1FFF7FAFE000601D52868D0E7EF
:109EA000C5F800907946C7F800A04846C8F80010E9
:109EB000C7E708B5684600F0E3FF08B1002008BD19
:109EC0009DF800000028FAD00007012269462BF017
:109ED00033F9000605D50B4800680028EFD00120B3
:109EE00008BD9DF8000008B1FF28F8D100208DF8CA
:109EF0000000684600F0BAFFE0E70000080000102C
:109F00000C000010040000105C1E00202DE9F04140
:109F10008046FB4816461D4600780F4680B11A461B
:109F200040462BF009F9F74C000606D42A4639467C
:109F30004046FFF7DBFE000602D52068BDE8F08151
:109F40002A4631464046BDE8F0412BF000B938B50D
:109F500002226946EC482BF0EFF8EA4C000602D5E5
:109F6000208885B201E0BDF8005001F092F9E74980
:109F7000E74A854206D100202060086078461060DC
:109F8000002038BD882020601120086078461060CD
:109F9000882038BD2DE9FF4FDA4CDC4EDC4FDFF86E
:109FA000688381B0994692468B4600254A465146C1
:109FB00001982BF0CCF8000611D401F06AF9ADF845
:109FC00000000222694640462BF0C1F8000606D484
:109FD0004A46594601982BF0AFF8000603D5206891
:109FE00005B0BDE8F08F4A465146584639F03CFA74
:109FF00010B9FFF7ACFF58B16D1CADB2032DD5D32E
:10A000008220206022203060784638608220E7E796
:10A01000002020603060784638600020E0E71CB502
:10A02000C0EBC000B84A401F10430A4607236946E8
:10A03000FFF7B0FF1CBD00B50246B34887B0801CD7
:10A040001C236946FFF7A6FF07B000BDC0EBC000A8
:10A05000AD4A401F104307222BF06EB838B5AD4C07
:10A060000246012369462046FFF750FF38BDA94B41
:10A070000146012218462BF05FB838B5A54C0246C0
:10A08000641C012369462046FFF740FF38BDA14B01
:10A0900001465B1C012218462BF04EB838B59D4C8A
:10A0A0000246A41C012369462046FFF72FFF38BD56
:10A0B000984B01469B1C012218462BF03DB838B541
:10A0C000944C0246E41C012369462046FFF71EFF1C
:10A0D00038BD904B0146DB1C012218462BF02CB8F2
:10A0E00038B58C4C0246241D012369462046FFF7F3
:10A0F0000DFF38BD874B01461B1D012218462BF072
:10A100001BB81CB5C0EBC00026300A4640F000501A
:10A1100007236946FFF7FAFE1CBDC0EBC0002630DE
:10A1200040F0005007222BF007B838B5794C0246B2
:10A130004B34012369462046FFF7E8FE38BD754BD6
:10A1400001464B33012218462AF0F6BF38B5714C50
:10A1500002464C34042369462046FFF7D7FE38BD3B
:10A160006C4B01464C33042218462AF0E5BF38B543
:10A17000684C02465034022369462046FFF7C6FE6B
:10A1800038BD644B01465033022218462AF0D4BF32
:10A1900038B5604C02465234042369462046FFF726
:10A1A000B5FE38BD5B4B01465233042218462AF0F7
:10A1B000C3BF38B5574C0246563402236946204681
:10A1C000FFF7A4FE38BD534B014656330222184612
:10A1D0002AF0B2BF38B54F4C0246583402236946C4
:10A1E0002046FFF793FE38BD4A4B01465833022202
:10A1F00018462AF0A1BF38B5464C02465A3401230E
:10A2000069462046FFF782FE38BD424B01465A336D
:10A21000012218462AF090BF38B53E4C02465B3406
:10A22000042369462046FFF771FE38BD394B0146CD
:10A230005B33042218462AF07FBF832208B502EB65
:10A2400080000A4640F0005004236946FFF75EFE96
:10A2500008BD832202EB800040F0005004222AF067
:10A260006BBF38B52B4C0246873404236946204621
:10A27000FFF74CFE38BD274B0146873304221846B2
:10A280002AF05ABF38B5234C02468B340223694664
:10A290002046FFF73BFE38BD1E4B01468B330222A2
:10A2A00018462AF049BF38B51A4C02468D340423AB
:10A2B00069462046FFF72AFE38BD164B01468D330E
:10A2C000042218462AF038BF38B5124C02469134A1
:10A2D000022369462046FFF719FE38BD0D4B0146A3
:10A2E0009133022218462AF027BF38B5094C02469E
:10A2F0009334012369462046FFF708FE38BD00006D
:10A300005C1E002004000010080000F0080000108F
:10A310000C00001028000020F94B014601221846CD
:10A320002AF00ABF38B5F64C0246641C042369467D
:10A330002046FFF7EBFDE1E7F14B01465B1C0422F1
:10A3400018462AF0F9BE38B5ED4C0246641D0423C8
:10A3500069462046FFF7DAFDD0E7E94B01465B1D71
:10A36000042218462AF0E8BE38B5E54C0246093406
:10A37000042369462046FFF7C9FDBFE7E04B0146CD
:10A380000933042218462AF0D7BE38B5DC4C024601
:10A390000D34012369462046FFF7B8FDAEE7D84BE0
:10A3A00001460D33012218462AF0C6BE38B5D44CFA
:10A3B00002460E34042369462046FFF7A7FD9DE7B9
:10A3C000CF4B01460E33042218462AF0B5BE38B5ED
:10A3D000CB4C02461234022369462046FFF796FD15
:10A3E0008CE7C74B01461233022218462AF0A4BE5E
:10A3F00038B5C34C02461434022369462046FFF7A1
:10A4000085FD7BE7BE4B01461433022218462AF035
:10A4100093BECD2208B502EB80000A4640F0005002
:10A4200004236946FFF772FD08BDCD2202EB8000D0
:10A4300040F0005004222AF07FBE40F20D1208B511
:10A4400002EB80000A4640F0005004236946FFF703
:10A450005DFD08BD40F20D1202EB800040F000509F
:10A4600004222AF069BE38B5A54C0246963404236E
:10A4700069462046FFF74AFD40E7A14B0146963367
:10A48000042218462AF058BE38B59D4C02469A342C
:10A49000042369462046FFF739FD2FE7984B014614
:10A4A0009A33042218462AF047BE38B5944C024627
:10A4B0009E34012369462046FFF728FD1EE7904B96
:10A4C00001469E33012218462AF036BE38B58C4C20
:10A4D00002469F34042369462046FFF717FD0DE727
:10A4E000874B01469F33042218462AF025BE38B513
:10A4F000834C0246A334042369462046FFF706FD39
:10A50000FCE67F4B0146A333042218462AF014BE12
:10A5100038B57B4C0246A734042369462046FFF732
:10A52000F5FCEBE6764B0146A733042218462AF0E9
:10A5300003BE38B5724C0246AB340123694620464F
:10A54000FFF7E4FCDAE66E4B0146AB330122184616
:10A550002AF0F2BD38B56A4C0246AC340223694693
:10A560002046FFF7D3FCC9E6654B0146AC33022217
:10A5700018462AF0E1BD38B5614C0246AE340423DA
:10A5800069462046FFF7C2FCB8E65D4B0146AE3394
:10A59000042218462AF0D0BD38B5594C0246B234D0
:10A5A000012369462046FFF7B1FCA7E6544B01465C
:10A5B000B233012218462AF0BFBD38B5504C0246CE
:10A5C000B334012369462046FFF7A0FC96E64C4BC6
:10A5D0000146B333012218462AF0AEBD38B5484CC7
:10A5E0000246B434022369462046FFF78FFC85E615
:10A5F000434B0146B433022218462AF09DBD38B5BC
:10A600003F4C0246B634042369462046FFF77EFCE1
:10A6100074E63B4B0146B633042218462AF08CBD43
:10A6200038B5374C0246BA34042369462046FFF752
:10A630006DFC63E6324B0146BA33042218462AF019
:10A640007BBD38B52E4C0246BE34042369462046F5
:10A65000FFF75CFC52E62A4B0146BE330422184643
:10A660002AF06ABD38B5264C0246C2340423694636
:10A670002046FFF74BFC41E6214B0146C233042242
:10A6800018462AF059BD38B51D4C0246C634012380
:10A6900069462046FFF73AFC30E6194B0146C633BF
:10A6A000012218462AF048BD1CB500EB800000F2DC
:10A6B0007D100A4640F0005005236946FFF726FC4E
:10A6C0001CBD00EB800000F27D1040F00050052220
:10A6D0002AF032BD4FF4CA7208B502EB40000A46B8
:10A6E00040F0005002236946FFF710FC08BD4FF40C
:10A6F000CA7202EB400040F0005002222AF01CBD5A
:10A70000BB0000204FF4CE7208B502EB40000A46B1
:10A7100040F0005002236946FFF7F8FB08BD4FF4F4
:10A72000CE7202EB400040F0005002222AF004BD3D
:10A730001CB500EB800001EB810100EB810000F211
:10A740008D1040F0005005236946FFF7DFFB1CBD6C
:10A7500000EB800001EB810100EB8100134600F269
:10A760008D1040F00050052219462AF0E5BC090181
:10A7700008B501EB800000F2D22040F00050042325
:10A780006946FFF7C3FB08BD090101EB80001346D2
:10A7900000F2D22040F00050042219462AF0CCBC2E
:10A7A0001CB500EB800001EB810100EB810000F2A1
:10A7B000CD3040F0005005236946FFF7A7FB1CBDD4
:10A7C00000EB800001EB810100EB8100134600F2F9
:10A7D000CD3040F00050052219462AF0ADBC38B506
:10A7E000F84C0246042369462046FFF78FFB85E5B7
:10A7F000F44B0146042218462AF09EBC1CB500EB1F
:10A80000800000F225500A4640F0005005236946BA
:10A81000FFF77CFB1CBD00EB800000F2255040F0F0
:10A82000005005222AF088BC38B5E64C02461834A0
:10A83000042369462046FFF769FB5FE5E14B0146CB
:10A840001833042218462AF077BC1CB500EB8000B0
:10A8500000F23D500A4640F0005005236946FFF7DC
:10A8600055FB1CBD00EB800000F23D5040F0005055
:10A8700005222AF061BC1CB500EB800000F25150AB
:10A880000A4640F0005005236946FFF73FFB1CBD18
:10A8900000EB800000F2515040F0005005222AF0F9
:10A8A0004BBC1CB500EB800000F265500A4640F03E
:10A8B000005005236946FFF729FB1CBD00EB800013
:10A8C00000F2655040F0005005222AF035BC1CB55E
:10A8D00000EB800001EB810100EB810000F265508C
:10A8E00040F0005005236946FFF710FB1CBD00EB4C
:10A8F000800001EB810100EB8100134600F26550FE
:10A9000040F00050052219462AF016BC1CB500EB99
:10A91000800001EB810100EB810000F22D6040F02E
:10A92000005005236946FFF7F1FA1CBD00EB8000DB
:10A9300001EB810100EB8100134600F22D6040F035
:10A940000050052219462AF0F7BB1CB500EB800029
:10A9500001EB810100EB810000F60D0040F000509A
:10A9600005236946FFF7D2FA1CBD00EB800001EB1E
:10A97000810100EB8100134600F60D0040F000500D
:10A98000052219462AF0D8BB1CB500EB800000F662
:10A9900079200A4640F0005005236946FFF7B6FAD1
:10A9A0001CBD00EB800000F6792040F0005005222D
:10A9B0002AF0C2BB40F6862208B502EB40000A46E8
:10A9C00040F0005002236946FFF7A0FA08BD40F6A8
:10A9D000862202EB400040F0005002222AF0ACBB7D
:10A9E0001CB500EB800001EB810100EB410000F69B
:10A9F0007D2040F0005005236946FFF787FA1CBD13
:10AA000000EB800001EB810100EB4100134600F6F2
:10AA10007D2040F00050052219462AF08DBB40F6FB
:10AA2000EE2208B502EB40000A4640F00050022337
:10AA30006946FFF76BFA08BD40F6EE2202EB4000D4
:10AA400040F0005002222AF077BB40F6F62208B50B
:10AA500002EB40000A4640F0005002236946FFF72F
:10AA600055FA08BD40F6F62202EB400040F00050D7
:10AA700002222AF061BB38B5534C024602236946D4
:10AA80002046FFF743FA39E44F4B014602221846AD
:10AA90002AF052BB38B54C4C0246A41C022369462E
:10AAA0002046FFF733FA29E4474B01469B1C02225C
:10AAB00018462AF041BB38B5434C0246241D0123F9
:10AAC00069462046FFF722FA18E43F4B01461B1D5A
:10AAD000012218462AF030BB38B53B4C0246641DB3
:10AAE000022369462046FFF711FA07E4364B014678
:10AAF0005B1D022218462AF01FBB38B5324C0246B5
:10AB0000E41D022369462046FFF700FA13E42E4BAA
:10AB10000146DB1D022218462AF00EBB38B52A4C2E
:10AB200002460934012369462046FFF7EFF913E492
:10AB3000254B01460933012218462AF0FDBA38B5E3
:10AB4000214C02460A34012369462046FFF7DEF90C
:10AB500013E41D4B01460A33012218462AF0ECBAD1
:10AB600040F6093208B502EB40000A4640F00050BA
:10AB700002236946FFF7CAF908BD40F6093202EB25
:10AB8000400040F0005002222AF0D6BA38B50E4CF0
:10AB900002464134022369462046FFF7B7F90EE426
:10ABA000094B01464133022218462AF0C5BA38B58E
:10ABB000054C02464334022369462046FFF7A6F9B6
:10ABC0000EE4000026050020000B0020FB4B014690
:10ABD000022218462AF0B0BA38B5F84C0246A41C36
:10ABE000042369462046FFF791F90AE4F34B014636
:10ABF0009B1C042218462AF09FBA38B5EF4C024637
:10AC0000A41D042369462046FFF780F934E4EB4B8A
:10AC100001469B1D042218462AF08EBA38B5E74C2F
:10AC200002460A34042369462046FFF76FF923E4FD
:10AC3000E24B01460A33042218462AF07DBA1CB5BD
:10AC400000EB800000F64C300A4640F0005005232F
:10AC50006946FFF75BF91CBD00EB800000F64C3045
:10AC600040F0005005222AF067BA38B5D34C0246AE
:10AC70002234042369462046FFF748F90DE4CF4B00
:10AC800001462233042218462AF056BA38B5CB4C76
:10AC900002462634012369462046FFF737F90DE4C2
:10ACA000C64B01462633012218462AF045BA40F623
:10ACB000663208B502EB80000A4640F000500423DB
:10ACC0006946FFF723F908BD40F6663202EB8000C3
:10ACD00040F0005004222AF02FBA1CB500EB80008F
:10ACE00001EB810100EB810000F6653040F000507F
:10ACF00005236946FFF70AF91CBD00EB800001EB54
:10AD0000810100EB8100134600F6653040F00050F1
:10AD1000052219462AF010BA1CB500EB800001EBA1
:10AD2000810100EB810000F6C93040F0005005239E
:10AD30006946FFF7EBF81CBD00EB800001EB8101D9
:10AD400000EB8100134600F6C93040F000500522A8
:10AD500019462AF0F1B940F61E5208B502EB800000
:10AD60000A4640F0005004236946FFF7CFF808BDBB
:10AD700040F61E5202EB800040F0005004222AF000
:10AD8000DBB938B58E4C0246012369462046FFF7F1
:10AD9000BDF80AE48A4B0146012218462AF0CCB9D4
:10ADA00038B5874C0246641C042369462046FFF7E9
:10ADB000ADF80BE4824B01465B1C042218462AF0D6
:10ADC000BBB938B57E4C0246641D04236946204653
:10ADD000FFF79CF80BE47A4B01465B1D04221846F2
:10ADE0002AF0AAB938B5764C0246093404236946DC
:10ADF0002046FFF78BF80BE4714B01460933042220
:10AE000018462AF099B938B56D4C02460D34042322
:10AE100069462046FFF77AF80BE4694B01460D338B
:10AE2000042218462AF088B938B5654C0246113418
:10AE3000022369462046FFF769F80BE4604B0146A0
:10AE40001133022218462AF077B938B55C4C024615
:10AE50001334022369462046FFF758F80BE4584B99
:10AE600001461333022218462AF066B938B5544C0D
:10AE700002461534012369462046FFF747F80BE4E4
:10AE80004F4B01461533012218462AF055B938B503
:10AE90004B4C02461634012369462046FFF736F82C
:10AEA000A5E4474B01461633012218462AF044B95F
:10AEB00038B5434C02461734012369462046FFF754
:10AEC00025F894E43E4B01461733012218462AF038
:10AED00033B9C90008B501EB400000F5576040F0F8
:10AEE000005002236946FFF711F808BDC90001EBC5
:10AEF0004000134600F5576040F00050022219460A
:10AF00002AF01AB940F6F85208B502EB40000A469A
:10AF100040F0005002236946FEF7F8FF08BD40F6F6
:10AF2000F85202EB400040F0005002222AF004B92F
:10AF300040F62E6208B502EB40000A4640F0005091
:10AF400002236946FEF7E2FF08BD40F62E6202EBDF
:10AF5000400040F0005002222AF0EEB81CB500EB91
:10AF6000800001EB810100EB810000F64D6040F0B4
:10AF7000005005236946FEF7C9FF1CBD00EB8000A9
:10AF800001EB810100EB8100134600F64D6040F0BB
:10AF90000050052219462AF0CFB81CB500EB8000FE
:10AFA00001EB810100EB810000F69D6040F0005054
:10AFB00005236946FEF7AAFF1CBD0000430B0020D5
:10AFC000620D002000EB800001EB810100EB8100AD
:10AFD000134600F69D6040F00050052219462AF005
:10AFE000ABB840F6047208B502EB40000A4640F0E8
:10AFF000005002236946FEF789FF08BD40F604723F
:10B0000002EB400040F0005002222AF095B840F6D2
:10B01000067208B502EB80000A4640F00050042397
:10B020006946FEF773FF08BD40F6067202EB80002A
:10B0300040F0005004222AF07FB84FF4716208B546
:10B0400002EB40000A4640F0005002236946FEF73A
:10B050005DFF08BD4FF4716202EB400040F000500C
:10B0600002222AF069B82DE9F8430422694600203B
:10B070002AF09BF9954C00060FD495490098822739
:10B08000944D954E4FF0190888420DD1042269461F
:10B0900010462AF08AF9000602D52068BDE8F88338
:10B0A0008E490098884206D027607846C5F800800F
:10B0B00030608220F2E7002020602860784630600F
:10B0C0000020EBE72DE9F043804EDFF80882DFF83F
:10B0D000089291B000254FF400570024611968468A
:10B0E00000F0EBF82022694620462AF073FA0006A9
:10B0F0000ED42034BC42F1D300246119684600F01C
:10B10000DCF8202208A920462AF04FF9000603D5D2
:10B11000306811B0BDE8F083202208A9684638F0F5
:10B12000A3F940B1822019213060C8F80010794697
:10B13000C9F80010EDE72034BC42DED3ED1DFF2D31
:10B14000CBD9002030607946C8F80000C9F800105B
:10B15000DFE770B58CB000208DF824005C480A90C1
:10B160002422694604202AF020F9584D000617D4FD
:10B17000FFF7A8FF000613D400244FF40056012265
:10B1800009A920462AF026FA000609D4641CB44214
:10B19000F5D32422694604202AF01CFA000602D5C1
:10B1A00028680CB070BD04220AA900202AF012FA07
:10B1B000F7E738B504466946002009F0A2FD01060C
:10B1C000424801D500685EE4BDF8001001B10121DC
:10B1D0002170002101603F48016078463E490860C7
:10B1E000002050E4FF2009F0C6BE10B588B06846C4
:10B1F000C11D06F0BFF8354C00060BD40DF10E0052
:10B20000FEF7C0F9000605D40DF11500FEF7BAF9F6
:10B21000000602D5206808B010BD6846FEF70BFF97
:10B22000F9E738B5FEF793FE284C48B36846FFF7B8
:10B23000C0FF00061FD49DF80000F0B1702014F08C
:10B240000CF9000617D4712014F007F9000612D487
:10B250006F2014F002F900060DD4FFF7C6FF0006B8
:10B2600009D4722014F0F9F8000604D46F2014F009
:10B27000F4F8000604D5206805E4FFF7B6FFF8E708
:10B2800014490020206008607846134908600020B7
:10B2900009E400B589B01E226946114829F04CFF27
:10B2A000000604D50948008880B209B000BD1C2101
:10B2B0000DF10200F8F7EAFFF7E7002200F8011BA2
:10B2C000491C521C202AF9D37047000004000010CA
:10B2D000CC2C5140080000100C000010CEFAADDE5E
:10B2E000100000F07FB5054603A8FEF7E1FE264CEE
:10B2F000000640D49DF80C00012832D00026022818
:10B3000009D08720206021480660784620490860DF
:10B31000872004B070BD002005F07AFA00062AD418
:10B320002888ADF804006888ADF8060028798DF803
:10B3300008008DF8096001A804F09EF900061AD4EF
:10B3400069462B2015F05EF8000614D411489DF8CC
:10B3500000100078C90704D0012802D001208DF820
:10B360000C0003A8FEF7ABFE000604D4284601F04B
:10B3700023FD000601D52068CBE703208DF80C00E3
:10B3800003A8FEF78BFEC4E70400001008000010BD
:10B390000C000010E81E002038B505466846FEF790
:10B3A00087FE0D4C000611D49DF80000032809D03B
:10B3B00087200A4920600020086078460849086014
:10B3C000872038BD05F0FCF9000601D5206838BD9E
:10B3D000284601F039FE38BD0400001008000010B6
:10B3E0000C00001038B504466846FEF761FE010601
:10B3F0000A4801D5006838BD9DF80010032909D01E
:10B4000087210160064900200860784605490860E8
:10B41000872038BD204601F009FF38BD0400001028
:10B42000080000100C00001038B504466846FEF70E
:10B430003FFE01060A4801D5006838BD9DF800109E
:10B44000032909D087210160064900200860784659
:10B4500005490860872038BD204601F0DDFF38BD72
:10B4600004000010080000100C00001038B504465D
:10B470006846FEF71DFE01060A4801D5006838BD82
:10B480009DF80010032909D087210160064900209A
:10B490000860784605490860872038BD204602F0DC
:10B4A0006FF838BD04000010080000100C000010F8
:10B4B00038B504466846FEF7FBFD01060A4801D58B
:10B4C000006838BD9DF80010032909D0872101606C
:10B4D000064900200860784605490860872038BD85
:10B4E000204602F02BF938BD0400001008000010BF
:10B4F0000C00001038B504466846FEF7D9FD010679
:10B500000A4801D5006838BD9DF80010032909D00C
:10B5100087210160064900200860784605490860D7
:10B52000872038BD204602F0BDF938BD0400001068
:10B53000080000100C00001038B504466846FEF7FD
:10B54000B7FD01060A4801D5006838BD9DF8001016
:10B55000032909D087210160064900200860784648
:10B5600005490860872038BD204602F077FA38BDCB
:10B5700004000010080000100C00001038B504464C
:10B580006846FEF795FD01060A4801D5006838BDFA
:10B590009DF80010032909D0872101600649002089
:10B5A0000860784605490860872038BD204602F0CB
:10B5B000E9FA38BD04000010080000100C0000106B
:10B5C00038B504466846FEF773FD01060A4801D502
:10B5D000006838BD9DF80010032909D0872101605B
:10B5E000064900200860784605490860872038BD74
:10B5F000204602F07FFB38BD040000100800001058
:10B600000C00001038B504466846FEF751FD0106EF
:10B610000A4801D5006838BD9DF80010032909D0FB
:10B6200087210160064900200860784605490860C6
:10B63000872038BD204602F0F1FB38BD0400001021
:10B64000080000100C00001038B56846FEF730FD09
:10B650000E4C000611D49DF80000032809D0872065
:10B660000B4920600020086078460A49086087205E
:10B6700038BD02F08BFC000601D5206838BD0420DF
:10B680008DF800006846FEF709FD38BD0400001083
:10B69000080000100C0000102DE9FE43294C002684
:10B6A0002068822800D001266846FEF701FD0006CA
:10B6B0003AD49DF800001D280DD101A800F04AF8E9
:10B6C000000631D42048018821F00201018000F0F9
:10B6D000A5FE000628D49DF8000000251B4FDFF8CA
:10B6E000708003280DD004280BD00E2809D01B2809
:10B6F00007D08720206079463D60C8F80010BDE87B
:10B70000FE83002002F084FC00060DD49DF80000AA
:10B710001B280BD06846FEF7DCFC000604D4684604
:10B72000FEF7BCFC000601D52068E8E716B1012051
:10B730000AF056FF256079463D600020C8F80010E9
:10B74000DDE70000040000104A1E00200800001081
:10B750000C0000102DE9F0479AB0824617A8FEF7BA
:10B76000A7FC504C000654D49DF85C10002505261B
:10B770004D4FDFF838810DF14C0904290AD01D29FD
:10B7800048D08720206079463D60C8F800101AB084
:10B79000BDE8F08718A9504602F085FD20B1922837
:10B7A0002AD0932875D123E09DF86000002873D03B
:10B7B0003F48007800286FD01D208DF85C0017A846
:10B7C000FEF76CFC000664D44846FEF744FF000612
:10B7D0005FD416A8FEF750FF00065AD40AF0E9FB22
:10B7E00060B3256079463D600020C8F80010CEE7C0
:10B7F000F8F71CFD0E2005E03868312849D1F8F72C
:10B8000015FD16208DF85C0017A8FEF747FCF8F729
:10B8100022FD3EE011A807F0CDFB000639D416A9A1
:10B82000139807F0CBFE000633D44846FEF709FF15
:10B8300000062ED416A8FEF715FFCDE70C208DF8D4
:10B8400001001398CDF802001698CDF8060068465E
:10B8500008F073FE00061CD4684609F0EFFF0006EE
:10B8600017D4FEF726FB18B1FEF7F7F9000610D43F
:10B87000684608F08DFE00060BD468460AF009F809
:10B88000000606D4FEF715FB28B1FEF7F2F9000614
:10B8900002D520687BE7FFE78DF85C6017A8FEF70C
:10B8A000FDFB74E704000010080000100C000010FD
:10B8B0000844000070B586B005460E4603A8FEF7A2
:10B8C000F7FB2D4C00064ED49DF80C001D280DD121
:10B8D00004A8FFF73FFF000645D42848018821F05F
:10B8E0000201018000F09AFD00063CD49DF80C1086
:10B8F00001292DD00020022909D08721216020496B
:10B90000086078461F490860872006B070BD298806
:10B91000ADF804106988ADF8061029798DF8081083
:10B920008DF8090001A803F0A7FE00061BD46946A4
:10B930002B2014F067FD000615D413489DF8001065
:10B940000078C90704D0012802D001208DF80C002E
:10B9500003A8FEF7B4FB000605D43146284603F0E1
:10B9600023F9000601D52068CFE706208DF80C00EA
:10B9700003A8FEF793FBC8E7040000104A1E00204E
:10B98000080000100C000010E81E002038B56846C2
:10B99000FEF78EFB0F4C000616D49DF8000006281B
:10B9A00009D087200C4920600020086078460B49A8
:10B9B0000860872038BD03F079F9000604D4684692
:10B9C000FEF787FB000601D5206838BD6846FEF704
:10B9D00065FB38BD04000010080000100C000010CA
:10B9E00038B505466846FEF763FB0F4C000612D4D7
:10B9F0009DF80000062809D087200C49206000200F
:10BA0000086078460A490860872038BD284603F058
:10BA100085F9000601D5206838BD07208DF80000A3
:10BA20006846FEF73BFB38BD04000010080000101C
:10BA30000C00001038B504466846FEF739FB0106D5
:10BA40000B4801D5006838BD9DF8001004290BD0C3
:10BA5000062909D087210160064900200860784640
:10BA600005490860872038BD204603F099FA38BDA3
:10BA700004000010080000100C00001038B5044647
:10BA80006846FEF715FB01060B4801D5006838BD76
:10BA90009DF8001004290BD0062909D087210160E8
:10BAA000064900200860784605490860872038BDAF
:10BAB000204603F037FB38BD0400001008000010DA
:10BAC0000C00001038B504466846FEF7F1FA01068E
:10BAD0000B4801D5006838BD9DF8001004290BD033
:10BAE000062909D0872101600649002008607846B0
:10BAF00005490860872038BD204603F0C5FB38BDE6
:10BB000004000010080000100C00001038B50546B5
:10BB10006846FEF7CDFA124C000617D49DF80000D7
:10BB2000022809D087200F4920600020086078464D
:10BB30000D490860872038BD002004F069FE00062A
:10BB400004D4284603F098FD000601D5206838BDCE
:10BB500001208DF800006846FEF7A0FA38BD00000D
:10BB600004000010080000100C00001038B5054655
:10BB70006846FEF79DFA1F4C000632D49DF800007F
:10BB800010281FD00CDC0C281CD004DC012819D094
:10BB900002280DD116E00D2814D00E2808D111E08E
:10BBA00013280FD014280DD015280BD0182809D031
:10BBB0008720114920600020086078460F490860FE
:10BBC000872038BD6846FEF77AFA000609D4684631
:10BBD000FEF786FA000604D4284605F02BFC000682
:10BBE00001D5206838BD08208DF800006846FEF7B2
:10BBF00055FA38BD04000010080000100C000010B9
:10BC00002DE9F04186B002A8FEF752FA504C00062A
:10BC10007ED49DF8080001274E4E0025082807D045
:10BC2000092805D00A2874D0872006B0BDE8F08125
:10BC300005F0AAFC009031684FF00A080191042831
:10BC400021D005DC48B1012809D0032829D118E00A
:10BC5000052802D0822824D11FE0009560E06846C4
:10BC6000FEF7BAFF000670D401A8FEF7C6FF000673
:10BC70006BD48DF8088002A8FEF710FA000664D491
:10BC80004EE0082000E009208DF8080002A8FEF729
:10BC900005FA00903068019042E003290DD0042994
:10BCA0000BD00AF053F803A8FEF753FF00064CD45C
:10BCB0009DF80C000E2803D011E006F0F1FF2FE0F4
:10BCC00004A9622014F09EFB00063ED49DF81000EB
:10BCD000C00704D00120F9F7F5F9000635D4009823
:10BCE000822801D0922801D106F0DAFF6846FEF7DB
:10BCF00073FF000629D401A8FEF77FFF000624D4B5
:10BD00009DF8080009280BD08DF8088002A801E0F2
:10BD10001BE00DE0FEF7C2F915E000BFCDE90075AC
:10BD2000009820600199316079460B4A11607CE7E8
:10BD30008120CDE900056846FEF74EFF000604D4D9
:10BD400001A8FEF75AFF0006E8D520686DE700005D
:10BD500004000010080000100C0000102DE9F04154
:10BD600086B003A8FEF7F5FE364C000660D402A8A4
:10BD7000FEF79EF900065BD401A8FEF737FF000628
:10BD800056D404A8FEF743FF000651D49DF80800DE
:10BD900087272D4D2D4E4FF000080A2801D0092885
:10BDA00035D106F08FFB000642D401980128684681
:10BDB00008D0FEF78EF900063AD49DF8080009284D
:10BDC00005D013E0FEF796F9000631D414E001988F
:10BDD000922801D0822802D113208DF800009DF80E
:10BDE0000C00142802D10C208DF800000198932833
:10BDF00002D10E208DF800006846FEF74FF90006CC
:10BE000016D49DF80800092814D00A2808D0276005
:10BE10007846C5F800803060872006B0BDE8F08124
:10BE20009DF80C000E2805D1FAF71CFC000601D580
:10BE30002068F2E701982060049929607946316012
:10BE4000EBE7000004000010080000100C000010D8
:10BE500038B505466846FEF72BF9164C00061FD488
:10BE60009DF800000C2809D087201349206000208D
:10BE70000860784611490860872038BD6846FEF79B
:10BE80001EF900060CD40D208DF800006846FEF760
:10BE900027F9000604D4284603F0B4FC000601D5B7
:10BEA000206838BD08208DF800006846FEF7F6F8D7
:10BEB00038BD000004000010080000100C00001045
:10BEC000F0B585B001A808F054FF344C000655D4F5
:10BED0006846FEF7EDF8000650D49DF800000225F4
:10BEE0002F4E304F13281ED00CDC0D281BD004DC45
:10BEF000012818D002280DD115E00E2813D01028E3
:10BF000008D143E014280ED015280CD018280AD0E8
:10BF10001B283BD0872020600020306078463860A6
:10BF2000872005B0F0BD012004F072FC000625D486
:10BF300004A804F001F9000622D59DF81000E8B12C
:10BF4000012809D0022810D0882020600920306004
:10BF5000784638608820E4E7F8F768F918208DF80B
:10BF6000000006E0F8F777F908E0F8F75FF98DF8D8
:10BF700000506846FEF792F80006F3D52068D0E737
:10BF80008DF800506846FEF789F8CAE792202060D5
:10BF90007846356038609220C3E700000400001046
:10BFA000080000100C0000102DE9F04385B0814618
:10BFB00002A808F0DEFE2C4C000645D40620F9F756
:10BFC00056FC2A4D2A4E38B90420F9F750FC18B90E
:10BFD0000120F9F74CFC80B16846FEF769F80006CD
:10BFE00032D49DF8000000274FF0870802280ED0B9
:10BFF0000D2817D0182829D114E091202060B120F5
:10C00000286078463060912005B0BDE8F08301A833
:10C01000FFF7CFF8000617D416499DF804000978F9
:10C02000084213D101A9484603F024FEA8B19DF8A7
:10C03000040048B1F8F7FAF818208DF800006846B7
:10C04000FEF72CF8F8F707F92068DDE7C4F8008060
:10C0500078462F6030608720D6E702208DF80000F8
:10C060006846FEF71BF8CFE7040000100800001038
:10C070000C00001008440000F8B506466846FEF7BC
:10C0800017F8504C000650D49DF800004E4D132870
:10C0900012D004DC01280FD00E2804D10CE01528A2
:10C0A0000AD01B2808D0872020600020286078460E
:10C0B000464908608720F8BDF9F7ADFE93281ED0E9
:10C0C0006846FDF7FCFF00062FD49DF800001B28F2
:10C0D00019D002208DF800006846FEF701F800062E
:10C0E00023D4012004F094FB00061ED4304606F051
:10C0F00047FA50B18F280FD0922816D117E0F8F7E1
:10C1000095F80E2019E01020E4E708208DF80000D3
:10C110006846FDF7C3FFF8BDF8F788F828680728D8
:10C1200001D1142009E0F8F796F82068F8BDF8F777
:10C130007DF828683128F6D116208DF80000684671
:10C14000FDF7ACFFEFE72DE9FC4101A8F8F733FF5D
:10C150001C4C00060BD4BDF804001B4E1B4F0025E1
:10C1600040B16946622014F04DF9000609D52068F7
:10C17000BDE8FC81812020607846356038608120F0
:10C18000F6E79DF80000800703D5002110A02FF0EE
:10C19000FEFEF8F715FF30B1F8F748F809F0D6FDC4
:10C1A000F8F759F8E3E70F48018841F002010180F0
:10C1B00001200AF015FA25607846356038600020C5
:10C1C000D6E7000004000010080000100C0000106A
:10C1D0008493818B888A809220848E8A938C858D2B
:10C1E00092800A004A1E0020F8B506460D466846B1
:10C1F000FDF75EFF1C4C00062DD49DF80020132A8D
:10C2000019D008DC012A16D0022A14D00E2A12D026
:10C21000102A06D10FE0142A0DD0152A0BD0182AA7
:10C2200009D0872011492060002008607846104915
:10C2300008608720F8BD6846FDF741FF00060AD474
:10C240006846FDF74DFF000605D42946304606F046
:10C2500061FB000601D52068F8BD08208DF80000BC
:10C260006846FDF71BFFF8BD040000100800001031
:10C270000C000010F8B506460D466846FDF718FF9D
:10C280001D4C000627D49DF800101C4A1C4810299C
:10C2900011D004DC02290ED00D2904D10BE01129A4
:10C2A00022D0142907D0872121600021116079460E
:10C2B00001608720F8BD6846FDF701FF00060AD43B
:10C2C0006846FDF70DFF000605D42946304606F006
:10C2D000DDFB000601D52068F8BD08208DF80000C0
:10C2E0006846FDF7DBFEF8BD91212160A9211160B0
:10C2F000794601609120F8BD04000010080000108C
:10C300000C0000103EB501A8FDF7C1FE214C00064F
:10C310003ED46846FDF7CCFE000639D402A90120C0
:10C3200026F07CF8000633D49DF800001A4D022850
:10C3300006D00E2804D0102802D00298C00705D0DD
:10C3400004F08CF880B1922822D114E09DF80420EA
:10C350008721124821600AB1042100E000212960F0
:10C360007946016087203EBD10208DF800006846A8
:10C37000FDF794FE3EBD2868312809D1F7F756FF36
:10C3800016208DF800006846FDF788FEF7F763FF7A
:10C3900020683EBD04000010080000100C000010D2
:10C3A00038B505466846FDF783FE184C00061DD4D7
:10C3B0009DF80000112809D0872015492060002031
:10C3C0000860784613490860872038BD12482968FC
:10C3D000016069684160A9688160342013F03DF80C
:10C3E000000603D42FF09FFF000601D5206838BD5A
:10C3F000284608F0F9FF10B109F0A8FCF6E7022082
:10C400008DF800006846FDF749FE38BD04000010B5
:10C41000080000100C000010B60700102DE9FC41C8
:10C420006846FDF745FE194C000622D49DF8000031
:10C430000025174E174F052809D01D2820D087202A
:10C4400020607846356038608720BDE8FC8101A90E
:10C450000120FDF7FEFE00060BD404F0CDF8000627
:10C4600007D401208DF800006846FDF717FE00068E
:10C4700001D52068E9E7019800B1012009F026FD07
:10C4800025607846356038600020DEE70400001043
:10C49000080000100C00001038B56846FDF708FED3
:10C4A0000E4C000611D49DF80000072809D0872003
:10C4B0000B4920600020086078460A490860872000
:10C4C00038BD04F0C1F8000601D5206838BD012050
:10C4D0008DF800006846FDF7E1FD38BD040000104E
:10C4E000080000100C00001038B504466846FDF73F
:10C4F000DFFD01060A4801D5006838BD9DF800102F
:10C50000032909D087210160064900200860784688
:10C5100005490860872038BD204604F01BFA38BD65
:10C5200004000010080000100C00001038B504468C
:10C530006846FDF7BDFD01060A4801D5006838BD13
:10C540009DF80010032909D08721016006490020C9
:10C550000860784605490860872038BD204604F009
:10C5600071FA38BD04000010080000100C00001023
:10C5700038B504466846FDF79BFD01060A4801D51B
:10C58000006838BD9DF80010032909D0872101609B
:10C59000064900200860784605490860872038BDB4
:10C5A000204604F0C7FA38BD04000010080000104F
:10C5B0000C00001038B504466846FDF779FD010609
:10C5C000204801D5006838BD9DF8001001290BD026
:10C5D000022909D0872101601B49002008607846A4
:10C5E0001A490860872038BD204604F021FC38BD78
:10C5F00038B504466846FDF75BFD0106114801D5D4
:10C60000006838BD9DF8001001290FD0032910D013
:10C6100004290ED005290CD0872101600A49002089
:10C620000860784609490860872038BD0121204606
:10C6300005E009F0E5FB2FF076FE0021084604F046
:10C6400071FC38BD04000010080000100C00001040
:10C650002DE9F84380466946012025F0DFFE104CA5
:10C6600000060DD400980F4E0F4FC0074FF0000585
:10C6700009D000220121404604F0E0FC000609D563
:10C680002068BDE8F88387202060784635603860F0
:10C690008720F6E725607846356038600020F0E7AF
:10C6A00004000010080000100C00001038B504460B
:10C6B0004FF00040FDF784FA000602D516480068E6
:10C6C00038BD2046FDF775FD00061FD4A01CFDF700
:10C6D00081FD00061AD4201DFDF78DFD000615D43E
:10C6E0000AF03AF8000602D509F030FB0EE0684681
:10C6F000FDF736FD000609D46846FDF7F9F8000697
:10C7000004D46846FDF722FD000602D5FDF753FB71
:10C7100038BDFDF7BBFA38BD040000102DE9F0412B
:10C7200088B001A8FDF7B3FC384C00065ED49DF834
:10C730000400374F374E48B1912020609C20306074
:10C7400078463860912008B0BDE8F08106A9012044
:10C7500025F064FE000649D406984FF00005C00796
:10C7600046D06846FDF7A4FC00063FD46846FDF7B6
:10C77000A6FC00063AD46846FDF7B2FC000635D4A4
:10C7800008208DF800006846FDF788FC00062DD4CF
:10C790004FF001088DF8088002A8FEF7D0F90006D6
:10C7A00024D403208DF80C0003A8FDF7BEFC00067E
:10C7B0001CD419490220087014482560FEF70CFAB1
:10C7C000000613D413483560FEF717FA00060DD49F
:10C7D000ADF8108004A8FEF7D9F9000606D4ADF82C
:10C7E000145005A8FEF7E3F9000608D52068AAE76B
:10C7F000872020607846356038608720A3E7256071
:10C8000078463560386000209DE700000400001085
:10C810000C00001008000010481E00202DE9FF4702
:10C820000646684603F0BDFFA24C000665D4BDF87D
:10C8300000004FF4B46148433178C1EB011100EBC3
:10C8400081007178451802A8FEF7B3FC000654D4A5
:10C8500003A8FAF70FF800064FD49DF80C00E8B3D0
:10C8600095499DF80800DFF854920978DFF850A246
:10C8700008424FF086074FF0170817D0694602208C
:10C8800006F042FC000638D401A9032006F03CFC67
:10C89000000632D4BDF80000BDF80410C0EB001053
:10C8A00000EB400001EB4010854215D36846FEF7CF
:10C8B000EBF8000621D401A8FEF7F6F800061CD418
:10C8C000BDF80000BDF80410C0EB001000EB400004
:10C8D00001EB401085420BD2276000E008E079466A
:10C8E000C9F800808620CAF8001004B0BDE8F087BF
:10C8F000304626F03AFB000601D52068F5E703F044
:10C90000FFFFF2E72DE9FF4781466946532013F008
:10C9100079FD684C000629D49DF8000000F0040061
:10C920008DF8000001A8FDF7C3FB00061ED49DF89A
:10C930000400624D624E0027DFF88881102817D06E
:10C9400009DC022814D00D2819D091210E287DD0A1
:10C950000F2806D19AE011280AD0192815D01A28D4
:10C9600013D003A8F9F786FF000670D52068BCE74E
:10C970004846FFF753FF05E088F800700FE048468F
:10C9800026F0F3FA0006F1D4F6E74846FFF746FF33
:10C990000028EBD198F80000C246022805D0276095
:10C9A00078462F60306000209FE79DF8000020B19E
:10C9B0004D2012F052FD0006D8D4484626F070FAF9
:10C9C0000006D3D4404999F8028088683F4A8B68B2
:10C9D0001B1A9342FBD3484626F062FA0006C5D4E0
:10C9E00099F80210414507D1822020600520286077
:10C9F00078463060822078E703218AF800103449B5
:10CA00004FF0010801A881F80080FDF773FB0006D4
:10CA1000ACD401A8FDF742FB0006A7D40420F8F728
:10CA2000B7FF0006A2D49DF8000020B1012009F054
:10CA3000D7FD00069AD402A9532013F0E3FC0006A8
:10CA400094D49DF8080010F0010001E01BE024E000
:10CA50008DF8080008D0012009F0C2FD000685D439
:10CA600009F0CAF8000681D49DF8080020B1012021
:10CA700009F0B6FD000686D4C4F8008078462F6021
:10CA80003060012031E7A020216001E0D220216048
:10CA9000286078463060912027E79DF80C108720A9
:10CAA000206011B10420286000E02F6078463060DB
:10CAB00087201AE704000010084400000800001056
:10CAC0000C0000104201001000000940E0C81000F6
:10CAD000641E00202DE9FE43054601A8FEF769FB10
:10CAE000AB4C00062BD49DF80400AA4EAA4F4FF081
:10CAF00086084FF01A09A8B1A848007848B16946DD
:10CB0000022006F001FB000619D4BDF800008542A2
:10CB10001CD36846F9F792F8000610D4BDF800005F
:10CB2000854213D302A8F9F7A5FE000607D49DF8A5
:10CB3000080098B16846FDF7A7FF000602D52068F7
:10CB4000BDE8FE83BDF80000854207D2C4F800802E
:10CB50007846C6F8009038608620F1E70020206013
:10CB60003060784638600020EAE72DE9F14F88B060
:10CB700000278DF8047003A90898F7F7B9FFBDF8EE
:10CB80000C0048F26901834D834E814C401E4FF0EA
:10CB900086094FF0140A884205D300BFC4F80090FC
:10CBA000C5F800A05EE001A9532013F02BFC00069D
:10CBB0007ED49DF8040000F004008DF8040068465F
:10CBC000FDF776FA0006F3D49DF80000102820D077
:10CBD00009DC02281DD00D281BD091210E2868D019
:10CBE0000F2808D198E0112813D0192811D01A283D
:10CBF0000FD01C280DD006A8F9F73CFE000657D42C
:10CC00009DF818108720002920607CD0042028601F
:10CC10008AE0BDF80C00FFF75DFFDFF8848138B3D0
:10CC2000862845D188F800709DF800001C2810D097
:10CC30001A283DD019283BD06846FDF740FA000677
:10CC400036D41C208DF800006846FDF727FA000650
:10CC50002ED40220F8F789FE000629D41A20C4F841
:10CC60000090286078463060862009B0BDE8F08FDB
:10CC700002A826F046F900064FF0010B07D54FF445
:10CC8000FA60ADF808008DF80AB08DF80BB005A970
:10CC900002A8F7F72DFFBDF80C10BDF8140098F8A6
:10CCA00000208142404610D9012A08D0418001E08D
:10CCB0005EE02EE088F800B0C4F800B062E0428880
:10CCC0008A4204D088F8007068E7012AF7D00898F3
:10CCD00026F06CF900064BD44FF0020988F800905A
:10CCE0009DF8040048B13A2012F0B7FB00063FD48B
:10CCF000012009F075FC00063AD40220F8F748FE3E
:10CD0000000635D400E00EE09DF800001C280FD08E
:10CD100018E0A020216001E0D22021602860784640
:10CD200030609120A1E72F607846306087209CE733
:10CD30006846FDF7CEF900061AD46846FDF7AEF94D
:10CD4000000615D403F0DCFD9DF80000192807D07B
:10CD50001A2805D0276078462F603060002084E7CD
:10CD60009DF8040050B13E2012F077FB000601D57B
:10CD700020687AE700210BA02FF009F988F80090CD
:10CD8000C4F800B078462F60306001206DE70000E5
:10CD900004000010080000100C00001008440000FF
:10CDA00042010010200A200A200A200A200A200A34
:10CDB000200A200A00000000F0B5054641799E4C8B
:10CDC0009E4F9F4E91B0862009B1042902D9206060
:10CDD000062005E0297909B11E2907D92060052020
:10CDE000386078463060862011B0F0BD69882888A8
:10CDF00003F06EFC00067DD468796946FDF78FFC70
:10CE0000000677D4BDF800100020A1F57F42FF3A5C
:10CE100071D0064600906846FDF7C8FA000669D44E
:10CE20006846FDF7FBFE000664D4012769463846D4
:10CE3000FDF7EFFA00065DD47F1CFFB2112FF5D38A
:10CE40006846FDF710FB00067ED46846FDF71CFB24
:10CE5000000679D4012769463846FDF7EEF9000649
:10CE600072D47F1CFFB20B2FF5D3012769463846D9
:10CE7000FDF771FF000667D47F1CFFB2112FF5D3B9
:10CE80006846FDF7ACFC00065ED46846FDF7CCFCB6
:10CE9000000659D46846FDF7E4F9000654D4684604
:10CEA000FDF701FA00064FD46846FDF7B5F9000614
:10CEB0004AD40127009669463846FDF7F8FE000679
:10CEC00042D47F1CFFB2052FF5D9ADF8006068464B
:10CED000FDF77DFA000637D46846FDF789FA0006AB
:10CEE00032D46846FDF7CEF900062DD46846FDF72A
:10CEF000EBF901E028E029E0000625D400960126A0
:10CF000069463046FDF799FA00061DD4761CF6B244
:10CF1000112EF5D32846FDF74CF9000614D4A81CB1
:10CF2000FDF758F900060FD4281DFDF764F9000637
:10CF30000AD4012009F054FB000605D44FF000404C
:10CF4000FCF73EFE000608D520684DE78B212160E6
:10CF5000386078463060084646E701248DF8004086
:10CF60006846FDF7E2F8000633D436480470681DC1
:10CF7000FDF70BFA00062CD46846FDF7F1F8000621
:10CF800027D46846FCF7B4FC000622D46846FDF7B7
:10CF9000DDF800061DD46846FDF7F3F8000618D446
:10CFA0006846FCF77EFC000613D46846FDF7DFF800
:10CFB00000060ED46846FDF7F5F8000609D4684669
:10CFC000FCF796FC000604D46846FDF7E1F800067D
:10CFD00002D5FCF7F0FE07E708F058FF000624D45E
:10CFE0008DF8014068798DF8020008F071FB0006A9
:10CFF0001BD4684607F0A1FA000616D4684608F06C
:10D000001DFC000611D4FCF728FE00060DD468466E
:10D0100007F0BEFA000608D4684608F03AFC00069D
:10D0200003D4FCF726FE000602D508F08FFED0E7F9
:10D03000FCF72CFED8E600000400001008000010E9
:10D040000C000010481E002070B5057A724E98B092
:10D050000446102D0AD986207049306003200860EC
:10D0600078466F490860862018B070BD0DB901255B
:10D07000257260681290214612A8FCF7B2FB0006E8
:10D0800005D44FF00040FCF79BFD000601D5306849
:10D09000EAE711A8FDF794F9000652D412A911A8E5
:10D0A000FCF7D6F900064CD411A8FDF77FF900066D
:10D0B00047D411A8FDF795F9000642D4BDF8440005
:10D0C000401CADF8440011A8FDF781F9000638D4E2
:10D0D00011A92846FDF7A9F9000632D412A911A812
:10D0E000FCF7B6F900062CD411A92846FDF791F9F2
:10D0F000000626D411A92846FDF7ACF9000620D475
:10D10000214611A8FCF7DEF900061AD411A9284619
:10D11000FDF793F9000614D404F10800FDF7C5F9F2
:10D1200000060ED42046FDF7D1F9000609D4201DD3
:10D13000FDF7DDF9000604D412A8FDF7E9F90006B1
:10D1400002D5FCF738FE8FE701202EF0A7FC000681
:10D1500058D409F07FF9000654D40D208DF8010051
:10D16000207A8DF80F006068CDF803002068CDF8B4
:10D1700007001298CDF80B002A4904A836F0A0F950
:10D180000DF10200FDF70BF900063BD4684607F0ED
:10D19000D4F9000636D4684608F050FB000631D4B6
:10D1A000012007F0E8FE00062CD411A8FEF701F8D4
:10D1B000000627D49DF8440090B11B48007878B150
:10D1C00014A8FDF7ECF800061CD48DF85C5020681C
:10D1D00015901298169014A806F00BFC000611D4B6
:10D1E000FCF73BFD00060DD4684607F0D1F90006B8
:10D1F00008D4684608F04DFB000603D4FCF739FD5F
:10D20000000602D508F0A2FD9BE706490020087041
:10D21000FCF73CFD28E700000400001008000010A7
:10D220000C000010040800100844000070B5057AD6
:10D23000744E98B00446102D0AD986207249306089
:10D2400003200860784671490860862018B070BDD8
:10D2500005B9012560681290214612A8FCF7C1FAB1
:10D26000000605D44FF00040FCF7AAFC000601D5EB
:10D270003068EBE76846FDF7A3F8000662D412A910
:10D280006846FCF706F900065CD46846FDF78EF8A0
:10D29000000657D46846FDF7B5F8000652D4BDF82D
:10D2A0000000401CADF800006846FDF7A1F800063C
:10D2B00048D46846FDF7BCFC000643D412A9684672
:10D2C000FCF7C6F800063DD46846FDF7A7FC00064B
:10D2D00038D469462846FDF7A8F8000632D412A9CA
:10D2E0006846FCF7D6F800062CD469462846FDF7B8
:10D2F00090F8000626D469462846FDF7ABF80006EC
:10D3000020D421466846FCF7FEF800061AD4694688
:10D310002846FDF792F8000614D404F10800FDF742
:10D32000C4F800060ED42046FDF7D0F8000609D454
:10D33000201DFDF7DCF8000604D412A8FDF7E8F87C
:10D34000000602D5FCF737FD80E709F063F8000618
:10D350004FD40E208DF80500207A8DF813006068F8
:10D36000CDF807002068CDF80B001298CDF80F001B
:10D37000274905A836F0A4F80DF10600FDF70FF8CF
:10D38000000636D401A807F0D8F8000631D401A869
:10D3900008F054FA00062CD46846FDF70AFF000690
:10D3A00027D49DF8000090B11A48007878B114A8ED
:10D3B000FCF7F5FF00061CD48DF85C502068159032
:10D3C0001298169014A806F064FB000611D4FCF71E
:10D3D00044FC00060DD401A807F0DAF8000608D4D2
:10D3E00001A808F056FA000603D4FCF742FC000638
:10D3F00002D508F0ABFCA5E7054900200870FCF752
:10D4000045FC23E704000010080000100C00001089
:10D41000040800100844000030B504460079544D5B
:10D4200093B008B110280AD98620524928600320F9
:10D430000860784650490860862013B030BD4FF030
:10D440000040FCF7BDFB000601D52868F5E76846FB
:10D45000FCF7B6FF000636D421466846FCF719F8FB
:10D46000000630D46846FCF7A1FF00062BD42079D3
:10D470006946FCF7DAFF000625D421466846FCF72A
:10D4800008F800061FD420796946FCF7C2FF0006A1
:10D4900019D4201DFDF780F8000614D42046FDF7AE
:10D4A0006AF800060FD46846FDF7A2F900060AD410
:10D4B00021466846FBF7CCFF000604D46846FDF71A
:10D4C0008EF9000602D5FCF776FCB6E708F082FF7D
:10D4D000000647D408208DF805000025CDF8065039
:10D4E0000DF10B00FDF72FF800063BD46846FDF761
:10D4F0003BF8000636D4BDF80000ADF80C008DF8FE
:10D500000A502068CDF80E0001A807F016F80006B2
:10D5100028D401A808F092F9000623D46846FDF744
:10D5200048FE00061ED49DF8000048B1134800785C
:10D5300030B12068129012A806F0FEFA000611D44D
:10D54000FCF78BFB00060DD401A807F021F80006BC
:10D5500008D401A808F09DF9000603D4FCF789FB64
:10D56000000602D508F0F2FBADE7FCF78FFB64E79D
:10D5700004000010080000100C0000100844000017
:10D5800030B504460079694D95B008B110280AD924
:10D59000862067492860032008607846654908604E
:10D5A000862015B030BD4FF00040FCF709FB0006A7
:10D5B00001D52868F5E711A8FCF702FF000650D452
:10D5C000214611A8FBF744FF00064AD411A8FCF736
:10D5D000EDFE000645D4207911A9FCF726FF0006D0
:10D5E0003FD4214611A8FBF733FF000639D4207938
:10D5F00011A9FCF70EFF000633D412A8FDF7CAFBF1
:10D6000000062ED49DF8480088B111A9FDF7B0FBA3
:10D61000000626D4214611A8FBF73BFF000620D4C4
:10D6200011A99DF84800FDF796FB000619D411A832
:10D63000FDF7DEF8000614D4214611A8FBF729FFF8
:10D6400000060ED411A8FDF7CAF8000609D4201D63
:10D65000FCF7A2FF000604D42046FCF78CFF00066E
:10D6600002D5FCF7A8FB9CE708F074FE000656D430
:10D6700004208DF8010013A94C2012F0C3FE00060F
:10D680004DD49DF84C00800702D49DF8480020B985
:10D69000684606F052FF000641D49DF84C009DF804
:10D6A000481000F00100401E084204D1684608F00E
:10D6B000C5F8000633D411A8FDF77BFD00062ED473
:10D6C0009DF8440048B11C48007830B1206814909F
:10D6D00014A806F05BFA000621D4FCF7BEFA000697
:10D6E0001DD49DF84C00800702D49DF8480020B955
:10D6F000684606F04DFF000611D49DF84C009DF8D9
:10D70000481000F00100401E084204D1684608F0AD
:10D71000C0F8000603D4FCF7ACFA000602D508F006
:10D7200015FB9EE7FCF7B2FA3BE70000040000108F
:10D73000080000100C0000100844000030B504463A
:10D740000079544D93B008B110280AD98620524967
:10D75000286003200860784650490860862013B08E
:10D7600030BD4FF00040FCF72BFA000601D52868C9
:10D77000F5E76846FCF724FE000636D421466846E5
:10D78000FBF766FE000630D46846FCF70FFE000685
:10D790002BD420796946FCF748FE000625D42146A3
:10D7A0006846FBF755FE00061FD420796946FCF752
:10D7B00030FE000619D4201DFCF7EEFE000614D43E
:10D7C0002046FCF7D8FE00060FD46846FDF736F871
:10D7D00000060AD421466846FBF73AFE000604D448
:10D7E0006846FDF721F8000602D5FCF7E4FAB6E733
:10D7F00008F090FD000647D407208DF805000025AD
:10D80000CDF806500DF10B00FCF79DFE00063BD451
:10D810006846FCF7A9FE000636D4BDF80000ADF856
:10D820000C008DF80A502068CDF80E0001A806F013
:10D8300084FE000628D401A808F000F8000623D4CE
:10D840006846FDF7B6FC00061ED49DF8000048B1FE
:10D850001348007830B12068129012A806F0C3F97E
:10D86000000611D4FCF7F9F900060DD401A806F062
:10D870008FFE000608D401A808F00BF8000603D4B8
:10D88000FCF7F7F9000602D508F060FAADE7FCF7FF
:10D89000FDF964E704000010080000100C000010FF
:10D8A0000844000070B504460079684E96B0032520
:10D8B00008B1102809D9862030606548056078468F
:10D8C00064490860862016B070BD4FF00040FCF738
:10D8D00077F9000601D53068F5E711A8FCF770FD6F
:10D8E000000650D4214611A8FBF7D3FD00064AD408
:10D8F00011A8FCF75BFD000645D4207911A9FCF7BF
:10D9000094FD00063FD4214611A8FBF7C2FD000696
:10D9100039D4207911A9FCF77CFD000633D412A874
:10D92000FDF738FA00062ED49DF8480088B111A9F9
:10D93000FDF71EFA000626D4214611A8FBF7A9FD23
:10D94000000620D411A99DF84800FDF704FA00064E
:10D9500019D411A8FCF772FF000614D4214611A8AF
:10D96000FBF797FD00060ED411A8FCF75DFF00063B
:10D9700009D4201DFCF710FE000604D42046FCF755
:10D98000FAFD000602D5FCF716FA9CE708F082FCC7
:10D99000000655D48DF8015013A94C2012F032FD29
:10D9A00000064DD49DF84C00800702D49DF8480035
:10D9B00020B9684606F0C1FD000641D49DF84C0030
:10D9C0009DF8481000F00100401E084204D168464E
:10D9D00007F034FF000633D411A8FDF7EAFB000678
:10D9E0002ED49DF8440048B11B48007830B120681F
:10D9F000149014A806F021F9000621D4FCF72DF9A3
:10DA000000061DD49DF84C00800702D49DF8480004
:10DA100020B9684606F0BCFD000611D49DF84C0004
:10DA20009DF8481000F00100401E084204D16846ED
:10DA300007F02FFF000603D4FCF71BF9000602D500
:10DA400008F084F99FE7FCF721F93CE70400001097
:10DA5000080000100C0000100844000010B5044637
:10DA600094B04FF00040FCF7ABF8000603D54348F4
:10DA7000006814B010BD12A8FCF7A2FC000626D462
:10DA800012A8FCF7CDFD000621D412981190214672
:10DA900011A8FBF7FEFC000619D411A8FCF786FCC0
:10DAA000000614D411A8FCF7E8FC00060FD42146A8
:10DAB00011A8FBF7CDFC000609D411A8FCF7D3FC94
:10DAC000000604D42046FCF79AFD000602D5FCF7B8
:10DAD00072F9CEE708F0B3FB000648D408208DF8B1
:10DAE00001001298CDF802000DF10700FCF76FFD60
:10DAF00000063CD411A8FCF77BFD000637D4BDF826
:10DB00004400ADF8080000208DF806002068CDF82C
:10DB10000A00684606F011FD000628D4684607F0A2
:10DB20008DFE000623D411A8FDF743FB00061ED48A
:10DB30009DF8440048B11248007830B12068139035
:10DB400013A805F0F9FF000611D4FCF786F80006CB
:10DB50000DD4684606F01CFD000608D4684607F0A0
:10DB600098FE000603D4FCF784F8000602D508F0FE
:10DB7000EDF8ACE7FCF78AF87BE700000400001042
:10DB80000844000030B5044695B04FF00040FCF763
:10DB900017F8564D000619D411A8FCF711FC000621
:10DBA00031D411A8FCF73CFD00062CD4214611A865
:10DBB000FBF74EFC000626D411A8FCF7F7FB000685
:10DBC00021D412A8FDF7E6F8000602D5286815B0A2
:10DBD00030BD9DF84800C8B111A9FDF7C9F800068D
:10DBE00011D4214611A8FBF754FC00060BD411A94F
:10DBF0009DF84800FDF7AFF8000604D42046FCF776
:10DC0000FEFC000611D5FCF7D6F8E0E711A8FCF7FA
:10DC100034FC0006F7D4214611A8FBF73AFC0006B5
:10DC2000F1D411A8FCF71FFCE6E708F0E8FA0006BB
:10DC300056D404208DF8010013A94C2012F0E2FB09
:10DC400000064DD49DF84C00800702D49DF8480092
:10DC500020B9684606F071FC000641D49DF84C00DE
:10DC60009DF8481000F00100401E084204D16846AB
:10DC700007F0E4FD000633D411A8FDF79AFA000678
:10DC80002ED49DF8440048B11948007830B120687E
:10DC9000149014A805F07AFF000621D4FBF7DDFFED
:10DCA00000061DD49DF84C00800702D49DF8480062
:10DCB00020B9684606F06CFC000611D49DF84C00B3
:10DCC0009DF8481000F00100401E084204D168464B
:10DCD00007F0DFFD000603D4FBF7CBFF000602D5FB
:10DCE00008F034F88FE7FBF7D1FF70E7040000106D
:10DCF0000844000030B5044695B04FF00040FBF7F3
:10DD00005FFF444D000656D412A8FCF759FB0006ED
:10DD100026D412A8FCF784FC000621D41298119096
:10DD2000214611A8FBF794FB000619D411A8FCF7B3
:10DD30003DFB000614D411A8FCF7B0FB00060FD47D
:10DD4000214611A8FBF784FB000609D411A8FCF7B3
:10DD50009BFB000604D42046FCF751FC000603D5CB
:10DD6000FCF729F815B030BD08F0E9F900064AD4EF
:10DD700011A8FDF71EFA000645D49DF8440048B1ED
:10DD80002548007830B12068139013A805F02BFFC8
:10DD9000000638D407208DF801001298CDF8020053
:10DDA0000DF10700FCF713FC000604D411A8FCF7E2
:10DDB0001FFC000601D52868D4E7BDF84400ADF883
:10DDC000080000208DF806002068CDF80A0068469B
:10DDD00006F0B3FB000616D4684607F02FFD0006D8
:10DDE00011D4FBF73AFF00060DD4684606F0D0FBCD
:10DDF000000608D4684607F04CFD000603D4FBF784
:10DE000038FF000602D507F0A1FFA9E7FBF73EFFA8
:10DE1000A8E70000040000100844000010B5044604
:10DE200096B04FF00040FBF7CBFE000603D55548F7
:10DE3000006816B010BD11A8FCF7C2FA00062ED477
:10DE400011A8FCF7EDFB000629D4214611A8FBF729
:10DE500020FB000623D411A8FCF7A8FA00061ED464
:10DE600012A8FCF797FF000619D49DF84800C8B126
:10DE700011A9FCF77DFF000611D4214611A8FBF77C
:10DE800008FB00060BD411A99DF84800FCF763FFBE
:10DE9000000604D42046FCF7B2FB000611D5FBF7C0
:10DEA0008AFFC6E711A8FCF7F9FA0006F7D4214665
:10DEB00011A8FBF7EEFA0006F1D411A8FCF7E4FA7A
:10DEC000E6E708F01CF9000656D403208DF801009F
:10DED00013A94C2012F096FA00064DD49DF84C0080
:10DEE000800702D49DF8480020B9684606F025FB5B
:10DEF000000641D49DF84C009DF8481000F0010048
:10DF0000401E084204D1684607F098FC000633D44E
:10DF100011A8FDF74EF900062ED49DF8440048B133
:10DF20001948007830B12068149014A805F085FED7
:10DF3000000621D4FBF791FE00061DD49DF84C008D
:10DF4000800702D49DF8480020B9684606F020FBFF
:10DF5000000611D49DF84C009DF8481000F0010017
:10DF6000401E084204D1684607F093FC000603D423
:10DF7000FBF77FFE000602D507F0E8FE8FE7FBF710
:10DF800085FE56E7040000100844000000B593B079
:10DF90004FF00040FBF714FE000603D51B48006855
:10DFA00013B000BD08F08BF8000626D410208DF8C1
:10DFB000010011A8FCF704FA00061ED41198CDF850
:10DFC0000200684606F0B9FA000616D4684607F063
:10DFD00035FC000611D4FBF740FE00060DD4684660
:10DFE00006F0D6FA000608D4684607F052FC000690
:10DFF00003D4FBF73EFE000604D507F0A7FEFBF7AF
:10E00000DAFECDE7FBF742FECAE70000040000108D
:10E01000F0B5734D070095B0288802D040F020007D
:10E0200001E040F0100028804FF00040FBF7C8FDF1
:10E030006C4E000671D412A8FCF7B1F9000668D442
:10E0400069469DF84800FCF76AFB000661D4BDF8FC
:10E0500000006946401CADF800009DF84800FCF740
:10E0600051FB000655D46846FCF77AF8000650D4F8
:10E070006846FBF74FFC00064BD46846FCF766F891
:10E08000000646D46846FCF77CF8000641D4684692
:10E09000FBF71BFC00063CD46846FCF768F800065A
:10E0A00037D46846FCF77EF8000632D46846FBF7A2
:10E0B00031FC00062DD46846FCF76AF8000628D427
:10E0C000002468460094FCF771F900067AD468468B
:10E0D000FDF76FF8000602D507F038FE19E00220C0
:10E0E0002DF0DCFC000614D438003F4F0DD09DF815
:10E0F000000028B1387818B104F0D2FD000608D429
:10E1000007F0A8FF000604D411E007F0A3FF000603
:10E1100004D5FBF750FE15B0F0BD53E09DF80000AC
:10E1200028B1387818B104F0BBFD0006D4D413A987
:10E130006A2012F032FA000644D49DF84C0010F028
:10E1400002008DF84C0002D0742011F086F98DF891
:10E1500000406846FCF719F90006BDD48DF8004070
:10E160006846FBF7E2FF0006B6D46846FBF7B1FF4E
:10E170000006B1D49DF80000022806D18DF80040B9
:10E180006846FBF77AFF0006A6D402208DF805004A
:10E1900007F09EFA00069FD401A806F0CEF900060B
:10E1A0009AD4FBF75AFD000696D401A806F0F0F9C0
:10E1B000000691D4FBF75DFD00068DD4FBF766FDEC
:10E1C000000601D53068A6E7288820F0B000288036
:10E1D00006483460046078460549086000209AE7E4
:10E1E0004A1E00200400001008440000080000102F
:10E1F0000C000010FE49008808807047FC4909881F
:10E2000001807047FA49008848807047F84949887A
:10E210000180704730B593B005460B208DF80100A2
:10E2200011A8FBF7AEFFF34C000630D4BDF8440054
:10E23000ADF80A0011A8FBF793FF000627D4119848
:10E24000CDF8060028798DF80C002888ADF802007A
:10E250006888ADF80400684606F06FF9000616D429
:10E26000684607F0EBFA000611D4FBF7F6FC00064F
:10E270000DD4684606F08CF9000608D4684607F00D
:10E2800008FB000603D4FBF7F4FC000602D5206867
:10E2900013B030BDD8490020206008607846D749C7
:10E2A00008600020F4E72DE9F34F9BB007461C9966
:10E2B000002011900870CE493888DFF83CB3088000
:10E2C000788848803879CB4D862408B11E2804D937
:10E2D00005212C60CBF8001012E0388848F6AD61BB
:10E2E000142688421DD878884FF01708B0F5B46F0F
:10E2F0000DD32C607846C149CBF80080086002E05D
:10E300007946BE48016086201DB0BDE8F08F05A8A3
:10E31000FBF759FF00067CD43888BDF814108842FA
:10E3200003D22C60CBF80060EAE70DD105A8FBF71B
:10E330005BFF0006EFD47888BDF81410884203D242
:10E340002C60CBF80080DBE702A8FBF76FFF00062C
:10E35000E1D405A8FCF734F80006DCD4059902984E
:10E36000814209D08C20286000207946CBF800003B
:10E37000A24801608C20C7E7022006F0FCFD0006E1
:10E38000C9D4012004F0E7FF0006C4D44FF00040D8
:10E39000FBF716FC0006BED46846FCF700F8000642
:10E3A0007DD405A8FCF70CF80006F9D4059898B1BF
:10E3B00002A99DF80000FCF784F90006F0D405A935
:10E3C00002A8FAF7ABFF0006EAD402A99DF8000004
:10E3D000FCF76AF90006E3D405A8FCF729FC00065F
:10E3E000DED4059898B102A99DF80000FCF734FC32
:10E3F0000006D5D405A902A8FAF790FF0006CFD4ED
:10E4000002A99DF80000FCF71AFC0006C8D402A976
:10E4100000E0D9E09DF80000FCF769F90006BFD4E0
:10E42000BDF8080002A9401CADF808009DF80000E6
:10E43000FCF750F90006B3D405A8FBF7D2FF00069D
:10E44000AED4BDF8140098B102A99DF80000FCF705
:10E45000F3FA0006A4D405A902A8FBF76DF800069C
:10E460009ED402A99DF80000FCF7D9FA000697D4C3
:10E4700005A8FBF7C7FF000692D4BDF81400A8B1A9
:10E4800002A99DF80000FCF7EDFA000688D405A962
:10E4900002A8FBF751F8000687D402A900E08AE23F
:10E4A0009DF80000FCF7D1FA000687D401208DF812
:10E4B0000400C0B205A9FBF7B8FF000684D4059894
:10E4C000B8B19DF8041002AA9DF80000FCF740F9CD
:10E4D000000685D405A902A8FAF720FF000688D413
:10E4E0009DF8041002AA9DF80000FCF721F900062F
:10E4F00085D49DF8040005A9FBF7ACFF000685D480
:10E500000598B8B19DF8041002AA9DF80000FCF728
:10E510003BF900068FD405A902A8FAF778FF000698
:10E5200089D49DF8041002AA9DF80000FCF71FF999
:10E53000000685D49DF80400401CC0B28DF804008C
:10E540001028B6D905A8FBF798FF000688D4059EC9
:10E550004FF000089EB102A99DF80000FCF798F961
:10E56000000684D405A902A8FAF7D8FE00068DD4C7
:10E5700002A99DF80000FCF77EF9000686D405A8E4
:10E58000FBF78CFF000687D405984FF00009B0F127
:10E59000000A13D002A99DF80000FCF78FF90006CD
:10E5A0008CD405A902A8FAF7B9FE000686D402A900
:10E5B0009DF80000FCF775F900068AD401A90B202C
:10E5C00011F020FF000601D528689DE69DF80400A3
:10E5D000012801D0032823D105A8FBF7F1FE00068E
:10E5E00086D402AA01219DF80000FCF7E9F807E0B3
:10E5F000661E002004000010080000100C0000102F
:10E60000000687D405A902A8FAF788FE000687D479
:10E6100002AA01219DF80000FCF7C2F8000688D488
:10E620009DF80400022803D0042801D0062873D1E5
:10E6300046EA0A0048EA090108436ED086EA0A0160
:10E6400088EA0900014368D000200990BAEB06016E
:10E6500079EB080005D2B6EB0A0A68EB0904012041
:10E6600004E0BAEB060A69EB080400201A900020C7
:10E6700081468046064601208DF80400C0B205A9F7
:10E68000FBF7D3FE00068BD405999DF8040019EB27
:10E69000010948EB060805A9FBF7DCFE000685D456
:10E6A000059810B10998401C09909DF80400401C81
:10E6B000C0B28DF804001028E0D9002610208DF893
:10E6C0000400C0B205A9FBF7B0FE000688D4059887
:10E6D000049030434BD00498AAFB003204FB002086
:10E6E0000AFB06015FEA58024FEA39001818514147
:10E6F0004A46434634F0C0FBBAEB000A049A64EB86
:10E700000104B9EB02091A9A68EB060832B1049ABF
:10E71000101A66EB010604E082E056E0049A101835
:10E720004E4109990590491E09919DF8041002AACD
:10E730009DF80000FCF744F80006A4D405A902A83F
:10E74000FAF7ECFD00069ED49DF8041002AA9DF88D
:10E750000000FCF725F8000695D400BF9DF80400E2
:10E76000401E10F0FF008DF80400AAD158E05AEACC
:10E770000400F3D059EA0800F0D19DF8040005A97F
:10E78000FBF768FE00068AD405980028E6D01A98A0
:10E7900048B1092028600020CBF800007846FE49E7
:10E7A00008600920B0E5099800EBD070421012EB28
:10E7B0000A0044EBE271099A4FEAE27334F05CFB21
:10E7C000BAEB000A64EB0104A8E701208DF804000D
:10E7D000C0B205A9FBF729FE0006AED40598B8B172
:10E7E0009DF8041002AA9DF80000FBF7E9FF00065F
:10E7F000A3D405A902A8FAF791FD00069DD49DF8BF
:10E80000041002AA9DF80000FBF7CAFF000694D48A
:10E810009DF80400401CC0B28DF804001028D7D920
:10E8200001248DF8044000BF9DF8040005A9FCF701
:10E830009FFA000687D40598B8B19DF8041002AA83
:10E840009DF80000FCF778FA000685D405A902A817
:10E85000FAF764FD000696D49DF8041002AA9DF80C
:10E860000000FCF759FA00068DD49DF80400401C06
:10E87000C0B28DF804001128D6D305A8FBF7B8FF65
:10E880000006AAD4059898B102A99DF80000FBF7EC
:10E89000C2FF0006A1D405A902A8FAF73FFD0006B1
:10E8A0009BD402A99DF80000FBF7A8FF000694D4B2
:10E8B00005A8FBF7C3FF00067DD4059898B102A90F
:10E8C0009DF80000FBF7CEFF000674D405A902A84E
:10E8D000FAF724FD00066ED402A99DF80000FBF7AC
:10E8E000B4FF000667D48DF8044000BF9DF8040013
:10E8F00005A9FBF7AEFC00065DD40598B8B19DF8FC
:10E90000041002AA9DF80000FBF7F1FF000652D4A4
:10E9100005A902A8FAF702FD00064CD49DF80410E0
:10E9200002AA9DF80000FBF7D2FF000643D49DF831
:10E930000400401CC0B28DF804000B28D6D305A8F3
:10E94000FBF73EFD000636D4059898B378883C2145
:10E95000B0FBF1F0401CC1B28DF8041002AA9DF882
:10E960000000FBF7E3FF000625D405A902A8FAF78B
:10E97000D5FC00061FD49DF8041002AA9DF80000E3
:10E98000FBF7C4FF000616D4397902AA9DF80000EF
:10E99000FBF7EBFF00060ED405A902A8FAF7BEFCB0
:10E9A000000608D4397902AA9DF80000FBF7CDFFD4
:10E9B000000600D400E087E08DF804409DF80400D4
:10E9C00005A9FCF781F900067ED49DF8041002AA7F
:10E9D0009DF80000FCF791F9000675D405A902A87E
:10E9E000FAF79CFC00066FD49DF8041002AA9DF86B
:10E9F0000000FCF772F9000666D49DF80400401C84
:10EA0000C0B28DF804000528D8D902A90120FBF76F
:10EA100084FB000658D405A90120FBF71AFC000668
:10EA200052D49DF80000012814D002280DD00328EC
:10EA30000BD004280ED0882002212860CBF80010CB
:10EA400079465548016088205EE405A902A8FAF7D6
:10EA500008FE03E005A902A8FAF7C8FD00067AD46B
:10EA600002A90120FBF74DFB000674D4012006F03B
:10EA700082FA00066FD413A8FCF79BFB00066AD449
:10EA800046499DF84C004FF092060978084267D03D
:10EA900016A9032006F0F2F900065CD418A9052097
:10EAA00004F032FB000656D4052216A918A834F04B
:10EAB000DBFC88B1FBF77FF9422010F0CEFC082088
:10EAC0002DF076FC312000E01BE02E60CBF800003A
:10EAD0007846314908605CE012A9002004F014FB7C
:10EAE000000638D49DF8480080062FD507F092FA2A
:10EAF000000604D43846FFF78DFB000602D507F068
:10EB000025F928E03888ADF828007888ADF82A0083
:10EB100038798DF82C0014A90AA805F0BBF8DBF8A9
:10EB2000000028280FD028780006E8D414A8FBF7A6
:10EB300088FD0006E3D415A8FBF794FD0006DED49B
:10EB40001C98047015E001201190EFE705A8FBF771
:10EB500037FC000602D5FBF72EF90CE4059840B906
:10EB600007F058FA0006CAD43846FFF753FB0006F0
:10EB7000C5D48DF8044001A8FBF77FFA0006BED487
:10EB8000119868B128212E60CBF800107946024810
:10EB90000160922019E500000C00001008440000FC
:10EBA000FBF774F811E50000F8B5054646793B4CD3
:10EBB0003B4A3C4B86200EB1022E02D92060072032
:10EBC00005E02E790EB11E2E06D9206005201060BA
:10EBD000784618608620F8BD29B16988288801F038
:10EBE00077FD000641D4002701260097694630468C
:10EBF000FBF723FB000638D4761CF6B20B2EF5D3B8
:10EC00006846FBF72EFB00062FD46846FBF74BFB4C
:10EC100000062AD46846FBF7FFFA000625D4ADF8B3
:10EC200000706846FBF72EFB00061ED46846FBF713
:10EC30004BFB000619D42846FBF7BBFA000614D498
:10EC4000A81CFBF7C7FA00060FD4281DFBF7D3FA60
:10EC500000060AD4012007F0C3FC000605D44FF0DB
:10EC60000040FAF7ADFF000601D52068F8BD02208C
:10EC70008DF800006846FBF758FA000607D40A49E9
:10EC800001200870681DFBF7FEFC000602D5FBF7AB
:10EC900092F8F8BDFAF7FAFFF8BD00000400001082
:10ECA000080000100C000010481E00201CB54FF09A
:10ECB0000040FAF785FF000602D5174800681CBD22
:10ECC00007F0DEFD00061ED400248DF800406846E3
:10ECD000FBF72BFA000616D48DF8044001A8FBF7C9
:10ECE000D2FC00060FD46846FBF7F3F900060AD4FD
:10ECF0009DF8000002280BD18DF800406846FBF714
:10ED0000BCF9000604D507F021F8FBF754F81CBD48
:10ED1000FAF7BCFF1CBD0000040000102DE9F04F05
:10ED2000054600799A4C9B4E9B4F97B04FF0860852
:10ED30004FF0050B08B11E2804D9C4F80080C6F8AE
:10ED400000B017E0288848F6AD614FF014098842FA
:10ED500005D900BFC4F80080C6F800900AE06888B2
:10ED60004FF0170AB0F5B46F0AD300BFC4F80080A3
:10ED7000C6F800A078463860862017B0BDE8F08F4E
:10ED800002A8FBF720FA000615D42888BDF8081061
:10ED90008842DFD309D102A8FBF726FA00060AD47D
:10EDA0006888BDF808108842E0D34FF00040FAF7B9
:10EDB00007FF000601D52068DFE76846FBF76DFC1A
:10EDC00000067CD402A8FBF731FA000677D402983B
:10EDD00098B103A99DF80000FBF7E3FD00066ED48F
:10EDE00002A903A8FAF79AFA000668D403A99DF8C5
:10EDF0000000FBF7C9FD000661D403A99DF80000DF
:10EE0000FBF7E5FD00065AD4BDF80C0003A9401C31
:10EE1000ADF80C009DF80000FBF7CCFD00064ED4C9
:10EE20000120804602A9FBF714FA000647D4029895
:10EE3000A8B103AA41469DF80000FBF7E1FD0006DA
:10EE40003DD402A903A8FAF769FA000637D403AA49
:10EE500041469DF80000FBF7C3FD00062FD408F1E2
:10EE60000100C0B280460A28DCD903A90120FBF7C3
:10EE700054F9000623D402A90120FBF7EAF90006A1
:10EE80001DD49DF800004FF0880801280BD00228FF
:10EE900003D00220C4F800801DE002A903A8FAF7FD
:10EEA000E0FB04E00BE002A903A8FAF79FFB0006D1
:10EEB00005D403A90120FBF724F9000602D5FAF7CF
:10EEC0007AFF5AE79DF80000012809D002280AD0ED
:10EED0000920C4F8008030607846386088204CE70C
:10EEE0008DF815B002E006208DF8150002A8FBF79A
:10EEF00048F9000642D4BDF80800401CADF81E00D9
:10EF000002A8FBF72DF9000638D40298401CCDF872
:10EF10001A0002A8FBF732FA00062FD402980890D4
:10EF20001E490DF1250034F0CBFA28798DF8240024
:10EF30002888ADF816006888ADF8180006F0C8FB00
:10EF400000061BD405A805F0F8FA000616D405A89B
:10EF500006F074FC000611D4FAF77FFE00060DD40B
:10EF600005A805F015FB000608D405A806F091FCDD
:10EF7000000603D4FAF77DFE000602D506F0E6FE91
:10EF80009DE7064900200870FAF780FEF5E60000CC
:10EF900004000010080000100C000010040800100D
:10EFA00030B5044600785C4D95B008B10A280AD9FE
:10EFB00086205A492860042008607846584908602D
:10EFC000862015B030BDA0681190211D11A8FAF758
:10EFD00008FC000605D44FF00040FAF7F1FD0006EA
:10EFE00001D52868EDE712A8FBF745F9000650D4D3
:10EFF00011A912A8FAF72CFA00064AD412A8FBF7B6
:10F0000030F9000645D412A8FBF746F9000640D4B3
:10F01000BDF84800401CADF8480012A8FBF732F9D3
:10F02000000636D4207812A9FBF713F9000630D475
:10F0300011A912A8FAF70CFA00062AD4207812A90E
:10F04000FBF7FBF8000624D412A8FBF7EFF8000644
:10F050001FD411A912A8FAF7FBF9000619D412A8B7
:10F06000FBF7DAF8000614D42046FBF73EF9000659
:10F070000FD4201DFBF756F900060AD404F108004E
:10F08000FBF761F9000604D411A8FBF76DF900063F
:10F0900002D5FAF790FE94E707F0FCF9000635D4A4
:10F0A00013A8FBF74CF8000630D49DF84C0002285A
:10F0B00003D107F0F9FB000628D49DF84C00012885
:10F0C00027D109208DF8010020788DF802001198D1
:10F0D000CDF80300684605F030FA000616D46846FD
:10F0E00006F0ACFB000611D4FAF7B7FD00060DD40C
:10F0F000684605F04DFA000608D4684606F0C9FBDC
:10F10000000603D4FAF7B5FD000602D506F01EFE90
:10F11000BFE7FAF7BBFD54E7040000100800001039
:10F120000C00001030B504460078544D93B008B17F
:10F130000A280AD9862052492860042008607846A7
:10F1400050490860862013B030BDA0681190211D81
:10F1500011A8FAF746FB000605D44FF00040FAF775
:10F160002FFD000601D52868EDE712A8FBF783F80C
:10F17000000650D411A912A8FAF78BF900064AD458
:10F1800012A8FBF76EF8000645D412A8FBF784F826
:10F19000000640D4BDF84800401CADF8480012A855
:10F1A000FBF770F8000636D4207812A9FBF751F867
:10F1B000000630D411A912A8FAF76BF900062AD478
:10F1C000207812A9FBF739F8000624D412A8FBF71F
:10F1D0002DF800061FD411A912A8FAF75AF9000653
:10F1E00019D412A8FBF718F8000614D42046FBF730
:10F1F0007CF800060FD4201DFBF794F800060AD413
:10F2000004F10800FBF79FF8000604D411A8FBF7EF
:10F21000ABF8000602D5FAF7CEFD94E707F05AF9ED
:10F22000000624D40A208DF8010020788DF8020011
:10F230001198CDF80300684605F07FF9000616D452
:10F24000684606F0FBFA000611D4FAF706FD000640
:10F250000DD4684605F09CF9000608D4684606F00F
:10F2600018FB000603D4FAF704FD000602D506F0E9
:10F270006DFDD0E7FAF70AFD65E700000400001015
:10F28000080000100C00001030B504460078564D00
:10F2900093B008B10A280AD986205449286004206E
:10F2A0000860784652490860862013B030BDA068D7
:10F2B0001190211D11A8FAF794FA000605D44FF019
:10F2C0000040FAF77DFC000601D52868EDE712A89A
:10F2D000FAF7F3FF000650D411A912A8FAF7B8F80C
:10F2E00000064AD412A8FAF7DEFF000645D412A899
:10F2F000FAF7F4FF000640D4BDF84800401CADF812
:10F30000480012A8FAF7E0FF000636D4207812A9C8
:10F31000FAF79FFF000630D411A912A8FAF7B9F83E
:10F3200000062AD4207812A9FAF787FF000624D411
:10F3300012A8FAF77BFF00061FD411A912A8FAF74A
:10F34000A8F8000619D412A8FAF766FF000614D42C
:10F350002046FAF7CAFF00060FD4201DFAF7E2FF95
:10F3600000060AD404F10800FAF7EDFF000604D401
:10F3700011A8FAF7F9FF000602D5FAF71CFD94E789
:10F3800007F0C8F8000629D411208DF8010012A852
:10F39000FAF771FF000621D41298CDF802001198F7
:10F3A000CDF80600684605F0C8F8000616D4684691
:10F3B00006F044FA000611D4FAF74FFC00060DD40B
:10F3C000684605F0E5F8000608D4684606F061FADC
:10F3D000000603D4FAF74DFC000602D506F0B6FC91
:10F3E000CBE7FAF753FC60E70400001008000010B8
:10F3F0000C0000102DE9F04F85B06846FAF747FE83
:10F40000F84F00060ED49DF80000DFF8DC93DFF81B
:10F41000DCA30024012809D001A90120FBF751F940
:10F42000000607D5386805B0BDE8F08F3C60C9F824
:10F4300000401CE18DF800400DF104029DF8000031
:10F440009DF80410135C401CC0B219448DF80410E0
:10F450008DF800000528F1D31046FAF787F800066A
:10F460007DD4A0460494ADF80C400124E04EDFF8B2
:10F4700084B325463078022805D000EB40000BEB22
:10F48000C00040688047E8B2054601A9FBF70CF9C7
:10F490000006E5D401A92846FBF7D1FB0006DFD41E
:10F4A00003A92846FBF716F90006D9D403A9284674
:10F4B000FBF728F90006D3D403A92846FBF7AFFAD7
:10F4C00000064CD403A92846FBF7BFFA000646D431
:10F4D0008DF800409DF8001001AA2846FBF728F996
:10F4E00000063CD49DF8001004AA2846FBF73FF91B
:10F4F000000634D49DF8001001AA2846FBF750F905
:10F5000000062CD49DF80000401CC0B28DF800000D
:10F510001028DFD901A92846FBF7ADF900061ED453
:10F5200001A92846FBF7BDF9000618D48DF8004064
:10F530009DF8001001AA2846FBF7C9F900060ED471
:10F540009DF80000401CC0B28DF800000A28EFD9D9
:10F550008DF800409DF8001001AA284600E073E0F5
:10F56000FBF7D4F900066FD49DF80000401CC0B230
:10F570008DF800001828EDD98DF800409DF8001096
:10F5800001AA2846FBF7E1F900065DD49DF80000CA
:10F59000401CC0B28DF800001E28EFD98DF8004045
:10F5A0009DF8001001AA2846FBF797FB00064BD4F4
:10F5B0009DF80000401CC0B28DF800000528EFD96E
:10F5C0008DF800409DF8001001AA2846FBF7A4FB27
:10F5D000000639D49DF80000401CC0B28DF8000030
:10F5E0001028EFD901A92846FBF708F900062BD40B
:10F5F00001A92846FBF729F9000625D46D1CEDB2B8
:10F60000042D7FF637AF25463078022805D000EB71
:10F6100040010BEBC10040688047E0B2044601A9FD
:10F62000FBF7B2F900060FD403A92046FBF7C2F995
:10F63000000609D428468DF80050C1B201AA204620
:10F64000FBF7CEF9000602D5FAF7B5FBEBE69DF81D
:10F650000000401CC0B28DF800000A28EDD9641CDF
:10F66000E4B2022CD0D9C7F80080C9F800807946EE
:10F670000020CAF80010D6E6F0B504460179594DCD
:10F68000594E5A4F93B0862009B11E2902D92860DD
:10F6900005200DE0218848F6AD62914202D928602C
:10F6A000142005E06188B1F5B46F07D328601720F6
:10F6B000306078463860862013B0F0BD12A9022071
:10F6C00005F03BFE000615D4BDF84800A0B104F0DB
:10F6D00043FE00060ED446480678012E04D00120D1
:10F6E00006F07EFF000605D44FF01040FAF768FAE6
:10F6F000000609D52868DFE7912028608A2030605D
:10F70000784638609120D7E7FFF774FE000620D4D2
:10F7100001F0F6F800061CD42046FBF7ACF9000611
:10F7200017D4A01CFBF7B6F9000612D4201DFBF776
:10F73000C2F900060DD401208DF800006846FAF7E2
:10F740009CFC000605D469462B2010F05BFE0006E9
:10F7500002D5FAF730FBAFE79DF80000C00701D1F2
:10F760006079E8B3012E49D06846FAF7F9FC000643
:10F7700033D46846FAF7BCF800062ED46846FAF788
:10F78000E5FC000629D406F05DFA000625D41A49E6
:10F790000220087012208DF805006946042005F04B
:10F7A0006DFB000619D4BDF80000401CADF8060042
:10F7B00020798DF810002088ADF808006088ADF839
:10F7C0000A006846FAF7CCFC000606D400980390BD
:10F7D00001A804F0DDFE000610D506F0B7FAB8E780
:10F7E0000CE0000004000010080000100C000010E5
:10F7F000E81E002034030010481E0020FAF746FAE5
:10F800005AE70000F8B505460379384C3849394ABB
:10F8100086200BB11E2B02D9206005200EE02B881C
:10F8200048F6AD671426BB4202D920600E6006E0A0
:10F830006B88B3F5B46F06D3206017200860784654
:10F8400010608620F8BD2C490120FAF73AFF000627
:10F8500040D42A490220FAF734FF00063AD4284659
:10F86000FAF7A7FC000635D4A81CFAF7B3FC00068B
:10F8700030D4281DFAF7BFFC00062BD400256846BB
:10F880000095FBF7A9F9000624D468460095FBF71C
:10F89000B4F900061ED48DF800606846FBF74FF9F6
:10F8A000000617D40120ADF800006846FBF76EF99A
:10F8B00000060FD469461C2010F0A4FD000609D4F0
:10F8C0009DF8000040B1ADF800506846FAF74FFCD3
:10F8D000000601D52068F8BD032009498DF8000015
:10F8E000022008706846FAF720FCF8BD04000010FA
:10F8F000080000100C000010741E0020791E00206B
:10F90000481E00202DE9FC414FF00040FAF758F95D
:10F910004C4C00067ED46846F9F734FE00062AD423
:10F9200001273E46F0B205466946FAF7EAFB0006B3
:10F9300021D46D1CEEB20B2EF4D300256846009541
:10F94000FAF704FC000616D4ADF800506846FAF742
:10F950000EFC00060FD468460095FAF719FC000665
:10F9600009D4ADF800700220C0B206466946FBF724
:10F97000F7F8000605D506F0E9F9FAF71CFABDE834
:10F98000FC81761CF0B21B28EED92F4F0422694669
:10F99000384625F0D1FB00064ED42C4E0098B042DC
:10F9A00027D004226946381D009525F0D0FB0006BB
:10F9B00042D4254804226946083025F0C8FB0006D9
:10F9C0003AD42148042269460C3025F0C0FB0006D9
:10F9D00032D41D4804226946103025F0B8FB0006D9
:10F9E0002AD4042269463846009625F0B0FB00066A
:10F9F00022D41548042269461430009525F0A7FB4F
:10FA0000000619D4104804226946183025F09FFBDF
:10FA1000000600E010E00FD40B48042269461C30B9
:10FA200025F095FB000607D40748042269462030DC
:10FA300025F08DFB000601D52068A0E7FAF726F92E
:10FA40009DE700000400001004000020CEFAADDEA7
:10FA5000FEB56846F9F78AFD284C000640D4002719
:10FA60000125ADF808702E46F0B206466946FAF751
:10FA70001BFE000634D402A93046FAF72BFE00061E
:10FA80002ED402A93046FAF73DFE000628D402A97A
:10FA90003046FAF7C4FF000622D402A93046FAF72E
:10FAA000D4FF00061CD469463046FAF7E4FE00068F
:10FAB00016D469463046FAF7F4FE000610D4761CD8
:10FAC000F6B2042ED0D9E8B205466946FAF75CFFD3
:10FAD000000605D402A92846FAF76CFF000601D5F6
:10FAE0002068FEBD6D1CEDB2022DECD904482760E4
:10FAF00007607846034908600020FEBD040000103E
:10FB0000080000100C0000107CB506466846F9F7A6
:10FB10002DFD0D4D000607D401246A4631462046CE
:10FB2000FAF7F4FE000601D528687CBD641CE4B237
:10FB3000052CF2D305490020286008607846044966
:10FB4000086000207CBD00000400001008000010C8
:10FB50000C0000107CB506466846F9F707FD0D4D10
:10FB6000000607D401246A4631462046FAF7EDFE26
:10FB7000000601D528687CBD641CE4B2052CF2D3D4
:10FB80000549002028600860784604490860002084
:10FB90007CBD000004000010080000100C000010E4
:10FBA000FEB507466846F9F7E1FC144D000617D488
:10FBB0000026012402966A4639462046FAF7B8FD27
:10FBC00000060DD402AA39462046FAF7D0FD0006F9
:10FBD00006D46A4639462046FAF7E2FD000601D50A
:10FBE0002868FEBD641CE4B2052CE4D304482E60F2
:10FBF00006607846034908600020FEBD040000103E
:10FC0000080000100C0000102DE9FC410746684672
:10FC1000F9F7ACFC144E000615D401252C46E0B2D1
:10FC200004466A463946FAF752FE00060BD4641CB5
:10FC3000E4B2052CF3D3E8B204466A463946FAF733
:10FC4000CFFE000602D53068BDE8FC81641CE5B239
:10FC5000032DF0D305490020306008607846044940
:10FC600008600020F0E70000040000100800001009
:10FC70000C0000102DE9F04F97B080464FF00009BE
:10FC80008A4681F80090052003F065FBFC4C0006D5
:10FC90007ED4FF2005F06FF90006F9D415A8FBF714
:10FCA00088FA0006F4D46946002005F02AF8000618
:10FCB000EED4BDF800009027F24DF34E192802D380
:10FCC00001202760E1E06946022005F036FB0006CE
:10FCD000DED4BDF8000090B1EC480DF12C0B00789B
:10FCE00000287CD06946012005F00BF80006CFD42F
:10FCF000BDF80000402805D303202760C5E00C2094
:10FD00002760C2E014A9002003F0FEF90006BFD46A
:10FD10009DF85000010902D004202760B5E00107DA
:10FD20000BD5400709D4872020607846C5F800909D
:10FD30003060872017B0BDE8F08F03A9052003F0DD
:10FD4000E3F90006A4D46946032005F097F80006FD
:10FD50009ED42068052805D0052203A9684633F003
:10FD600083FBD0B19DF8500000077DD56946002087
:10FD700005F084F800068BD403A90B2003F0C4F926
:10FD8000000685D40C2203A9684633F06DFB00E021
:10FD90008EE028B10520276077E00720276074E017
:10FDA00003A90C2003F0B0F9000691D4062208F153
:10FDB000060103A833F058FB10B10620276064E069
:10FDC00003A9112003F0A0F9000671D406224146D0
:10FDD00003A833F049FB18B10820276055E0D4E0B0
:10FDE00069460E2003F090F9000661D403A800F0E4
:10FDF000D8FC00065CD4BDF80000BDF80C108842A9
:10FE000007D963200FF029FB000651D40920276091
:10FE10003BE003A9F4F7D1FD9DF80C00694600F51D
:10FE2000FA60ADF82C009DF80D008DF82E009DF8BD
:10FE30000E008DF82F000F2003F066F9000637D46E
:10FE4000BDF800103C20B1FBF0F28DF83020B1FB82
:10FE5000F0F200FB12108DF831008DF8329003A9FA
:10FE6000102003F051F900E023E0000620D4694699
:10FE7000042005F003F800061AD4BDF80000BDF810
:10FE80000C10884206D00A2027602860784630602F
:10FE900090204FE76946062003F036F9000672D439
:10FEA000BDF80C00BDF80010401C8142EBD110E001
:10FEB00069E003F069FA00287FF46FAF0BF10400EA
:10FEC00022F0EEFF00065ED40BA823F01AF800061D
:10FED00059D404F081FA000655D40BF10701002033
:10FEE00004F0CCFF00064ED4D8F80610CDF83F1031
:10FEF000B8F80A00ADF84300D8F80010CDF8451066
:10FF0000B8F80400ADF8490013A9042004F0B6FFC6
:10FF1000000638D4D8F806100791B8F80A00ADF8F2
:10FF20002000D8F80010CDF82210B8F80400ADF881
:10FF30002600D8F80C000A9006A90BA8F4F7D8FD03
:10FF4000BDF84C00ADF81A0006A8FAF732F9000621
:10FF500019D49DF830109DF83100C1EB011100EB70
:10FF60008100ADF800006846FAF734F900060AD4BB
:10FF70004748FAF740F9000605D44FF00040F9F77A
:10FF80001FFE000604D52068D4E60BF1040097E7B5
:10FF900006F06CFB00066ED406A806F07CFB00069B
:10FFA00069D49DF85000000707D43848007820B184
:10FFB0000BA803F0F7F900065DD4344F4FF00108A9
:10FFC0008AF800803878D8B103F095FC000652D446
:10FFD0000121304806F08DFB00060AD5F4F726F91A
:10FFE00002F05EFEF4F737F905F0B0FEF9F7E3FE34
:10FFF000C9E703F0C0FC00063DD420680028E7D024
:020000040001F9
:10000000112005F050F9000635D406A9002005F0AE
:100010005AF900062FD4387858B107A9052003F003
:1000200073F8000627D406A9012005F04CF9000654
:1000300021D4122005F037F900061CD49DF8540095
:1000400050B36846FAF78CF8000614D46846F9F7FE
:100050004FFC00060FD46846FAF778F800060AD479
:10006000FBF7C3F8000606D44F468AF80090F9F76C
:100070000DFE00065AD505F069FEF9F79CFE59E61B
:1000800004000010080000100C00001008440000DC
:10009000C11E002020060010FFE747468DF80080B3
:1000A0006846FBF79FF80006E5D4ADF81090CDF850
:1000B0000C908DF81290B84638468DF80070C0B29A
:1000C00003A9FAF71EF80006D5D49DF80000401CDD
:1000D000C0B28DF800000A28F1D94F4603A8CDF828
:1000E0000C90FAF733F80006C5D403A80397FAF783
:1000F0004FF80006BFD4ADF80C7003A8FAF737F834
:100100000006B8D44046ADF80C808DF80080C0B22F
:1001100003A9FAF725FD0006ADD49DF80000401CA8
:10012000C0B28DF800001B28F1D999E72760784606
:100130002F6030600020FDE52DE9F04796B00021EA
:1001400080460170052003F006F9C04C00067DD4FE
:10015000FF2004F010FF0006F9D415A8F9F797FF67
:100160000006F4D49DF85400B94EBA4D48B1912020
:1001700020609C20286078463060912016B0BDE851
:10018000F0876946012004F0BCFD0006DFD4BDF80D
:1001900000009027402802D30320276027E069460B
:1001A000022005F0CAF80006D1D4BDF80000E0B185
:1001B00003F0EAF80006CAD428684FF002094FF0AD
:1001C000920A232809D00FA9002002F09DFF000603
:1001D000BDD49DF83C0000090BD0C4F800A07846BF
:1001E000C5F8009030609220C8E70C202760286096
:1001F00061E003A9052002F087FF0006A7D4694645
:10020000032004F03BFE0006A1D420684FF0070A4B
:1002100028B90522694603A833F026F998B39DF85A
:100220003C0000077DD56946002004F027FE00064B
:100230008DD403A90B2002F067FF000687D40C229F
:1002400003A9684633F010F920B100E0A6E00520CC
:100250002760CCE769460E2002F056FF000695D4D1
:1002600003A800F09EFA000690D4BDF80000BDF887
:100270000C10884208D063200FF0EFF8000685D4F8
:1002800009202760B3E713E06946042004F0F6FD77
:10029000000689D403A9102002F036FF00067DD4A1
:1002A000BDF80000BDF80C104FF00A0A884206D0D5
:1002B0002760C5F800A07846306090205EE7694668
:1002C000062002F021FF000668D4BDF80C00BDF83E
:1002D0000010401C8142EBD103A90C2002F014FF56
:1002E00000065BD46946012004F0C8FD000655D421
:1002F0000622694603A833F0B7F810B1062027603C
:1003000075E703A9112002F0FFFE000646D46946F6
:10031000022004F0B3FD000640D4062203A968467B
:1003200000E005E033F0A0F830B1082027605EE778
:1003300003F02AF80028BBD106AD281D22F0B0FD3D
:1003400000067BD406A822F0DCFD000676D4E91D69
:10035000002004F093FD000670D40DF12B01012064
:1003600004F08CFD000669D40DF13101022004F087
:1003700085FD000662D40EA9042004F07FFD00066E
:100380005CD4BDF83800ADF8420010A906A8F4F717
:10039000AFFB11A9052002F0B7FE00E04EE0000619
:1003A0004CD44FF00040F9F70BFC000646D406F0A1
:1003B00084F9000639D49DF83C00000704D406A84F
:1003C00002F0F0FF000630D4012188F8001003F09D
:1003D00092FA000629D4204D01211F4806F089F920
:1003E00000060AD5F3F722FF02F05AFC00061CD4DF
:1003F000F3F731FF2078000617D403F0BCFA0006AB
:1004000013D495F840000028E6D1112004F04BFFEA
:1004100000060AD410A9012004F055FF000604D4F8
:10042000122004F040FF000604D505F08FFCF9F718
:10043000C2FCA3E6F9F72AFC000601D520689DE678
:1004400088F80090012006F0CBF897E60400001031
:100450000C00001008000010200600102DE9F043E9
:100460008BB007A9012021F0D9FF5E4C00064FD4C4
:10047000684602F09FFD00064AD408A9032004F054
:10048000FDFC594DDFF86481000616D400270522D3
:1004900008A903A832F0E8FF80B142200EF0DDFF8A
:1004A000000635D4922020603120794628609220C1
:1004B000C8F800100BB0BDE8F08301279DF81100CB
:1004C0004FF0000641074FF0870903D4C4F80090AD
:1004D0002E6077E040065ED502F0B7FE00067FD4BE
:1004E00043482BF069FE00067AD406A8F9F7E0FD30
:1004F000000675D49DF818000E2801D0002FE5D015
:1005000060200EF0AAFF000603D500BF05F01EFC18
:1005100066E002F039FF000662D4684600F041F957
:1005200000065DD40DF1020000F01FF9000657D45B
:100530001E208DF80400684602F0AAFF00064FD482
:100540008DF800606846F9F798FD000648D46846C3
:1005500002F0C3FC000643D4BDF80000401E80B288
:1005600003F092F900063BD4224D0121214806F008
:10057000C0F8000606D5F3F759FE02F091FBF3F739
:100580006AFE2DE003F0F7F9000629D495F8400043
:100590000028EAD11BE00798C00707D08DF800605B
:1005A0006846F9F76AFD00061AD410E06846F9F7C4
:1005B0006EFD000614D49DF8000040B10420C4F87C
:1005C0000090286079468720C8F8001072E7332031
:1005D0000EF043FF000603D402F0D1FF000695D4CD
:1005E000206867E704000010080000100C000010ED
:1005F000082300102006001038B54FF00040F9F72E
:10060000DFFA104D000617D400248DF8004068462C
:10061000F9F7BBFE000606D48DF800406846F9F7EE
:1006200084FD000602D5F9F7C6FB38BD6846009484
:10063000F9F7BCFE000601D5286838BDF9F726FB9E
:1006400038BD0000040000101CB54FF00040F9F761
:10065000B7FA000602D51D4800681CBD01A8FAF7CC
:100660001CF800062CD46846F9F77AFD000627D45A
:100670006846F9F73DF9000622D46846F9F766FDA9
:1006800000061DD46846F9F77CFD000618D46846BC
:10069000F9F707F9000613D46846F9F768FD000674
:1006A0000ED400248DF8044001A8F9F7ECFF0006F1
:1006B00006D48DF800406846F9F737FD000602D5EC
:1006C000F9F779FB1CBDF9F7E1FA1CBD0400001035
:1006D0002DE9FC5F9B4D9C4E9C4C894607004FF0DA
:1006E00086084FF0140A03D048F6AD60874204D95B
:1006F000C4F80080C5F800A008E04FF0170BB9F56A
:10070000B46F08D3C4F80080C5F800B078463060F4
:100710008620BDE8FC9F01A8FAF7B6F900060BD4C5
:10072000BDF804003F1A4FF4B4604743E0D4684674
:10073000FAF7BAF9000601D52068EAE7BDF800101B
:10074000A9EB0100C019DDD40021B0F5B46F06DBC0
:100750008A2020607846296030608A20D9E72160AD
:100760007846296030600020D3E738B504466846F3
:1007700022F096FB0106754801D5006838BD9DF84A
:1007800000209DF80110C2EB021201EB82012180D2
:10079000002101606B48016078466B4908600020C9
:1007A00038BD38B50446684622F0ABFB000602D5DA
:1007B0006648006838BD21466846F4F799F938BDA7
:1007C0007CB50025ADF800506846FFF7CEFF5F4CC2
:1007D000000604D401A8FFF7E4FF000601D5206855
:1007E0007CBDBDF80010BDF80400FFF771FF55494E
:1007F000554A38B191202060882008607846106002
:1008000091207CBD256078460D60106000207CBD85
:100810002DE9FE43DFF8388181464A4E98F8000002
:10082000494F4A4C002510B188F8005062E06946F3
:100830003D200FF0B2FE000651D49DF80000E8B351
:10084000012188F8001001A8FFF78FFF000646D4A9
:1008500002A8FFF7A6FF000641D4BDF80800BDF8C6
:100860000410C0EB001000EB400001EB401801A8A1
:10087000FAF7F5FA000632D402A8FAF7DFFA000612
:100880002DD4BDF80800BDF80410C0EB001000EB3B
:10089000400001EB40109DF80010C1EB011100EB8E
:1008A0008101414526D8B9F1000F1BD062200EF01E
:1008B000D4FD000613D46946532000E01AE00FF07F
:1008C000A1FD00060BD49DF8000010F002008DF889
:1008D000000007D0012005F083FE000602D5206845
:1008E000BDE8FE83872020600520306078463860B0
:1008F0008720F5E725607846356038600020EFE70F
:100900001CB56846FFF731FF104C00060ED401A855
:10091000FFF747FF000609D401A8FAF785FA000699
:1009200004D46846FAF791FA000601D520681CBD88
:1009300004490020206008607846034908600020D0
:100940001CBD0000080000100C0000100400001086
:100950004601001010B5044694B04FF00040F9F77E
:100960002FF9000603D53648006814B010BD201DCD
:10097000FAF77BF9000617D404F10800FAF786F9B4
:10098000000611D4207A12A9FAF79EF900060BD4BA
:10099000211D12A8F8F75CFD000605D4207A12A9E3
:1009A000FAF785F9000602D5F9F705FADDE711A98E
:1009B0004B200FF027FD00063CD49DF84400C007F3
:1009C00003D005F0C7FD000634D413208DF80100D4
:1009D000207A8DF802006068CDF803009DF844008D
:1009E000800704D5684603F0A8FD000622D49DF8D0
:1009F0004400C00704D0684604F020FF000619D464
:100A0000F9F72BF9000615D49DF84400800704D5AA
:100A1000684603F0BDFD00060CD49DF84400C007F5
:100A200004D0684604F035FF000603D4F9F721F935
:100A3000000602D505F08AF9B6E7F9F727F994E739
:100A40000400001010B5044694B04FF00040F9F7D0
:100A5000B7F8000603D53648006814B010BD201D55
:100A6000FAF703F9000617D404F10800FAF70EF9B3
:100A7000000611D4207A12A9FAF726F900060BD441
:100A8000211D12A8F8F705FD000605D4207A12A949
:100A9000FAF70DF9000602D5F9F78DF9DDE711A98E
:100AA0004B200FF0AFFC00063CD49DF84400C0077B
:100AB00003D005F06FFD000634D414208DF801003A
:100AC000207A8DF802006068CDF803009DF844009C
:100AD000800704D5684603F030FD000622D49DF857
:100AE0004400C00704D0684604F0A8FE000619D4EC
:100AF000F9F7B3F8000615D49DF84400800704D533
:100B0000684603F045FD00060CD49DF84400C0077C
:100B100004D0684604F0BDFE000603D4F9F7A9F836
:100B2000000602D505F012F9B6E7F9F7AFF894E739
:100B30000400001070B596B0002604468DF8506091
:100B40004079B74DA0B114A8F9F7B9FC000674D4E8
:100B50009DF8500008B110280AD98620B1492860B4
:100B6000032008607846B0490860862016B070BD42
:100B70004FF00040F9F724F80006E8D46079002827
:100B800075D06846F9F71CFC00066CD4A0792146A4
:100B90000028684652D0F8F77CFC000663D468460B
:100BA000F9F704FC00065ED469469DF85000F9F799
:100BB0003CFC000657D4A07921460028684640D066
:100BC000F8F767FC00064ED469469DF85000F9F727
:100BD00020FC000647D414A8F9F7DEFC000642D436
:100BE0002046F9F7C8FC00063DD420796946FAF79B
:100BF000BFF800067FD421466846F8F729FC0006B6
:100C000079D420796946FAF7A6F8000673D4A0795A
:100C10000028684618D0F9F7EBFD00066BD4214692
:100C20006846F8F715FC000665D46846F9F7D7FD65
:100C3000000660D405F0A3FA73E0BFE0F8F708FC03
:100C4000ABE7F8F705FCBDE7F9F7F8FD000652D46D
:100C500021466846F8F7FCFB00064CD46846F9F7D5
:100C6000E3FDE5E703E046E005F070F843E013A894
:100C7000F9F7A6FB00063ED413A8F9F7D1FC00064D
:100C800039D413980090A07921460028684635D0C1
:100C9000F8F7FFFB00062ED46846F9F787FB00063D
:100CA00029D42046F9F7ABFC000624D4A07900280B
:100CB000684626D0F9F7E1FB00061CD421466846B9
:100CC000F8F7C6FB000616D46846F9F7CCFB000619
:100CD00011D420796946FAF74BF800060BD4214667
:100CE0006846F8F7B5FB000605D420796946FAF79F
:100CF00032F8000613D5F9F75EF837E7F8F7A8FBE6
:100D0000C8E7F9F7CBFB0006F5D421466846F8F7AB
:100D10009FFB0006EFD46846F9F7B6FBD7E705F06E
:100D20004EFA0006A0D4A079A8B108208DF80500DD
:100D300020798DF80A00617901A871B1CDF80660BB
:100D4000C01DF9F700FC00068ED46846F9F70CFCCC
:100D5000000689D40EE00720E8E71399CDF80610C5
:100D6000C01DF9F734FC000628D46846F9F740FCAA
:100D7000000623D4BDF80000ADF80C002068CDF8C3
:100D80000E0012A94C200FF03DFB000616D49DF872
:100D90004800800704D501A803F0CFFB0006C1D4AA
:100DA0009DF84800C00704D001A804F047FD0006E4
:100DB000B8D46846FAF7FDF9000601D52868D5E6EB
:100DC0009DF8000060B11948007848B1206815907E
:100DD000A079002815A820D002F0AEFE0006A1D40C
:100DE000F8F73BFF00069DD49DF84800800704D526
:100DF00001A803F0CDFB000694D49DF84800C0077D
:100E000004D001A804F045FD00068BD4F8F725FFB7
:100E1000000687D4F8F73AFFA8E602F0E4FEDDE723
:100E200004000010080000100C000010084400002E
:100E300071B581B04FF00040F8F7C2FE7A4C000661
:100E40003CD403208DF800006846F9F76EF90006DF
:100E500062D419208DF800006846F9F770FE00068C
:100E60005AD472490220087001A91920F9F778FEB6
:100E7000000623D4012005F0B3FB00064CD403F098
:100E80003DFD000648D4BDF8040003F09DFC0006BB
:100E900042D420680025052807D0654E03F07BFD6D
:100EA000000639D42068D8B913E0F8F784FF0006AB
:100EB00004D401202AF06CFF000601D520687CBD17
:100EC000812020605B48056078465B49086081208E
:100ED0007CBD7078062803D0052801D00B28DDD111
:100EE0002BF021FA000617D401202AF051FF00064A
:100EF00012D4012005F074FB00060DD48DF80050CB
:100F00006846F9F712F9000606D48DF800506846D5
:100F1000F9F715FE000602D5F8F74DFF7CBDF8F78E
:100F2000B5FE7CBD2DE9F843064689464FF00040EA
:100F3000F8F746FE3C4C00066CD496B103208DF8C1
:100F400000006846F9F7F1F8000622D419208DF860
:100F500000006846F9F7F3FD00061AD43349022071
:100F600008706846F9F70DF9000653D46946192050
:100F7000F9F7F6FD00064DD4012005F031FB00061F
:100F800007D404F09DFD000603D404F0ABFD000679
:100F900003D5F8F710FFBDE8F8832068254FDFF888
:100FA0009880002505280FD1F8F705FF000631D4F9
:100FB00001202AF0EDFE00062CD481202060794625
:100FC0003D60C8F80010E6E704F0D1FD000606D445
:100FD00020680028F8D02BF0A6F9000602D504F00E
:100FE000B5FED6E7F8F752FE000613D4A6B1484680
:100FF00005F0F6FA00060DD48DF800506846F9F7B2
:1010000094F8000606D48DF800506846F9F797FD6D
:10101000000601D52068BEE7256079463D600020C6
:10102000C8F80010B7E7000004000010481E0020B8
:10103000C2070010080000100C0000102DE9FC4150
:101040002F4C90460F460026C0B3FAF782F840B105
:10105000F3F7ECF800212BA02AF099FFF3F7FBF847
:1010600043E08DF800606846F8F7F8FF6846F9F746
:1010700004F802208DF800006846F9F731F8000600
:1010800033D46846F9F71BF800062ED46846F9F702
:1010900005F8000629D40120ADF80400054601A991
:1010A0002846F9F75DFD00061FD46D1C1B2DF6D9EF
:1010B00003F092F9FEF726FC000616D4C7B14046AD
:1010C0000FF084FE000610D400200FF050F9000647
:1010D0000BD40EF093FA20B900200EF0EFFC0006BE
:1010E00003D4F4F712F9000602D52068BDE8FC81AC
:1010F0000B482660066078460A4908600020F5E73C
:10110000040000108EE8A8A1AAA020A8ADA8E6A817
:10111000A0ABA8A7A0E6A8A8208E87930A0000008D
:10112000080000100C0000102DE9F0418AB0BB4807
:10113000F8F728FABA48F8F725FA06A8FAF739F8BE
:10114000B84C000652D49DF818000527B64EDFF8BB
:10115000DC82002510B307A912200FF053F9000616
:1011600044D408A92E200FF04DF900063ED405A85E
:10117000F9F7EFFC000639D49DF81C10C80705D01C
:101180009DF814000E2812D0142810D09DF81400D9
:101190000F2803D19DF82000800708D427607946E6
:1011A00035600520C8F800100AB0BDE8F081A04FF6
:1011B000880715D5002003F042FE000616D46946C4
:1011C000002003F000FE000610D4BDF8021002203B
:1011D00003F01FFE000609D4BDF80200788008E085
:1011E0000021022003F015FE000601D52068DBE790
:1011F0007D803D702560794635600020C8F800107C
:10120000D2E72DE9F04F89B04FF00005854CDFF8AB
:101210001C82854F06008DF814504FF0050B04D04A
:10122000012E02D0022870D09DE0DFF804A24FF01A
:1012300000096946022003F0C6FD20B1052830D020
:1012400093287DD152E09AF8000060B1BAF80210FC
:10125000BDF80220481C824211D0022003F0D9FDC3
:10126000000674D44AE001218AF80010BAF802108E
:10127000BDF802204B1C9A42EFD1AAF80220684820
:1012800001A9F8F774FA000661D464480DF1090168
:10129000F8F76DFA00065AD4BDF80210AAF8021049
:1012A0002CE0012E1FD105A8F8F7F1FE00064ED460
:1012B0009DF81400B8B106A90120F9F702FA00065A
:1012C00045D406A95648F8F752FA00063FD406A9B5
:1012D0000220F9F7F6F9000639D406A94F48F8F7C5
:1012E00046FA000633D48AF8005034E0BAF8021007
:1012F000491CAAF802103868082828D109F1010908
:10130000B9F1640F95DB2EE0FFE705A8F8F7BFFE03
:1013100000061CD49DF81400E8B106A90120F9F7D5
:10132000D0F9000613D406A93D48F8F720FA0006C4
:101330000DD406A90220F9F7C4F9000607D400E08D
:1013400005E006A93548F8F712FA00060BD5206823
:1013500009B0BDE8F08FC4F800B079463D600520C3
:10136000C8F80010F4E7256079463D600020C8F811
:101370000010EDE72DE9F04F83468DB08A46084610
:10138000F8F700F95846F8F7FDF80AA8F9F711FF41
:10139000244C000630D49DF82800DFF89080224FBE
:1013A000002578B3002003F04AFD000624D46946E6
:1013B000002003F008FD00061ED4BDF80210022034
:1013C00003F027FD000617D405AE0DF11D0905A990
:1013D000022003F0F8FC206810B193280FD015E02C
:1013E000311D5846F8F7C3F9000605D44946504662
:1013F000F8F7BDF9000606D520680DB0A9E73868F2
:101400000828E4D002E020680528E0D1256079466C
:101410003D600020C8F80010EFE70000971E002094
:10142000901E002004000010080000100C000010A6
:10143000480100102DE9F84F054600794C4C4D4FFE
:10144000DFF83481862608B11E2802D905202660DF
:101450004AE0288848F6AD614FF0140A884203D963
:101460002660C7F800A040E068884FF0170BB0F581
:10147000B46F03D32660C7F800B036E06846F9F7CA
:1014800003FB000667D42888BDF80010401A4FF40B
:10149000B46148435FEA0009E2D46846F9F704FB07
:1014A000000658D46888BDF80010411A11EB090FE6
:1014B000E0D432490120F9F704F900064BD4304951
:1014C0000220F9F7FEF8000645D468790F380D2898
:1014D00008D2DFE800F010101010100710101010E4
:1014E0000710100008202660386079468620C8F86A
:1014F0000010BDE8F88F2846F8F75BFE00062AD4F6
:10150000A81CF8F767FE000625D4281DF8F773FE1F
:10151000000620D4681DF9F712FB00061BD4002535
:1015200068460095F9F758FB000614D46846009504
:10153000F9F763FB00060ED40120ADF80000684601
:10154000F9F724FB000606D4ADF800506846F9F719
:101550002EFB000601D52068CBE7032009498DF852
:101560000000022008706846F8F7DFFDC1E70000C0
:1015700004000010080000100C000010741E002071
:10158000791E0020481E00202DE9F04F91B005A8DB
:10159000F9F7DFFAFA4C00067ED46846F9F700FB4B
:1015A0000006F9D4DFF8DCA34FF010014FF0020978
:1015B0009AF800004FF0000802074FF0010734D5F9
:1015C0009DF81400A0F10E020E2A6DD2DFE802F0A1
:1015D00007070F0F0F1C076C6C6C6C6C6C0F8AF894
:1015E00002008DF8141009E0ADF800905CE0BDF841
:1015F0000010032958D1401C8DF8140005A8F9F7F4
:101600009EFA0006C8D4EFE7BDF8000003284BD1CE
:101610009AF802008DF81400554605A8F9F78FFADC
:101620000006B9D4ADF800903CE0554640063BD5E5
:101630009DF814000E2804D00F2802D0102833D1B2
:1016400015E0BDF80020042A2ED18AF802008DF89A
:10165000141005A8F9F773FA00069DD41420ADF80C
:1016600000006846F9F792FA000695D41CE0BDF830
:101670000000032818D1ADF800706846F9F797FA12
:10168000A8788DF8140005A8F9F759FA000688D44F
:101690000420ADF8000000E05DE26846F9F776FA54
:1016A0000006AFD485F800809DF81420B64DB74EE3
:1016B00088214FF0640B4FF010401C2A72D2DFE8F3
:1016C00012F07100BB0464066406640664064206F8
:1016D00042064206420642064206420642061C00F6
:1016E0001C000E031604AB0382040C059F069F0624
:1016F0009F069F067100A304C102BDF800200A2ABC
:101700007BD007DCDAD2DFE802F04D1A51F29CBE42
:10171000D4E3F4FADFF878B25A2A67D008DC0B2A4F
:101720007ED00C2A7DD0392A7CD0402A3AD117E2CB
:101730005B2A78D0642A77D0B42AF7D124E0914983
:1017400012200EF05FFE000687D49AF800100120E8
:1017500001F048018AF8001004F042FF000684D42A
:101760009DF814000E280DD1694662200EF04AFE45
:1017700000068CD49DF80000C00703D0F3F78CFC62
:10178000000684D4B4202DE07E496920491C0EF067
:1017900039FE000685D49AF80100000603D504F04E
:1017A000CFFF60E2D5E2ADF80090F7E004F0CBFFA8
:1017B0000006C9D40EA92E200EF024FE0006C3D4C4
:1017C0009DF814000E2805D00F2810D19DF8380080
:1017D00080070CD5FFF7A8FC0006B5D420680528C3
:1017E00005D00A20ADF80000D8E006E000E10420B2
:1017F00041E200BFADF80070F5E30020FFF701FD06
:101800000006A1D42068002872D00EA92E200EF068
:10181000F9FD000698D49DF814000E280BD004E0C2
:1018200083E05CE0D5E033E1BEE00F28DFD19DF836
:1018300038008007DBD56B200DF00FFE00068ED43C
:10184000D5E70FA969200EF0A8FE000687D49DF801
:101850003C00C00603D404F0F8FF000689D46846B3
:10186000F9F7B4F9000684D4BDF80000042801D2C9
:10187000401CF4E3ADF800706846F9F798F90006EB
:1018800088D40520AEE704F0DDFF000691D4684659
:10189000F9F79CF900068CD4BDF800000228E7D3C4
:1018A000ADF800706846F9F782F9000687D4062083
:1018B00098E704F0D0FF00068FD46846F9F786F960
:1018C00000068AD4BDF800000428D1D3072089E798
:1018D0001B200DF0C2FD000693D40C2082E704F01B
:1018E000AEFF00068DD408207CE708E001E020E090
:1018F00057E004F0A1FF00068CD4092072E704F041
:1019000098FF000686D40EA92E200EF07BFD00065F
:1019100095D49DF814000E2805D00F287ED19DF88F
:10192000380080077AD50B205CE70220FFF769FCBE
:101930006FE204F011FF000688D40EA92E200EF0ED
:1019400061FD00068AD49DF814000E2805D00F28EA
:101950007DD19DF83800800779D50E4D01206F812B
:101960002AF09CF800068BD456200DF076FD000678
:1019700086D4A5F80A9002202AF090F8F3E300003C
:10198000040000106C1E0020080000100C00001065
:101990000000094008230010ADF800B06846F9F7D0
:1019A000F5F811B0BDE8F08F2AF08EFC000688D45F
:1019B0002068052804D09DF814000E2807D079E18E
:1019C000C4F800807846C5F8008030602FE35A20C4
:1019D00008E7F8F7F5F8000684D4FDF70BFD0006DC
:1019E0007ED4F8F753F975E32760C5F8008025E148
:1019F0006846F9F7DEFB000684D49DF8000038B392
:101A0000FD484FF05B09007800283FF4CCAE6846F3
:101A1000F8F75FFB00068FD4F84800E066E2007834
:101A2000D8B19DF800001B2817D06846F9F75EF87A
:101A3000000687D46F46B81CF9F769F8000692D4FF
:101A4000381DF9F775F800068DD4684601E079E392
:101A50007BE001F01DFD000685D46946042003F0FB
:101A60000DFA000684D4BDF80000401C80B201F0DD
:101A70000BFF50B192286ED1F2F7D8FB13208DF8EE
:101A800000006846F8F71BFBF7E3ADF80090FEE2B4
:101A9000D948007828B30121D94804F02AFE00066D
:101AA00085D401F068FF000696D4D54890F8400030
:101AB000002885D16846F8F70CFB00068CD49DF809
:101AC00000000E283DD06846F9F710F8000693D4C0
:101AD000DAF8081001919AF80C108DF8081001E05E
:101AE000F2E039E0DAF80D10CDF809109AF811009B
:101AF0008DF80D0004200DF1020103F0BFF900067E
:101B000089D4BDF80200401CADF80200112003F09A
:101B1000CAFB00068DD46946022003F0D4FB000600
:101B200087D4122003F0BFFB000688D4022003F004
:101B300086F9000688D46946022003F044F90006BD
:101B40008AD4FEF7DDFE000686D4DBF808104020BC
:101B5000CAF8041046E683E2A94981F84080A9E763
:101B6000DBF80810DAF80400081AA649884203D204
:101B7000A548007801289CD1C1468DF800806846B0
:101B8000F8F77BFA00068BD4B84638460DF11C0BEB
:101B9000C7B269463846F8F794FD000684D4C7EB0F
:101BA000C70101EB0B0AAAF107013846F8F74EFA14
:101BB00000068CD4AAF107006946F7F7D8FD0006A5
:101BC00085D47F1CF8B20428E2D907A8F8F733FAC5
:101BD000000695D406A8F9F7ECFA000690D49DF813
:101BE000180018B9F9F701FB000689D469461220DC
:101BF0000EF008FC00068DD49DF8000040070AD5C1
